:020000040800F2
:1000000000000120ED440008892700088B27000824
:100010008D2700088F2700089127000800000000A6
:10002000000000000000000000000000932700080E
:10003000952700080000000097270008992700086E
:100040003D4500083D4500089D2700083D45000846
:100050003D4500083D450008A9270008AF270008D6
:100060003D4500083D450008E12700083D450008E2
:10007000B5270008B7270008B9270008C5270008DA
:10008000D1270008DD2700083D4500083D45000850
:10009000000000003D450008E32700083D4500083A
:1000A0003D4500083D4500083D4500083D45000828
:1000B0003D4500083D4500083D4500083D45000818
:1000C0003D4500083D4500083D4500083D45000808
:1000D0003D450008ED2700083D4500083D45000866
:1000E0003D450008E9270008F92700083D450008BC
:1000F0003D45000800000000000000003D450008EC
:100100003D4500083D450008052800083D4500081C
:100110003D4500083D4500083D4500083D450008B7
:100120003D4500083D4500083D4500083D450008A7
:080130003D4500083D450008B3
:1001380010B5054C237833B9044B13B10448AFF319
:1001480000800123237010BD4C0100200000000036
:100158004013010808B5034B1BB103490348AFF32B
:10016800008008BD00000000500100204013010875
:1001780014214160704714207047406A704700009E
:10018800790100087F01000883010008990100082F
:1001980010B5044604F1100000F05CFCC4F8F80047
:1001A8000148C4F87C0110BD88010008F8B5E6B024
:1001B80004460D4616461F460A4906A800F0CAFE20
:1001C80070996F9A05910492009733466E996D9ACB
:1001D800039102922A466C990191214600F060F839
:1001E80067B0F0BD94010008F8B5E6B004460D46C6
:1001F80016461F46094906A800F0ACFE6F996E9A8C
:100208000491039200976D996C9A0291019233467A
:100218002A46214600F087F867B0F0BD940100082F
:1002280038B500281CBF01680029184A23D1184B8B
:100238001C684FF6F0710C404CF24025AC421FBFD1
:100248001B6819404CF27024A14212D1114D296843
:1002580079B911490B68C3F30B03B3F58A6F1FBF54
:100268000968C1F30B0140F28343994204BF01219D
:10027800117028B905E0094B994204BF012111709A
:100288004068BDE8324001F09FBE00BF6801002011
:1002980000ED00E0002004E00010005C000037489A
:1002A8002DE9F04104460D46216816464A681F4666
:1002B80090478046B8F5403F2ED122680A99936846
:1002C800204698478046B8F5403F25D12368089ACC
:1002D8000799D3F80CC02046E0478046B8F5403F60
:1002E8001AD12368069A39461F692046B8478046BE
:1002F800B8F5403F10D1236829465D69324620464B
:10030800A8478046B8F5403F06D123680B9A09995B
:100318009D692046A847804621680A68204690477C
:100328004046BDE8F0812DE9F04104460D462168BC
:1003380016464A681F4690478046B8F5403F2ED17A
:1003480022680A999368204698478046B8F5403F46
:1003580025D12368089A0799D3F80CC02046E047AE
:100368008046B8F5403F1AD12368069A39461F6976
:100378002046B8478046B8F5403F10D12368294643
:100388005D6932462046A8478046B8F5403F06D109
:1003980023680999DD6900222046A847804621681C
:1003A8000A68204690474046BDE8F0814FF4403047
:1003B80070470000F0B50C4685B0114600281A4673
:1003C8001CBF0568002D0B4B11D082B104B971B95F
:1003D8000D9860B10F9E0E9F0A9B0290049603979A
:1003E8000B980C9E009001962046A8470346184695
:1003F80005B0F0BD020003002DE9F04F0646D0B06D
:100408000868F56DD6F860E0726EB76EF36E00BAE4
:1004180000906C46486800BA60600DF14008886832
:1004280000BAA060C86800BAE060086900BA206134
:10043800486900BA6061886900BAA061C86900BAF1
:10044800E061086A00BA2062486A00BA6062886A95
:1004580000BAA062C86A00BAE062086B00BA2063FA
:10046800486B00BA6063886B00BAA063C86B00BAB7
:10047800E063402058F80C1C58F820CC58F838ACE9
:100488008CEA010158F840CC8AEA01018CEA01099A
:100498004FEAF979401E48F8049BEBD187EA02003D
:1004A80000EA0E00784010EBF5610098DFF824C4EC
:1004B80041186144C81882EABE032B404FEAF06134
:1004C80053405918636859186144CF194FEAB50366
:1004D80083EABE01014081EABE0111EBF765A1681C
:1004E8004D196544A91883EAB0023A404FEAF1650C
:1004F8005A405519E26855194FEAB70282EAB0071F
:1005080065440F4005EBBE0E97EAB00717EBFE6592
:1005180027697D194FEAB10782EA0701654401EAB4
:100528000E01EB18514011EBF36561694D194FEA63
:10053800BE0187EA010E65440EEA030E15EBB00012
:100548008EEA070E0EEBF065D4F818E075446544A2
:10055800AA1881EAB30505404FEAF26E4D40AE4451
:10056800E569AE44E64477444FEAB00080EAB30E4A
:100578000EEA020E8EEAB30E0EEBF765D4F820E011
:1005880075446544691880EAB2053D404FEAF16E4A
:100598004540AE44656AAE44E6440EEBB3034FEA09
:1005A800B70787EAB20E0EEA010E8EEAB20E0EEB1C
:1005B800F365D4F828E075446544281887EAB1053E
:1005C8001D404FEAF06E7D40AE44E56AAE44E64415
:1005D8000EEBB2024FEAB30383EAB10E0EEA000E45
:1005E8008EEAB10E0EEBF265D4F830E0754465443E
:1005F800EF1983EAB00515404FEAF76E5D40AE4447
:10060800656BAE44E6440EEBB1014FEAB20282EAF2
:10061800B00E0EEA070E8EEAB00E0EEBF165D4F8B6
:1006280038E075446544EB1882EAB7050D404FEA97
:10063800F36E5540AE44E56BAE44E6440EEBB000B5
:100648004FEAB10181EAB70E0EEA030E8EEAB70E41
:100658000EEBF065D4F840E07544654481EAB30ECA
:10066800AA180EEA000E4FEAF2658EEA010E7544EA
:10067800DDF844E04FEAB000754480EAB30E654403
:100688000EEA020E15EBB7078EEAB30E0EEBF7650E
:10069800DDF848E04FEAB202754480EA020E65448C
:1006A8000EEA070E69188EEA000E0EEBF165DDF80A
:1006B8004CE07544654405EBB3034FEAB70E1427C5
:1006C8000DF1500CDFF810528EEA010B82EA0B0B89
:1006D8000BEBF36A5CF804BBDA44AA44504483EA9F
:1006E800B10B4FEAF06A8EEA0B0BDA445CF804BBF4
:1006F800DA44AA44524480EAB30B4FEAF26A8BEA1E
:10070800B10BDA445CF804BBDA444FEAB000AA44FF
:1007180080EA020BD6448BEAB30B0BEBFE6A5CF85B
:1007280004BBDA444FEAB202AA4482EA0E0B0AEB8F
:10073800B10180EA0B0B0BEBF16A5CF804BBDA44FD
:100748007F1DAA44282F0AEBB3034FEABE0EBBD382
:100758003C2F61D3502F4DD204EB870CC7F15407BF
:100768005E4CA7FB04A504465D4FA8088EEA010A63
:1007780082EA0A0A5CF804BB0AEBF3655D447D195A
:100788002C1983EAB10A4FEAF4658EEA0A0A55443D
:100798005CF804AB5CF804BB55447D19AA1884EADC
:1007A800B30A4FEAF2658AEAB10A55445D444FEA52
:1007B800B4047D1984EA020AAE448AEAB30A0AEB51
:1007C800FE655CF804AB55444FEAB2027D1982EA33
:1007D8000E0A15EBB10184EA0A0A5CF804BB0AEBBD
:1007E800F1655D447D1915EBB303401E4FEABE0E5B
:1007F800BCD12046F46D1B19F365336EC9183166F8
:10080800716E71447166B36ED218B266F16E40189B
:10081800F06650B0BDE8F08F4EEA010B0EEA010A0F
:100828000BEA020B4BEA0A0A0AEBF36554F827A015
:10083800DFF8B0C0554443EAB10B654403EAB10A96
:100848000BEA0E0B28184BEA0A0A7F1C0AEBF06524
:1008580054F827A0554440EAB30B654400EAB30AAC
:100868000BEAB10BAA184BEA0A0A7F1C0AEBF265DD
:1008780054F827A055444FEAB00040EA020B6544FB
:1008880000EA020A0BEAB30BAE444BEA0A0A7F1CE1
:100898000AEBFE6554F827A055444FEAB20242EA33
:1008A8000E0B654402EA0E0A0BEA000B15EBB101C8
:1008B8004BEA0A0A7F1C0AEBF16554F827A0554455
:1008C8007F1C65443C2F05EBB3034FEABE0EA3D350
:1008D80040E700BF9979825AA1EBD96ECDCCCCCC38
:1008E800D6C162CADCBC1B8F00B581B00168074A5B
:1008F800914200D110B9064801B000BD7C2110F02A
:1009080083FC4FF4003001B000BD00BFFC090008B3
:10091800030002002DE9F0410B4A92E8F85188B033
:10092800694681E8F8510268084B9A4200D118B923
:10093800074808B0BDE8F0811422083000F04FFBEA
:1009480008B0BDE8F08100BFDC090008FC09000818
:1009580003000200152904D20268044B9A4200D110
:1009680008B903487047083000F048BBFC09000884
:100978000300020010B481B013460268074CA2427B
:1009880000D118B901B010BC0548704701B000F19A
:10099800240210BC083000F035BB00BFFC09000879
:1009A8000300020010B481B013460268074CA2424B
:1009B80000D118B901B010BC054870470A4601B00B
:1009C80000F1240110BC083000F070BBFC090008DD
:1009D800030002000123456789ABCDEFFEDCBA981E
:1009E80076543210F0E1D2C300000000000000008D
:1009F80000000000F10800081D0900085D09000852
:100A08007D090008AD09000801040008790F0008F5
:100A1800C50F0008810F0008F0B5A3B004460B48C5
:100A280002900D4616461F46094B0822402104A88D
:100A380000F0D1FA28980190009733462A462146BB
:100A480002A800F01BF823B0F0BD00BFFC090008A5
:100A5800100A000810B5040008BF002408D0054893
:100A6800054B20600822402104F1080000F0B3FA89
:100A7800204610BDFC090008100A00082DE9F041C5
:100A880004460E46216817464A681D469047804628
:100A9800B8F5003F19D1226806999368204698470F
:100AA8008046B8F5003F10D123683146DE683A46E3
:100AB8002046B0478046B8F5003F06D12368079A1C
:100AC80029461D692046A847804621680A682046AD
:100AD80090474046BDE8F08110B500F033FA4FF476
:100AE800403400280EBF034C4FF4C07110F08CFB4B
:100AF800204610BD0200030010B5044600F022FA9B
:100B080008B9054810BD0021A160D0F87C21116802
:100B180088474FF4403010BD0200030070B504460A
:100B28000D4600F00FFA064E40B1D0F87C0141683E
:100B38008847A84224BF65604FF44036304670BDF0
:100B4800020003002DE9FF4715000C4600D02CB128
:100B5800064600F0F7F95FEA000801D16448C3E0EF
:100B6800D8F8F80001684A689047B0F5003F17D1F7
:100B7800D8F87C118A68404690478146B9F1810FC0
:100B880080F09E80A94508F1FC0A17D2D8F8F80031
:100B98000368D3F80CC02A462146E047B0F5003F69
:100BA80040F08E80D8F8F8000368D3F810C06A4681
:100BB8005146E047B0F5003F76D10AE0002004E056
:100BC800215C0AF800100098401C00900098A84288
:100BD800F6D34FF0000C4749474A484B01AC009800
:100BE800844558D2D3E9007001ADC5E9007010788A
:100BF80000281ABF042086464FF0000E085854F803
:100C08000E5028443E4D05600127D0F800E087606B
:100C1800019D4F681AF80C007D408EEA050585F0A5
:100C2800040E65680F687D4085F0FC05754485F005
:100C3800A30568400AF80C000CF1010CCFE7D3E9D2
:100C4800004501A8C0E9004510782E4D002814BFC2
:100C58004FF0040E4FF0000E01A8744651F80EE054
:100C68000459A6440127CEF80050DEF80040CEF81B
:100C780008704D68019F40687D406C400D68684071
:100C880084F0040480F0FC00041984F057040AF886
:100C98000C400CF1010CCC45D1D3D8F8F800016810
:100CA8004A689047B0F5003F0AD1D8F8F8000368C1
:100CB800D3F80C804A465146C047B0F5003F01D0F2
:100CC800114811E0002006E05AF8201081F06A313E
:100CD8004AF82010401CB0EB990FF5D3B06840F0EB
:100CE8000100B0604FF4403004B0BDE8F08700BFA9
:100CF80002000300D813010868010020240F00082F
:100D0800ADBE4ED70DBE75A10100030038B50C4627
:100D1800017A1546CA0702D500F014F908B908483F
:100D280032BDD0F8F80003682146DC682A46A0479F
:100D3800B0F5003F01D0034832BD4FF4403032BD1A
:100D480002000300010003002DE9F84191B00546B7
:100D58000E461746402101A810F056FA297AC8070E
:100D680004D5284600F0EEF8040002D1DFF8A4808C
:100D78004BE0D4F8F800DFF8A0800368D3F810C07F
:100D88006A4601A9E047B0F5003F3ED1D4F8F80023
:100D980001684A689047B0F5003F36D1D4F87C1115
:100DA8008A6820469047D4F8F830024618461B68EF
:100DB800D3F80CC004F1FC01E047B0F5003F24D1A2
:100DC800D4F87C0141688847D4F8F83002461846C0
:100DD8001B68D3F80CC001A9E047B0F5003F14D157
:100DE800D4F8F8000268696893689847B0F5003F3E
:100DF8000BD1D4F8F80003681C693A463146A0477D
:100E0800B0F5003F08BF4FF44038404612B0BDE887
:100E1800F08100BF02000300010003002DE9F84142
:100E2800A5B0074688461646402115A810F0ECF9EB
:100E380000220492402105A810F0E6F9387AC1078B
:100E48005ED5384600F07EF8050059D0D5F8F80090
:100E58002D4C0368D3F810C06A4605A9E047B0F5E1
:100E6800003F3CD1D5F8F80001684A689047B0F5D2
:100E7800003F34D1D5F87C118A6828469047D5F8C8
:100E8800F830024618461B68D3F80CC005F1FC017F
:100E9800E047B0F5003F22D1D5F87C01416888478A
:100EA800D5F8F830024618461B68D3F80CC005A9D7
:100EB800E047B0F5003F12D1D5F8F800026879682C
:100EC80093689847B0F5003F09D1D5F8F800036852
:100ED8001D6904AA15A9A847B0F5003F01D020460E
:100EE8000FE00A4B0A490B4A0396029101924046C9
:100EF8001C68049B009415AA796800F0E5F900E0E5
:100F0800054826B0BDE8F08101000300E0130108A0
:100F1800936E030026C703000200030004B001011A
:100F280000170145E10A0008010B0008250B00081D
:100F3800B50300084D0B0008150D0008510D0008F9
:100F4800250E00080168024A914218BF0020704728
:100F58002C0F000810B5040008BF002404D0034873
:100F68002060204609688847204610BD2C0F0008DD
:100F780020225C3010F046B9F0B58468A30800223E
:100F880004F0030407E000F15C0555F8226035BA67
:100F980041F82250521C9A42F5D300220BE000F18E
:100FA8005C0502EB830755F82360D500C5F11805E9
:100FB800EE40CE55521CA242F1D3F0BD30B5C46804
:100FC80003690022E31AD5188C5C0544521C082AD0
:100FD8002C77F8D330BD0360C1600261704738B523
:100FE800044615460022626023685A68904700202C
:100FF8006061A061A5604FF4003032BD81604FF49C
:10100800003070472DE9F84304462079D4F80C8065
:10101800450748BF244845D466691D46A8F1010024
:1010280000EAD60306EBC506B6EBC50F666102D229
:10103800A669761CA6611746A66906EB5576A661D1
:101048000E46E918884225D2A8EB03094A463146DC
:10105800F81810F0D7F82268136839460FE04246AE
:10106800384610F0CFF823681A683946204690476A
:1010780007E0311811F00300F1D122681368204607
:101088009847484600EB0809A9F10101A942F0D3A5
:10109800002300E000202A1A3118F81810F0B2F8DE
:1010A8004FF40030BDE8F283040002002DE9FC4F44
:1010B800024685B0D0681369DFF86CC1DFF86C812F
:1010C800A0EB030A506840F004005060002703A812
:1010D80002900DF10C0ED8E9003403A8544DC0E974
:1010E80000342878534D00280CBF00230423994668
:1010F8005CF803305EF80940234401261D601C6833
:101108009E60DCF80430039DDCF80090DEF8046093
:101118005D406540484C654089EA0606474C664094
:101128007519474C6540D8E9006B03AC0028C4E941
:10113800006B0EBF002404200424029E5CF800000B
:10114800345920183F4C04600126046886600398CF
:10115800029E43406340384C7068634089EA00004F
:10116800364C6040034438484340280018BF0120EB
:101178005B1E9B41042F2CBFC0B2D80F02F1140391
:1011880053F8200007F00303C3F10303DB00D84042
:101198000DF807007F1C082F9DD315460C466A6979
:1011A800AB69E868D20842EA4372401E00EA0207C7
:1011B800002302409B420AD8524508D28020E055BD
:1011C8007F1C574516D2AAEB0701E01910E08020D2
:1011D800E05500E0E355E8687F1C8742FAD32A68A7
:1011E800136828469847BAF1000F03D051462046A5
:1011F80010F00AF82A68069E059F936869462846F3
:1012080098472A68D2F8009021462846C8472B6894
:10121800DA683946284690470EB1A86830604FF41E
:10122800003007B0BDE8F08FD81301085412000849
:10123800680100205FC5109304850012FC68017ADC
:10124800C0F524FF24AF33D426AF698B04B0010165
:1012580000170145F8B501240094002300240DE08F
:10126800009D065D0F5D7E40F643761CF60F86F006
:10127800010635400095641C009DEB189442EFD39D
:101288001846F2BDF8B5002301240094002A11E0A5
:10129800009C85188F1815F8016C17F8015C6E40D2
:1012A800F643761CF60F86F0010634400094009C45
:1012B800E318521EECD11846F2BD00005D1200087A
:1012C8008D120008010000002DE9F84F1D46DDF8D9
:1012D80028900B9F0D9C4FF0FF3300930E469246CB
:1012E800D9F800B0804632465146D847834664B3A1
:1012F800D9F8043032465146404698476FEA0B0207
:10130800521C42EA0B0200996FEAD2735B1C194027
:10131800C2430091521C024300996FEAD2735B1CCE
:101328001940009186F05531484087EA000181F064
:101338005531216080F05531C943491C0843009A52
:101348006FEAD070401C82430092D9F80800012847
:1013580009D17540E943491C0D4300986FEAD572DD
:10136800521C90430AE0F11C85EA9102D243521CB8
:10137800154300986FEAD5735B1C984386F0AA362C
:10138800009086EA0B0686F0AA33F243DB430C98FA
:10139800C2F3C0725B1C42EAD3720099D243521C5A
:1013A80091430091774000998843009987F0AA37C4
:1013B8000F403843BDE8F28F034613F8012B002A8B
:1013C800FBD1181A0138704781F0004102E000BFD4
:1013D80083F0004330B54FEA41044FEA430594EAED
:1013E800050F08BF90EA020F1FBF54EA000C55EA28
:1013F800020C7FEA645C7FEA655C00F0E2804FEAF9
:101408005454D4EB5555B8BF6D420CDD2C4480EADA
:10141800020281EA030382EA000083EA010180EA0A
:10142800020281EA0303362D88BF30BD11F0004F58
:101438004FEA01314FF4801C4CEA113102D040428E
:1014480061EB410113F0004F4FEA03334CEA1333C9
:1014580002D0524263EB430394EA050F00F0A780E1
:10146800A4F10104D5F1200E0DDB02FA0EFC22FADC
:1014780005F2801841F1000103FA0EF2801843FAD0
:1014880005F359410EE0A5F120050EF1200E012AC1
:1014980003FA0EFC28BF4CF0020C43FA05F3C018FF
:1014A80051EBE37101F0004507D54FF0000EDCF178
:1014B800000C7EEB00006EEB0101B1F5801F1BD321
:1014C800B1F5001F0CD349085FEA30004FEA3C0C25
:1014D80004F101044FEA445212F5800F80F09A801B
:1014E800BCF1004F08BF5FEA500C50F1000041EB1F
:1014F800045141EA050130BD5FEA4C0C404141EB23
:101508000101013C28BFB1F5801FE9D291F0000F1D
:1015180004BF01460020B1FA81F308BF2033A3F1CC
:101528000B03B3F120020CDA0C3208DD02F1140CC3
:10153800C2F10C0201FA0CF021FA02F10CE002F1FE
:101548001402D8BFC2F1200C01FA02F120FA0CFCF7
:10155800DCBF41EA0C019040E41AA2BF01EB045140
:10156800294330BD6FEA04041F3C1CDA0C340EDC3E
:1015780004F11404C4F1200220FA04F001FA02F381
:1015880040EA030021FA04F345EA030130BDC4F13F
:101598000C04C4F1200220FA02F001FA04F340EA34
:1015A8000300294630BD21FA04F0294630BD94F0E5
:1015B800000F83F4801306BF81F480110134013DCC
:1015C8004EE77FEA645C18BF7FEA655C29D094EA3D
:1015D800050F08BF90EA020F05D054EA000C04BFBB
:1015E8001946104630BD91EA030F1EBF00210020A6
:1015F80030BD5FEA545C05D14000494128BF41F045
:10160800004130BD14F580043CBF01F5801130BDA8
:1016180001F0004545F0FE4141F470014FF0000033
:1016280030BD7FEA645C1ABF194610467FEA655CE4
:101638001CBF0B46024650EA013406BF52EA033586
:1016480091EA030F41F4002130BD00BF90F0000F74
:1016580004BF0021704730B54FF4806404F13204B0
:101668004FF000054FF0000150E700BF90F0000F69
:1016780004BF0021704730B54FF4806404F1320490
:1016880010F0004548BF40424FF000013EE700BF60
:1016980042004FEAE2014FEA31014FEA02701FBFF0
:1016A80012F07F4393F07F4F81F06051704732F022
:1016B8007F4208BF704793F07F4F04BF41F4002179
:1016C800704730B54FF4607401F0004521F00041D7
:1016D8001CE700BF50EA010208BF704730B54FF061
:1016E80000050AE050EA010208BF704730B511F062
:1016F800004502D5404261EB41014FF4806404F19A
:1017080032045FEA915C3FF4D8AE4FF003025FEA1F
:10171800DC0C18BF03325FEADC0C18BF033202EBA3
:10172800DC02C2F1200300FA03FC20FA02F001FAFD
:1017380003FE40EA0E0021FA02F11444BDE600BFA0
:101748004FF0FF3C06E000BF4FF0010C02E000BF85
:101758004FF0010C4DF804CD4FEA410C7FEA6C5C68
:101768004FEA430C18BF7FEA6C5C1BD001B050EA0B
:10177800410C0CBF52EA430C91EA030F02BF90EAF6
:10178800020F0020704710F1000F91EA030F58BFB5
:10179800994208BF90422CBFD8176FEAE37040F017
:1017A800010070474FEA410C7FEA6C5C02D150EAB5
:1017B800013C07D14FEA430C7FEA6C5CD6D152EA70
:1017C800033CD3D05DF8040B704700BF8446104635
:1017D80062468C461946634600E000BF01B5FFF734
:1017E800B7FF002848BF10F1000F01BD4DF808ED04
:1017F800FFF7F4FF0CBF012000205DF808FB00BFD5
:101808004DF808EDFFF7EAFF34BF012000205DF82E
:1018180008FB00BF4DF808EDFFF7E0FF94BF01207B
:1018280000205DF808FB00BF4DF808EDFFF7CEFF7C
:1018380094BF012000205DF808FB00BF4DF808EDBB
:10184800FFF7C4FF34BF012000205DF808FB00BF8C
:101858004FEA410212F5001215D211D56FF47873D0
:10186800B3EB625212D94FEAC12343F0004343EA73
:10187800505311F0004F23FA02F018BF404270474E
:101888004FF00000704750EA013005D111F00040D8
:1018980008BF6FF0004070474FF00000704700BF6E
:1018A80080F0004002E000BF81F0004142001FBF0D
:1018B8005FEA410392EA030F7FEA226C7FEA236C16
:1018C8006AD04FEA1262D2EB1363C1BFD21841400B
:1018D80048404140B8BF5B42192B88BF704710F0A1
:1018E800004F40F4000020F07F4018BF404211F044
:1018F800004F41F4000121F07F4118BF494292EAAC
:10190800030F3FD0A2F1010241FA03FC10EB0C00D7
:10191800C3F1200301FA03F100F0004302D5494264
:1019280060EB4000B0F5000F13D3B0F1807F06D311
:1019380040084FEA310102F10102FE2A51D2B1F109
:10194800004F40EBC25008BF20F0010040EA0300FE
:101958007047490040EB0000013A28BFB0F5000F7E
:10196800EDD2B0FA80FCACF1080CB2EB0C0200FA34
:101978000CF0AABF00EBC25052421843BCBFD04083
:101988001843704792F0000F81F4000106BF80F4FD
:1019980000000132013BB5E74FEA41037FEA226CC0
:1019A80018BF7FEA236C21D092EA030F04D092F08B
:1019B800000F08BF0846704790EA010F1CBF0020BF
:1019C800704712F07F4F04D1400028BF40F000401C
:1019D800704712F100723CBF00F50000704700F03C
:1019E800004343F0FE4040F4000070477FEA226263
:1019F80016BF08467FEA23630146420206BF5FEA34
:101A0800412390EA010F40F4800070474FF0000333
:101A180004E000BF10F0004348BF40425FEA000CFA
:101A280008BF704743F0964301464FF000001CE0A2
:101A380050EA010208BF70474FF000030AE000BFF8
:101A480050EA010208BF704711F0004302D5404236
:101A580061EB41015FEA010C02BF844601460020A8
:101A680043F0B64308BFA3F18053A3F50003BCFAC3
:101A78008CF2083AA3EBC25310DB01FA02FC634470
:101A880000FA02FCC2F12002BCF1004F20FA02F277
:101A980043EB020008BF20F00100704702F120026A
:101AA80001FA02FCC2F1200250EA4C0021FA02F2CB
:101AB80043EB020008BF20EADC7070474FEA40029F
:101AC800B2F1FE4F0FD34FF09E03B3EB12620DD964
:101AD8004FEA002343F0004310F0004F23FA02F0CE
:101AE80018BF404270474FF00000704712F1610F75
:101AF80001D1420205D110F0004008BF6FF000404C
:101B080070474FF00000704753B94AB9002908BF21
:101B180000281CBF4FF0FF314FF0FF3000F070B9C4
:101B2800ADF1080C6DE904CE00F006F8DDF804E02C
:101B3800DDE9022304B070472DE9F047089E0D4601
:101B480004460F46002B4AD18A42944665D9B2FA18
:101B580082F343B102FA03FCC3F120029F4020FA4A
:101B680002F217439C404FEA1C4E1FFA8CF5B7FB54
:101B7800FEF1220C0EFB117742EA074201FB05F049
:101B880090420AD91CEB020201F1FF3780F01B8159
:101B9800904240F2188102396244121AA4B2B2FB90
:101BA800FEF00EFB102244EA024400FB05F5A542B4
:101BB8000AD91CEB040400F1FF3280F00681A5422B
:101BC80040F203816444023840EA0140641B00216A
:101BD8001EB1DC400023C6E90043BDE8F0878B4214
:101BE80008D9002E00F0EC800021C6E9000508465F
:101BF800BDE8F087B3FA83F1002949D1AB4202D39B
:101C0800824200F2F780841A65EB0302012017462E
:101C1800002EE2D0C6E90047DFE702B9FFDEB2FADC
:101C280082F3002B40F08F808A1A4FEA1C471FFA74
:101C38008CFE0121B2FBF7F507FB1520220C42EAC6
:101C480000420EFB05F0904208D91CEB020205F198
:101C5800FF3802D2904200F2CA804546121AA4B256
:101C6800B2FBF7F007FB102244EA02440EFB00FE29
:101C7800A64508D91CEB040400F1FF3202D2A645A0
:101C880000F2BA801046A4EB0E0440EA05409FE734
:101C9800C1F120078B4022FA07FC4CEA030C05FA35
:101CA80001F420FA07F3FD40234300FA01F94FEA53
:101CB8001C401FFA8CFEB5FBF0F81C0C00FB1855F5
:101CC80044EA054408FB0EF5A54202FA01F20BD9D5
:101CD8001CEB040408F1FF3A80F08780A54240F22B
:101CE8008480A8F102086444641B9DB2B4FBF0F33D
:101CF80000FB134445EA044403FB0EFEA64508D93D
:101D08001CEB040403F1FF306BD2A64569D9023BF2
:101D1800644443EA0840A0FB0283A4EB0E049C42FF
:101D2800C6461D4655D352D056B1B9EB0E0364EBE7
:101D3800050404FA07F7CB40CC401F43C6E90074FA
:101D48000021BDE8F087C3F1200102FA03FC20FA64
:101D580001F225FA01F19D402A434FEA1C471FFA78
:101D68008CFEB1FBF7F007FB1015110C41EA054199
:101D780000FB0EF58D4204FA03F408D91CEB0101AF
:101D880000F1FF382FD28D422DD902386144491B0A
:101D980092B2B1FBF7F507FB151142EA014205FBC8
:101DA8000EF1914208D91CEB020205F1FF3816D258
:101DB800914214D9023D6244521A45EA004139E77A
:101DC8003146304609E73946E7E61046FCE6C145A4
:101DD800AAD2B8EB020E63EB0C050138A4E745461E
:101DE800EAE7034695E74046D1E7D0467CE7023D5F
:101DF800624433E708460BE76444023843E700BF10
:101E0800704700BF1348144A08B54FF00043C0E9B3
:101E180000230422002342610122C2614FF4805151
:101E280007220383C0E90233C0E90933C0E90C1271
:101E38000361837680F8203080F82C30826380F844
:101E48003C30C36402F0DEFB18B1BDE8084000F086
:101E5800F3BB08BD6C010020002401400268084B58
:101E68009A4282B00AD14FF0B0431A6E42F400721F
:101E78001A661B6E03F400730193019B02B070474E
:101E8800002401400268054B9A4201BF4FF0B0425E
:101E9800136E23F400731366704700BF00240140DB
:101EA80030B585B000240546CDE901440394FFF719
:101EB800A9FF144802F03EFF08B100F0BDFB11482D
:101EC800039401A9CDE9015402F0FAFC08B100F02D
:101ED800B3FB0C4802F058FE08B100F0ADFB4FF020
:101EE800FF31084802F08EFC064802F005FF05485D
:101EF80002F0E2FC0446034802F0A8FE204605B0C2
:101F080030BD00BF6C010020014B024A1A607047C7
:101F18006C0100200024014008B50948FFF7C0FF04
:101F280068B1084BB3F8AA304FF6FF72934216BF58
:101F380040F6E442044B5343B3FBF0F398B208BDB8
:101F4800002000B40075FF1FD8084C0013B500230B
:101F5800ADF80630FFF7E0FF04461948FFF7A0FF89
:101F6800184BB3F8C820B3F8A8108A4204FB00F055
:101F780018D040F6E443B0FBF3F364205B1A434304
:101F8800521A93FBF2F31E331BB2ADF80630BDF8BC
:101F980006305BB21B02ADF80630BDF8060000B291
:101FA80002B010BD4FF47A7240F6FF73B0FBF3F342
:101FB8005343A3F53923A3F50C6340F6C412E0E7B5
:101FC800001000B00075FF1F4FF0B04382B09A6A4E
:101FD80022F480529A629A6C42F480529A649B6C02
:101FE80003F480530193019B002002B070474FF027
:101FF800B04382B09A6C02439A649B6C034001938D
:10200800019B02B0704708B50420FFF7F0FF0120DC
:10201800FFF7EDFF0220FFF7EAFF002211460B2031
:1020280002F026FF0B2002F055FF002211460C207B
:1020380002F01EFF0C2002F04DFF002211460D2079
:1020480002F016FF0D2002F045FF002211460E2077
:1020580002F00EFF0E2002F03DFF002211460F2075
:1020680002F006FF0F2002F035FF00221146102073
:1020780002F0FEFE102002F02DFF00221146112072
:1020880002F0F6FE112002F025FF0022362011464C
:1020980002F0EEFEBDE80840362002F01BBF00004B
:1020A80008B503F05FF910B16FF0040008BD064BE6
:1020B8009A6942F040429A614CF2FA321A6103F08E
:1020C80063F90028F2D0EFE700400058F0B585B07A
:1020D80000230C4600930646A8B3FFF7E1FF054628
:1020E80070BB03F03FF988BB1A481B4A02230193CF
:1020F800D0F8E01506F1784302EA8121B3FBF1F745
:1021080001FB1733DB0A0293D0F8E00504F17841AC
:102118000139314402EA8022B1FBF2F002FB1011CE
:10212800C3EBD1230133694601A8039303F0ACF94B
:1021380020B102280CBF01256FF0010503F024F936
:10214800284605B0F0BD6FF00505F9E76FF0040506
:10215800F6E700BF0070FF1F00FCFF03014B18608B
:1021680000207047D00100202DE9F04F89B0B0F170
:10217800006F06460F460092C0F0C580DFF89881D0
:10218800664DD8F8E03505EA832303F10063013B87
:10219800984200F2B880002800F0B880002900F0CA
:1021A800B58040EA02035B0740F0B080FFF778FF94
:1021B8000446A0BB03F0D6F8002840F0AA80D8F85F
:1021C800E01506F1784205EA8121B2FBF1F301FB43
:1021D8001322009B03F17843013B3344B3FBF1F036
:1021E80001FB1033DB0A01334FEAD22AA3EBD222D8
:1021F800012A039388BFC6F30A050AF58038C6F199
:10220800080398BF009D069388BFC5F500654FEA8F
:10221800C828B346039B9A4505D303F0B5F8204672
:1022280009B0BDE8F08FA6F10803069A1A44954252
:1022380019D804950197CDF814B04FF00009059B03
:1022480009EB0301049B99453ED3009BAB442F4403
:102258005D1BB5F5006F28BF4FF400650AF1010A50
:1022680008F50068D6E753F8081F5A68B2F1FF3F2F
:1022780008BFB1F1FF3FD8D0294B186810B96FF0EB
:102288000504CAE7B8F1000F04D04FF400624146D4
:102298000EF054FBDFF88890D9F80030CBF30A0031
:1022A80039461844AAB20EF049FB4FF40061404683
:1022B800FFF70CFF08BBD9F8003001934FF4006317
:1022C800CDF814800493B8E7019B07914B4402931F
:1022D8000120D3E9002303F091F888B90799019BFD
:1022E800D1E9000259F80310029B5B689A4208BFC3
:1022F800884205D109F10809A1E76FF001048CE7CC
:102308006FF0030489E74FF0FF3488E76FF00504A6
:1023180085E76FF0040482E70070FF1F00FCFF03ED
:10232800D0010020B1F1006F70B511D30B4BD3F879
:10233800E0650B4B03EA862303F10063013B9942F6
:1023480006D840B139B192B20EF0F8FA002070BD4B
:102358004FF0FF30FBE76FF00500F8E70070FF1F54
:1023680000FCFF03B0F1006F10B40DD3084BD3F895
:10237800E045084B03EA842303F10063013B9842DC
:1023880002D810BCFFF7A2BE4FF0FF3010BC704758
:102398000070FF1F00FCFF034FF0B04382B0DA6CFF
:1023A8000243DA64DB6C03400193019B02B070477F
:1023B80030B5012087B00024CDE90444FFF7ECFFD5
:1023C8000220FFF7E9FF0420FFF7E6FF01250222BC
:1023D8000DEB00014FF404134FF09040CDE90123B9
:1023E800039503F09FF84FF4441301A94FF0904070
:1023F800CDE90235019503F095F804230DEB0301AF
:102408000C48CDE90135CDE9034403F08BF82246A9
:102418002146062002F02CFD062002F05BFD224634
:102428002146072002F024FD072002F053FD07B0E3
:1024380030BD00BF0004004808B51248124A134BCB
:10244800C0E9002300230122C0E90232C0E90433B5
:10245800C0E90633036203F09DF908B100F0ECF817
:102468000848002103F0E7F908B100F0E5F805484D
:10247800002103F006FA18B1BDE8084000F0DCB806
:1024880008BD00BF94020020005800405D3E302087
:1024980070B596B005461422002103A80EF086FEFA
:1024A8003822002108A80EF081FE2A68304B9A4293
:1024B8005BD18023089308A84FF440230E9303F0C0
:1024C8003BFF08B100F0B8F84FF0B0444FF4C050EB
:1024D800E36C43F00103E364E36C03F0010302934C
:1024E800029B12230026CDE903030323CDE90563EC
:1024F8004FF09040042303A9079303F013F8A36D4A
:10250800DFF870C043F48003A365A36D1A4C03F48D
:1025180080030193019B26620D23C4E900C3204672
:102528008023C4E90266C4E90436C4E9066602F0F9
:1025380031FD08B100F080F8104AEC63A562104C38
:102548000E23C4E900231021002380222046C4E979
:102558000213C4E90423C4E90633236202F01AFD16
:1025680008B100F069F8AC63A56216B070BD00BF91
:102578000058004044000240D401002058000240A6
:102588003402002000B59BB04822002108A80EF0B4
:102598000DFE1822002102A80EF008FE03F096F99D
:1025A8004FF0B0420120D2F8903023F01803C2F85F
:1025B8009030D2F8003423F4C06343F40073C2F8B7
:1025C8000034D2F8003403F4C0630193019B242340
:1025D800089381230B930023CDE91003B02208A8A8
:1025E800CDE9122303F0EAFA08B172B6FEE74F23E9
:1025F800CDE90230CDE90400CDE90600022102A8A8
:1026080003F076FD08B172B6FEE71BB05DF804FB77
:1026180008B501F0A5FFFFF7B5FFFFF7C9FEFFF703
:10262800F2FCFFF709FF00F0D7FD40F6B83000F0E4
:1026380049FA00F0D8FDFCE772B6FEE700B58DB0A8
:102648002C22002101A80EF0B1FD1748174B03609A
:102658001F2383604FF080420023C0E90433C0E9A0
:10266800072383614FF48073436203F0EBFF08B1E3
:10267800FFF7E2FF0C4804F011F908B1FFF7DCFF9F
:102688004FF0005300220793074808924FF48073D5
:1026980001A9029206920B9304F034F808B1FFF7EF
:1026A800CBFF0DB05DF804FBE802002000280040D5
:1026B80010B5044690B03822002102A80EF076FD2D
:1026C8002268194B9A422CD14FF48033029302A806
:1026D8004FF480730F9303F02FFE08B1FFF7ACFFA0
:1026E8004FF0B0430220D3F8902042F40042C3F8E0
:1026F80090209A6D42F480629A659B6D002203F4E3
:10270800806311460193019B02F0B2FB022002F0A4
:10271800E1FB00222A20114602F0AAFB2A2002F03F
:10272800D9FB10B010BD00BF002800407047000062
:1027380008B501F02BFF044B0120C3F88800BDE861
:10274800084003F01BB900BF0004005801F025BF82
:1027580008B501F022FF00F063FCFFF729FEFFF740
:1027680052FCBDE80840FFF767BE08B501F00EFF50
:10277800BDE808400121002003F0B0B87047704759
:10278800FEE7FEE7FEE7FEE7FEE7704770477047A3
:1027980070470000014804F0A7B800BFE802002015
:1027A800012002F0EBBF022002F0E8BF704770473B
:1027B800014802F069BD00BFD4010020014802F0C1
:1027C80063BD00BFC0030020014802F05DBD00BF2B
:1027D80060030020FFF7F2BF7047202002F0CEBF51
:1027E80070470000014804F043BC00BF20040020EB
:1027F800014803F0ABBE00BFE8020020014804F026
:102808009EBA00BF4C0300202DE9F04389B08046F2
:102818000020109E0790894615461F46FDF700FDCB
:10282800F0B9104CCDE90090CDE9020407AB0E4891
:102838000593142304933A46434629460068FDF756
:10284800B9FD2346324604F1140153F8044B42F80B
:10285800044B8B42F9D1079B337509B0BDE8F0836F
:102868000120FAE720030020D41301087FB5124C99
:1028780000253C2302A86375CDE90255257500F0B3
:10288800C3F8042303AA009412210C48FFF7BCFFE5
:102898000B49142220460EF079FC0646B0FA80F067
:1028A800400960750090074B2A46294602200DF022
:1028B8003DFF304604B070BD340300201A140108EF
:1028C800D2060020FC130108054808B50823036058
:1028D80004F050F818B1BDE80840FFF7ADBE08BDD8
:1028E8004C0300204FF0B04307B55A6E42F0010286
:1028F8005A665B6E002203F00103019311463220F1
:10290800019B02F0B5FA322003B05DF804EB02F047
:10291800E1BA00000CB407B5054A05AB10210193D4
:102928000EF016FB03B05DF804EB02B0704700BF71
:102938002C14010830B585B0044602A80D460EF0E7
:1029480033F9BDF90C30064A00931021029B20464A
:10295800FFF7E0FF2046FEF72FFD288005B030BDC9
:102968002C1401084FF0B04210B5936823F40043CB
:1029780093600EF0A1F90E4B01241C7000F0B6F81C
:102988000DF06AFE0B480DF081FE0B4B4FF4004230
:102998001A6103200DF080FEFFF7B6FA00F012F975
:1029A8000DF076FF21462046BDE810400DF090BF9F
:1029B800580300203D290008004000580DF09EBF34
:1029C80008B5FFF7A9FA40F6B83398420CD8B0F525
:1029D800E16F0BD3FE23A0F5E16058434FF49663F3
:1029E800B0FBF3F0C0B208BDFE20FCE70020FAE718
:1029F8007FB5684600F0CAF80198FFF75FF800B2A3
:102A080007B05DF804FB0000194A38B5D2F88035E4
:102A1800591C044619D101F0C7FD054601F0D0FD47
:102A2800054401F0C7FD2B0EE3712B0CA3712B0A93
:102A38006371030EE370C0F30742C0F307232571E7
:102A4800C0B2A2706370207038BD190AC371817159
:102A5800190C1B0E41710371D2F88435C370D2F87A
:102A68008405C0F30722C0F30743000EE9E700BF5F
:102A78000070FF1F38B5094BD3F880350360013368
:102A8800054609D101F090FD044601F093FD44404C
:102A980001F096FD44402C6038BD00BF0070FF1F58
:102AA800012102200DF0FEBE002102200DF0FABE29
:102AB80000207047024B187808B100F0BBB8704787
:102AC8005803002082B00190019802B000F04EB97E
:102AD8004FF0B04382B0DA6C42F00202DA64DB6C89
:102AE80003F002030193019B02B070472DE9F04304
:102AF800254C87B001F06AFD01F070FD01F076FD0C
:102B08000123002502934FF48059032301A920468D
:102B180004934FF4005803950595FFF7D9FFFFF785
:102B2800D7FFFFF7D5FFFFF7D3FFCDF8049002F0EA
:102B3800F9FC01A920464FF40067CDF8048002F0A3
:102B4800F1FC01A920464FF40046019702F0EAFC87
:102B580001A92046019602F0E5FC2A46494620468E
:102B680002F006FE2A464146204602F001FE2A46A9
:102B78003946204602F0FCFD2A463146204602F03E
:102B8800F7FD07B0BDE8F0830004004810B504461F
:102B9800FFF7DCF9074BA36040F30F20FEF73AFF7D
:102BA800054B064A2360064B6060C4E903230020F6
:102BB80010BD00BF0000484200007A440D093E00E5
:102BC800AB03050000207047014B1868704700BF31
:102BD8005C0300200320704708B501464FF47A7261
:102BE80000238002890DFEF78FFF08BD4FF47A732A
:102BF800A0FB0303800A40EA83507047034B9868A0
:102C08009A689042FBD1C043704700BF002800403B
:102C180008B5FFF7F3FF014B186008BD5C030020FF
:102C280008B5FFF7EBFF024B1B68C01A08BD00BFD1
:102C38005C030020024B187808B1FFF7DFBF70472C
:102C48005903002010B5074B074C0122DA654FF4F1
:102C58008071204603F040FC4FF0FF3323630020CF
:102C680010BD00BF00280040E802002002460021F5
:102C7800014803F04ABE00BFE802002002460121D5
:102C8800014803F042BE00BFE802002010B58CB036
:102C98002C220021044601A80EF088FAFFF7D2FF83
:102CA8000C4B0D481B681C440023089306934FF0F7
:102CB8000053E443079301224FF4807301A902945F
:102CC8000B9303F01FFD08B1FFF7B6FC00200CB012
:102CD80010BD00BF5C030020E802002038B505469F
:102CE800FFF78CFF02210446074803F015FEC4F3E2
:102CF80009024FF47A71A2FB0121920AA30A2A80E1
:102D080043EA805038BD00BFE80200200148002196
:102D180003F002BEE80200200148012103F0FCBDD7
:102D2800E8020020F8B50F4D2E78CEB90E4C4FF0C2
:102D3800FF372763FFF782FCFFF784FF4FF48071AA
:102D4800204603F0C9FB2046276303F089FD32467D
:102D58002046022103F0D9FDFFF75AFF01232B700B
:102D68000020F8BD59030020E8020020014610B5F4
:102D78004FF47A7200238002890DFEF7C5FE0146E2
:102D8800FFF73CFF0446FFF739FF031B8B4200D3D4
:102D980010BD00BFF7E70EF097B8000010B5064C5D
:102DA8000221204603F0B8FD0221421C2046BDE85E
:102DB800104003F0AABD00BFE80200201648174AD9
:102DC80008B54FF4E133C0E9002300230C22C0E921
:102DD8000233C0E90523C0E90733C0E909330361B9
:102DE80004F027FF08B1FFF727FC0B48002105F086
:102DF8009CF808B1FFF720FC0748002105F0B5F85A
:102E080008B1FFF719FC044805F06FF818B1BDE8E0
:102E18000840FFF711BC08BD200400200044004012
:102E280070B596B005461422002103A80EF0BEF92D
:102E38003822002108A80EF0B9F92A68334B9A42C3
:102E480061D10223089308A8314B0A9303F074FA5E
:102E580008B1FFF7F1FB4FF0B0430C219A6D2D4CF0
:102E680042F400329A659A6D02F400320292029A94
:102E7800DA6C42F00102DA64DB6C03F001030193BF
:102E8800019B02230026CDE903130323CDE9056343
:102E98004FF09040072303A9079302F043FB1E4815
:102EA80026621423C4E900031023C4E9023620462D
:102EB8008023C4E90436C4E9066602F06BF808B159
:102EC800FFF7BAFB154AEC67A562154C1323C4E952
:102ED8000023204600238022C4E90233C4E90423E6
:102EE800C4E90633236202F055F808B1FFF7A4FBE2
:102EF8002520C5F8804000220221A56201F0B8FF14
:102F0800252001F0E7FF16B070BD00BF0044004067
:102F180004000C00C0030020800002406C00024046
:102F28006003002002680E4B9A4210B5044616D181
:102F38004FF0B0420C21936D23F4003393654FF0AA
:102F4800904002F09BFBE06F02F098F8D4F8800004
:102F580002F094F8BDE81040252001F0C9BF10BD6B
:102F68000044004008B50A460146024803F0E4FF61
:102F7800002008BD2004002013B5114B114C186027
:102F88004FF40013009302AB13E90600204604F047
:102F980050FF2368DA69D103FCD4DA695202FCD500
:102FA8009A68084842F480029A6004F088FF06494B
:102FB8000448012204F0F6FE002002B010BD00BF54
:102FC800B404002020040020BC04002008B5074BEE
:102FD8001860FFF718F8FFF7F1FE054AD2F88030BD
:102FE80043F00063C2F88030002008BDB804002018
:102FF8000008005808B54FF0B04308489A6B42F4EF
:1030080000329A639A6B22F400329A63FFF78AFFC0
:103018000F2001F06DFF002008BD00BF2004002034
:1030280008B5074804F005FE08B1FFF705FB054899
:1030380001F0B0FF18B1BDE80840FFF7FDBA08BDC0
:1030480020040020C00300200268044B9A4203D1E8
:10305800034B00201B681847704700BF004400401E
:10306800B804002002680B4B9A4210B504460FD1F1
:10307800094B1B682BB1D0F8902012B907480121E1
:10308800984720460549BDE81040012204F08ABE51
:1030980010BD00BF00440040B4040020BC04002060
:1030A80013B5134C23785BB9E37C03F0FF023BB9FB
:1030B800104B1146022002B0BDE810400DF036BB9F
:1030C800FFF7D4FB00380C4B18BF012040001870E4
:1030D8001A78022A02BF00222270E2741B78009339
:1030E8000022064B114603200DF020FB02B010BD54
:1030F800D206002088140108C5040020A414010881
:1031080038B5174C237853BBE37C03F0FF0233BB7D
:10311800144D2B68012B0CD92B68042B09D81146A8
:10312800114B02200DF002FB104A0421012000F08F
:103138004DFB2B68042B12D900220D4B114602209F
:103148000DF0F4FAFFF792FB00380A4B18BF012084
:10315800400018701B78022B04BF0023237038BD71
:10316800D2060020C0040020BB140108E0140108A6
:10317800E5140108C504002070477047022808B507
:103188000ED801221021074802F0F2FA3220FFF788
:1031980099FCBDE8084003480022102102F0E8BA73
:1031A80008BD00BF000400487047000010B50121A9
:1031B80004464FF0904002F0D5FA054AB0FA80F381
:1031C8005B0913701378A370024B01221A7010BDAB
:1031D800C4040020D106002008B5FFF7C3FBBDE8F2
:1031E800084000F0B7BC4FF0FF300DF0EBBB704764
:1031F800014BD870704700BF5C000020014B187469
:10320800704700BF5C00002007B5064B00221B5C1E
:1032180000931146044B02200DF088FA03B05DF8C4
:1032280004FB00BF321501081815010808B5022073
:1032380000210DF08FFBBDE8084001480DF0F2BDFC
:1032480020060020002101200DF084BB37B504467C
:10325800002832D090F90650002D30D11B480DF0CF
:1032680093FD1B4B2A46294602200DF05FFAE379AD
:10327800012B0CBF174B184B2A46294602200DF08C
:1032880055FA164BE2791A701978154A154B012927
:1032980018BF1346002200931146134B01200DF06E
:1032A80045FA94F90530019394F90430009300220B
:1032B8000E4B114602200DF039FA03B030BD002242
:1032C8000B4B114602200DF031FAEAE7BC0500204D
:1032D8003F1501085415010871150108EC05002077
:1032E8003A150108361501088E150108C61501089A
:1032F800AD15010813B50D4CA0B120600C480DF0B8
:1033080043FD21680A480DF0C7FD09480DF08AFD04
:10331800236800930022074B114603200DF006FA9C
:1033280002B010BD42F210732360E7E7740000207A
:1033380020060020EF15010813B50D4C2060236806
:103348000BB90C4B23600C480DF01EFD21680A4890
:103358000DF0A2FD08480DF065FD236800930022DA
:10336800064B114603200DF0E1F902B010BD00BF75
:103378000C000020A086010038060020181601085D
:1033880038B504460D4607484FF40061FEF7EAFFDA
:1033980030B92A4621460348BDE83840FEF7E4BE66
:1033A80038BD00BF00F003080A460149FEF7BABF5E
:1033B80000F0030870B516480DF0E6FC05F03AFA7F
:1033C800044650B10022134B114602200DF0AEF90D
:1033D800BDE8704010480DF025BD104D104B024659
:1033E800014602200DF0A2F901260E4B2E7022464E
:1033F800214602200DF09AF90B4805F0ADF828781F
:10340800314604F0FFFD02480DF00CFDE0E700BF77
:103418002006002054160108F005002000000020B6
:1034280072160108861601085C00002030B587B0C6
:10343800FFF7C6FA044604F0DBFE054680B1002417
:103448003E480DF0A1FC3E4B3C481968A14238BFEC
:1034580021460DF021FD39480DF0E4FC07B030BDE0
:1034680003A8FFF7A3FE374A3749042313705368AC
:103478000878187053685D705368182199705368FC
:103488000121D970516823B203EB430303EB4313C3
:10349800FE24B3FBF4F30B712C4B197849B31D7060
:1034A800536860F07F001870052313702849294C71
:1034B8000978012988BF00235370637A33B104F077
:1034C80083FE012802D120460DF05EFC224B1D48E8
:1034D800D978002204F0A2FE0446D8B91F4B187010
:1034E8001F4B0146187001221E4B03200DF01EF9D8
:1034F800A6E71B4B1B7813B9184B1B7843B15368CD
:103508000121597153689DF80E1099710723CDE771
:103518000523CBE7063492D104F050FE0446002878
:103528008ED001224FF47A730021B0FBF3F31046DA
:1035380000930D4B0DF0FAF882E700BF200600203B
:103548007400002004000020B80500205006002068
:10355800C5040020BC0500205C000020D106002026
:10356800E7060020A5160108B416010800B50346B1
:103578008DB000282CD0407802280AD003282AD001
:10358800164B0022114602200DB05DF804EB0DF039
:10359800CDB81A7F0B92DA7E0A929A7E09925A7EE9
:1035A80008921A7E0792DA7D06929A7D05925A68E9
:1035B8000492DA68039293F914200292B3F9122064
:1035C80001921B7C00930022054B11460DF0AEF8CA
:1035D8000DB05DF804FB034BD3E700BFD21601081A
:1035E800E91601085B17010801284FF000020CBF1B
:1035F800024B034B114602200DF098B87A170108C8
:103608008C1701081FB50446002831D00378002B19
:103618002ED01D480DF006FC002211461B4B02203F
:103628000DF084F894F91830039394F90A30029352
:10363800237C0193E368009300221146144B032076
:103648000DF074F80022134B114603200DF06EF8AC
:10365800237A012B0ED1617A0F4A104B002908BF3B
:1036680013460022009311460D4B03200DF05EF81F
:1036780004B010BD00220B4B1146032004B0BDE876
:1036880010400DF053B800BF08060020A517010828
:10369800D617010807180108A0170108A117010883
:1036A800141801082518010808B5104B012200213B
:1036B80002201A700DF04EF90D480DF0B3FB0D4BBA
:1036C8001B788BB10C4B1A7872B9DB7C63B90B4B46
:1036D8001A68042A9EBF1A6801321A600021BDE8E0
:1036E800084010200DF036B908BD00BF5006002074
:1036F80038060020EC050020D2060020C004002077
:10370800044B1B78022B03D1002108200DF022B9AD
:10371800704700BF0000002008B505F094F880B994
:1037280004F052FD01280CD1BFF34F8F0549064B19
:10373800CA6802F4E0621343CB60BFF34F8F00BF47
:10374800FDE708BD00ED00E00400FA0510B505F03E
:103758000DF910F1080F07D1064B0022BDE8104003
:10376800114602200CF0E2BF013001D1024BF4E710
:1037780010BD00BF33180108491801087047704789
:1037880070470000012813B5044603D0022817D05B
:1037980002B010BD01464FF0904001F0E3FFB0FACF
:1037A80080F04009002200901146074B20460CF09B
:1037B800BDFF0021022002B0BDE810400DF0CAB8DC
:1037C80000210820F7E700BF6118010873B5054616
:1037D8000C46164604F00CFD0346002838D0002499
:1037E80026480DF0D1FA264B24481968A14238BF63
:1037F80021460DF051FB214802B0BDE870400DF0A4
:1038080011BB4A68F05CD0540133DAB2A242F8D353
:103818001C4B0D701B78012B88BF00244C701A4C70
:10382800637A33B104F0D0FC012802D120460DF0B0
:10383800ABFA164B1648D978002204F0EFFC044680
:1038480040B90146134B012203200CF06FFFC7E774
:103858000F49DAE70634C2D104F0B0FC0446002868
:10386800BED04FF47A730122B0FBF3F3002100932A
:103878000320094B0CF05AFFB2E700BF20060020D6
:1038880074000020C5040020BC0500205C00002056
:1038980004000020A5160108B4160108044B1B7883
:1038A80023B9044A05210120FFF790BF704700BFE4
:1038B800C50400207F18010810B5002490B03C22F0
:1038C800214601A800940DF071FC2C4B2022DA72DD
:1038D80019788DF8001059788DF8011099788DF8BD
:1038E8000210D9788DF8031019798DF804105979D8
:1038F8008DF8051099798DF80610D9798DF807108B
:10390800197A8DF80810597A8DF80910997A8DF876
:103918000A108DF80B2021460DF10B0258180131C1
:10392800007B02F8010F1C29F8D193F828208DF8A4
:10393800282093F829208DF8292093F82A208DF83B
:103948002A2093F82B208DF82B200DF12B01002233
:103958009818013290F82C0001F8010F142AF7D1B9
:1039680007484FF40061FEF7FDFC20B904484022E7
:103978006946FEF7F9FB10B010BD00BF78000020C3
:1039880000F80308014940220CF0D8BF00F80308EA
:1039980070B52A4D28796B794D2BC0B233D1C0EB65
:1039A800001080000A2838BF0A204FF47A73584361
:1039B800234BAC791860EB794D2BE4B22BD1C4EBD7
:1039C8000414A40095F82C301E4E63BB95F83F30C4
:1039D8004BBB42F21070FFF78DFC3068FFF7ACFC70
:1039E8002B7A194A1949DBB213706B7A184ADBB281
:1039F80013700023EA1892F82C20D2B2CA5401336B
:103A0800142BF7D170BD6B79482B0ABF4FF4616353
:103A18006B795843C6E7EB79482B0ABF4FF46163CB
:103A2800EB795C43CEE7FFF765FC012C38BF012436
:103A38004FF47A735C433460CFE700BF780000200E
:103A4800740000200C000020E6060020D2060020AA
:103A5800C504002010B590B000213C2201A80091B7
:103A68000DF0A4FB4022374968460CF067FF9DF82B
:103A780000203AB99DF80100182803D19DF80210DA
:103A8800012914D0002211462F4B03200CF04EFEC2
:103A9800FFF712FF2D48142200210CF059FF4FF4B4
:103AA8007A70FFF70FF8FFF773FF10B010BD284BBF
:103AB8001A70587099709DF80310D9709DF8041009
:103AC80019719DF8051059719DF8061099719DF8A6
:103AD8000710D9719DF8081019729DF809105972CC
:103AE8009DF80A1099729DF80B1001F03F01D972E8
:103AF800D87AD1B288421BD89DF8282083F828208C
:103B08009DF8292083F829209DF82A2083F82A2067
:103B18009DF82B2083F82B200DF12B0100229818FB
:103B2800013211F8014F80F82C40142AF7D1BAE776
:103B380001F140006844194410F8340C087301324C
:103B4800D6E700BF00F8030885180108D206002050
:103B580078000020F0B50B238BB012220024012539
:103B6800CDE90632032718231721CDE9043122466F
:103B78005C4B03942146CDE90155009728460994EA
:103B88000CF0D4FD584B009522462146CDE901742E
:103B980002200CF0CBFD02260523CDE90063224666
:103BA800524B0294214630460CF0C0FD504B009514
:103BB80022462146CDE9017430460CF0B7FD09A92B
:103BC800204604F023FE099BC3F307220292C3F3A5
:103BD80007421B0E019200932246464B214630466F
:103BE8000CF0A4FD09A9284604F010FE099BDAB2DE
:103BF8000392C3F307220292C3F307421B0E0192FA
:103C0800009322463C4B214630460CF08FFD3B4B3F
:103C18003B48009422464FF4FA710DF057F8394B9F
:103C28003948009422464FF4FA710DF04FF8374B9B
:103C3800374800942A464FF4FA710DF047F82046A9
:103C4800FEF78CFA08B1FEF7F7FC324B009400221D
:103C58004FF4FA6130480DF039F8304A002101205C
:103C68000CF034FF2E4A002102200CF02FFF2D4AC1
:103C7800002104200CF02AFF2B4A002108200CF018
:103C880025FF00F0B3FB2949294804F075FD2948B0
:103C980004F062FC1E480DF0C5F8274B0021187887
:103CA80004F0B0F925490094254B096825480022FD
:103CB8000DF00CF823480DF0B5F8FFF7CBFE224ABB
:103CC800002110200CF002FF204B21481968214BDD
:103CD800009400220CF0FAFF1D480DF0A3F80BB079
:103CE800F0BD00BFC71801080E1901082F190108F7
:103CF800501901087119010892190108F7310008D3
:103D08000806002087370008D405002085370008FA
:103D1800BC05002009370008F00500205983000879
:103D28003534000855370008BD330008000003018A
:103D3800100000205C00002000000020740000201B
:103D48003532000820060020093100080C00002048
:103D580038060020B136000810B50024A2B07C2235
:103D6800214603A802940DF021FA53238DF8083058
:103D78004FF48C73ADF80A3001238DF80C30ADF890
:103D88000440FEF71DFEFE23B0FBF3F000EB4000FD
:103D980000EB40108DF80D0001A800F0CDFBA0B994
:103DA80058238DF80E3007243022802108480DF062
:103DB800FDF9224602A906480DF029FA044A2146CF
:103DC8000120FFF703FD22B010BD0624ECE700BF79
:103DD80051060020F0B50378592B95B0044640F001
:103DE800F18105295FD84378443B162B5BD8DFE87F
:103DF80013F01F015A000F015A0017015A005A0008
:103E08005A005A0079005A00FA005A005A005A001B
:103E180095015A005A009D005A005A005A0017008E
:103E28008578482D17D1B24A14210120FFF7CEFC1E
:103E380041F28830FEF746FE0022AE4B11460320C1
:103E48000CF074FC40F6B830FEF73CFE15B0BDE847
:103E5800F040FFF761BC532D0ED130228021A648D7
:103E68000DF0A4F9FFF778FF41F28830FEF72AFE3B
:103E7800A14A152101206EE0432D16D1002404A883
:103E88008DF8104004F0E0FA9B4A4C231370182375
:103E980093709DF81030547001204133D070137125
:103EA8000521FFF793FC15B0F0BD442DFBD1924CD2
:103EB8002C228021201D0DF079F9002325706370D4
:103EC80001251823A370E5702571FEF779FDFE23FF
:103ED800B0FBF3F000EB400000EB401060712246AD
:103EE8000621C7E78378303BDBB2092BDBD8834C4C
:103EF800834A23702378DBB253727F4A59231370A5
:103F08004D23537023783033937003210120FFF73A
:103F18005DFC2378009300227A4B114601200CF0B7
:103F280005FC15B0BDE8F040FFF7C6BC8578482D04
:103F380016D1714A562313700023537018239370B7
:103F480003231371172353710B2301209371122339
:103F5800D070D371082115B0BDE8F040FFF736BC2A
:103F6800432DA0D1644C00213C2205A804910DF0FA
:103F78001DF904A8FFF706FD2422802104F10C0096
:103F88000DF014F99DF8103063709DF81130A3708E
:103F98009DF81230E3709DF8133023719DF81430AA
:103FA80063719DF81530A3719DF81630E3719DF883
:103FB800173023729DF81830257063729DF81B50D6
:103FC8009DF81930A3729DF81A30E3722A4607A9A2
:103FD800257304F10D000DF01AF905F10D012246C3
:103FE800C9B201205DE7807839280CD83038C0B2D2
:103FF800FFF7C2F8404A2378137063785370A378A8
:104008009370032136E715B0BDE8F040FFF746BCD2
:1040180080783928F7D83038C0B2FFF7AEF8E9E72A
:1040280080783928EFD83038C0B2FFF7A7F8E1E731
:104038008378303BDAB2092AE5D8C578303DEAB250
:10404800092AE0D80179A1F14802D2B20B2ADAD8BC
:104058002D4840FA02F2D007D5D40A224D2902FB96
:1040680003553FD13C235D43284B4FF47A70684396
:104078001860274B1860FFF73DF91F4A2378137023
:1040880063785370A3789370E378D37023791371AE
:1040980005210120FFF79AFB194B182200261E70F4
:1040A8005A7001229A70DA70A178303901EB8100D8
:1040B800E178303901EB4001C9B2197122795A719E
:1040C800144A1278D2B21A720C4A1278D2B25A72C0
:1040D800FFF7F2FB104B00953246314603200CF0F7
:1040E80025FBE0E64829BFD14FF46163BBE700BF79
:1040F800B6190108CB19010851060020C504002093
:1041080078000020ED190108DEF7FFFF7400002099
:104118000C000020E6060020161A01088678A6F191
:104128003007FBB2092B3FF66EAFC078A0F130051F
:10413800EBB2092B3FF667AF2379A3F14802D2B25D
:104148000B2A3FF660AF6D4941FA02F2D2073FF5FC
:104158005AAF0A224D2B02FB07552ED13C2255435C
:10416800674A59211170532151709670D07013719C
:1041780005210120FFF72AFB624B182200261E703A
:104188005A7001229A70DA70A178303901EB8100F7
:10419800E178303901EB4001C9B299712279DA71BD
:1041A800594A1278D2B21A72584A1278D2B25A724E
:1041B800FFF782FB564B00958EE7482BD0D14FF482
:1041C8006162CCE7502B5DD102297FF66CAE437853
:1041D800303B012B3FF667AE8378312B7FF463AE1B
:1041E8000B2904D8FFF75AFB0021454A42E6454D02
:1041F800484F0234002614F8012FA919303AD2B2D8
:104208000A730B7BCDE9026323780022CDE90063B2
:1042180011463B46032001360CF088FA0C2EEAD1F1
:10422800FEF7C2FF364B50221A7018229A700024EB
:1042380001225C70DA7003F8042F2A190134127B0A
:104248000C2C02F1300203F8012FF6D10022502382
:10425800114600930320304B0CF068FA00232B70B2
:1042680018236B700123AB70EB70274B1B78DBB204
:104278002B72264B1B78DBB26B72EC72FFF71CFBC0
:104288001121B2E7412B7FF40EAE4378432B7FF424
:104298000AAE16297FF407AE204D421C002312F8FF
:1042A800011FE9540133142BF9D1FEF7F9FE1C4B19
:1042B8005B7D012B19D113490023EA5CC81801332F
:1042C800D2B2142B80F82C20F7D1104B00221A7090
:1042D8001B78DBB24B72FFF7EFFA094A631E1534FD
:1042E8009C4206D1064A1621C4E5084B02221A70E0
:1042F800F3E713F8011F02F8011BF1E7DEF7FFFFF0
:104308005106002078000020E6060020C5040020A1
:104318004D1A0108981A0108C01A0108D20600208F
:104328003403002070B5054686B00C4600293BD002
:1043380028480CF077FD2678EEB1002D48D0686843
:104348002E78C0B1032E0BD0042E2FD0022E12D1FE
:10435800697801290FD00B060DD4FFF73BFD0AE061
:104368006B78012B07D10078012802D0022800D0F1
:1043780008B904F01FF8237C052B15D894F90A20F6
:10438800059294F909200492134A52F823300393B2
:1043980094F90830CDE901630022E36800931146DF
:1043A8000E4B03200CF0C2F906B070BD6B78012BE0
:1043B800E1D102780A4B02F001021A702AB9094BBE
:1043C800114603200CF0B2F9D5E7074B0022F7E7B6
:1043D8002E46D0E7D4050020441B0108EE1A010838
:1043E800B8050020DB1A0108E51A0108034B002272
:1043F800C3E902220122C3E900227047E80600202F
:1044080000487047E80600204FF0B04382B0DA6CED
:104418000243DA64DB6C03400193019B02B07047EE
:104428002DE9F04186B000240220154D0594FFF7D0
:10443800EBFF0420FFF7E8FF124F03944FF4807658
:1044480001230DEB0001CDE9016328460323049302
:104458004FF4005801F066F801A93846CDF80480F9
:1044680001F060F822464146384601F081F92846B5
:104478002246314601F07CF9204606B0BDE8F081BD
:104488000004004800080048032810B50ED8012889
:1044980010D868B902460B484FF4807101F068F9EA
:1044A800002209484FF4005101F062F9002010BDC4
:1044B8000122F0E7002203484FF4807101F058F917
:1044C8000122EEE700040048000800480220704777
:1044D800002070470120704700280CBF0F201620CD
:1044E800704700000D48854600F038F80C480D4923
:1044F8000D4A002302E0D458C4500433C4188C4237
:10450800F9D30A4A0A4C002301E013600432A2429C
:10451800FBD30CF053FEFEF77BF8FEE7000001200A
:10452800000000204C010020542601084C01002006
:1045380084240020FEE7000007B5AA2343700193F6
:10454800037800930022044B114601200CF0EEF88A
:10455800002003B05DF804FB5C1B010870470000F5
:1045680010B5032000F072FC01F018FB064B186030
:104578000F20FEF79DFA044618B9FEF700F9204609
:1045880010BD0124FBE700BFB80000204FF0E02277
:10459800136923F00203136170474FF0E022136997
:1045A80043F0020313617047014BD3F8900570473D
:1045B8000070FF1F014BD3F8940570470070FF1F70
:1045C800014BD3F8980570470070FF1F024A5368E3
:1045D80023F0010353607047002004E0024A536847
:1045E80023F0020353607047002004E0024A536836
:1045F80023F0040353607047002004E08068C0F390
:1046080080007047F7B5002301930446002800F0A6
:10461800E980856D25B9FDF721FCE56584F85450DE
:1046280023689A68D00040F1A1809A68D10000F10F
:10463800B480A26D42F01002A265E26D42F0010260
:10464800E26501251846FFF7D9FFA26D02F01002B6
:10465800024340F0C980A26D206922F4817242F0C1
:104668000202A2659A68D2075DD4226BA67E94F8EE
:104678002CC0003A18BF01221703D4E902120A43DA
:10468800217E42EA8132617E42EAC13242EA463202
:10469800002842EA4C02B4BF20F000414FF4001158
:1046A8003A430A4394F82010012903D1002E76D109
:1046B80042F48032616A21B1A66A01F4E0713143A3
:1046C8000A43D968E66C21F4FE3121F4FF711143E5
:1046D800D96094F83C206168012A01F0404C4CEA0A
:1046E800060609D1D4E910273A433243A66C32436F
:1046F80042EA0C0242F001061F693E4A3A40324340
:104708001A6121F00042B2F1804F0CD0B1F1004F94
:1047180009D0394ED6F8082701F4701122F4701226
:104728000A43C6F808275A69666BA16B22F007028C
:1047380032435A615A6922F0700242EA01125A6100
:10474800002835D19A6A62F00F029A625B6903F019
:1047580007039E423CD10023E365A36D23F00303C6
:1047680043F00103A365284603B0F0BD9A682349C6
:1047780022F0104222F0170242F080529A60204A3A
:104788001268B2FBF1F2013252000192019A002A3A
:104798003FF44BAF019A013AF7E7002552E7A16DC4
:1047A80041F02001A165E16D41F00101E16581E77A
:1047B800B0F5001FCAD19A6AE269013A92006FF017
:1047C8000F0102F01C0201FA02F2216E0A43BCE753
:1047D800A36D23F0120343F01003A365E36D43F0C8
:1047E8000103E3650125BEE7A36D43F01003A3654C
:1047F800F8E700BF02FCFF1F00200140400D030046
:10480800B8000020F8B54569082D04460E460AD0C0
:104818000368DB68D80705D5A36D43F02003A365BB
:104828000120F8BD0425FEF745F9074623681A68F4
:104838002A4221D0A26D42F40072A265DA6812F40D
:10484800406F14D1A27E92B91A6812070FD5184684
:10485800FFF7D4FE28BB5A6822F00C025A60A26DFA
:1048680022F4807222F0010242F00102A265207E49
:1048780000BB0C221A60D4E7711CD8D0FEF71AF9D5
:10488800C01BB04201D8002ED0D123681B682B4032
:10489800CCD1A26D84F8543042F00402A265032002
:1048A800BFE7A26D42F02002A265E26D42F001026C
:1048B800E265DCE70020B4E70368186C7047000085
:1048C800F7B50023019390F85430012B044600F00B
:1048D800C58005680669012380F854302846FFF72B
:1048E8008DFE002840F0B480D1E90020022826F08F
:1048F800040300F08280B3F1004FC2F3110E13D10C
:10490800AB6A43EA0E03AB628B68686903EA022369
:1049180023F07C4323F0FF0320EA02210B43002A03
:104928006B6126DB002055E0236E00F01F074FF077
:104938000F0C0CFA07FC6FEA0C0623EA0C0CBEF10C
:10494800000F11D1C2F38463BB4043EA0C03236612
:104958008008E36901309842D6D8A86AC2F3836315
:10496800BB4006403343CEE792FAA2F3B3FA83F38F
:10497800EAE73B493B48D1F80837824203F0E07543
:1049880019D11B02CED4D1F8083723F0E0732B439A
:1049980043F40003C1F80837334B1A68334BB2FBB2
:1049A800F3F20C2302FB03330193019B002BB9D0D4
:1049B800019B013BF8E72E48824210D113F080702A
:1049C800B0D1D1F8083723F0E0732B4343F080735C
:1049D800C1F80837002384F8543003B0F0BD2548E7
:1049E80082429FD113F480009CD1D1F8083723F07C
:1049F800E0732B4343F48003EAE7B3F1004F01BFB0
:104A0800AB6AC2F311018B43AB62002A8ADA1548FC
:104A180013498242D1F8083709D1D1F8082703F0A1
:104A2800A07322F0E0721343C1F808377AE7104800
:104A3800824204D1D1F8082703F44003F1E70D4876
:104A480082427FF46FAFD1F8082703F0C073E8E71C
:104A5800A26D42F02002A2651846BBE70220BCE71F
:104A680000200140001000B0B8000020400D0300F5
:104A7800004000B8002000B4026838B5044610466B
:104A8800FFF7BCFD08B9002038BD9368990707D423
:104A9800936823F0004323F0170343F01003936057
:104AA800FEF708F8054623689B685B07EBD5FEF719
:104AB80001F8401B0228F6D923689B685A07F2D5EB
:104AC800A36D43F01003A365E36D43F00103E365B1
:104AD8000120D9E773B50023026801939368DD07C5
:104AE800044602D5002002B070BD9168214B1942DE
:104AF80009D0A36D43F01003A365E36D43F00103F0
:104B0800E3650120EFE7936823F0004323F01703E0
:104B180043F001039360184BD3F8083718021CD4EC
:104B2800637E012BDED0FDF7C5FF144E05462268D3
:104B38001368DB07D6D49368D9075FBF93683340FF
:104B480043F001039360FDF7B5FF401B0228EED93F
:104B580023681B68DA07EAD4CBE7094B094A1B68C4
:104B6800B3FBF2F301330193019B002BD8D0019BD7
:104B7800013BF8E71700008000200140E8FFFF7FB5
:104B8800B8000020400D030038B504460068FFF760
:104B980035FD054620BB94F85430012B20D0012365
:104BA80084F854302046FFF795FFB0B9A36D22680A
:104BB80023F4706323F0010343F48073A3651C237B
:104BC800E065136084F85400936823F0004323F0F1
:104BD800170343F00403936038BD84F85450FBE78F
:104BE8000220F9E7026838B5936891680446C80757
:104BF80001D4002038BD9907FBD4936803F005035E
:104C0800012B19D1936823F0004323F0170343F0D5
:104C18000203936003231360FDF74CFF05462368E6
:104C28009B68DB07E5D5FDF745FF401B0228F6D951
:104C380023689B68DA07F2D5A36D43F01003A365D8
:104C4800E36D43F00103E3650120D3E770B5044643
:104C580000284BD0836D43F002038365FFF70CFFF8
:104C6800054668B92046FFF7BDFF054608B9012388
:104C7800A3652268936823F0104323F01703936019
:104C880023685A6822F4677222F003025A6040F2DD
:104C98009F321A60D968164A0A40DA601A6922F007
:104CA80040421A615A6922F007025A611A6A02F0F0
:104CB800F0221A625A6A02F0F0225A62DA6A02F0A4
:104CC800F022DA629A6A0B4A00269E62D2F8083706
:104CD80023F0FE73C2F808372046FDF7D3F8E665DF
:104CE8002666A66584F85460284670BD0125FBE752
:104CF80000023E830020014010B590F85430012B8B
:104D0800044615D0012380F85430FFF7B5FE58B992
:104D18002046FFF767FF38B9A36D23F4807323F0AB
:104D2800010343F00103A365002384F8543010BD48
:104D38000220FCE7F7B50023019390F85430012BCB
:104D480004467FD0012380F85430FFF74BFF2368D7
:104D58009A6812F00102054607D0A36D43F01003CC
:104D6800A365002384F854302DE0A16D364F21F45B
:104D7800817141F00201A165DE68D96826F4FF4619
:104D880026F07C0621F40041360421F00301360C9C
:104D9800D96008209968394041F0004199609968C4
:104DA800002913DA0199013101910199B1F52E3FDA
:104DB800F5D3A36D23F0120343F01003A36500237A
:104DC80084F854300125284603B0F0BDD3F8B41058
:104DD800013801F07F010A44DCD199681A48014082
:104DE80041F001019960D3F8B41021F07F0141EA44
:104DF800D202C3F8B4209A68024042F002029A60D4
:104E0800FDF758FE074623689A68D20708D4DA687F
:104E18003243DA60A36D23F0030343F001039FE7F5
:104E2800FDF748FEC01B0228EDD923689B68D90707
:104E3800E9D5A36D43F01003A365E36D43F00103C7
:104E4800E365BFE70225BEE7E8FFFF7F0749CA68B9
:104E580022F4E0620302120403F4E063120C134329
:104E680043F0BF6343F40033CB60704700ED00E0CC
:104E7800164B30B5DC68C4F30224C4F10703251DC2
:104E8800042B28BF0423062D4FF0FF358CBF033CAD
:104E9800002405FA03F321EA0303A54022EA0502E8
:104EA800A340002843EA0203ACBF00F16040084A6F
:104EB8004FEA0313B8BF00F00F00DBB2AABF00F53A
:104EC8006140135480F8003330BD00BF00ED00E0AE
:104ED80014ED00E0002807DB044A4109012300F033
:104EE8001F00834042F82130704700BF00E100E016
:104EF80000280CDB4309064900F01F00203301227B
:104F0800824041F82320BFF34F8FBFF36F8F704764
:104F180000E100E070B5D0E913456560446D14B157
:104F2800D0E916456560D0E9105404F01C06012448
:104F3800B4406C60046863608368102B0BBFA26088
:104F4800A160E160E26070BD0268416CD3B210B547
:104F5800083B1424B3FBF4F30B4CA24288BF0B4A62
:104F680021F0030199BF01F1804202F50232521883
:104F780007338264064AC26403F01F03012202FA5F
:104F880003F3036510BD00BF070402401C0802407C
:104F98008008024038B500285ED002682F4B9A423C
:104FA8004FF014014CD82E4B1344B3FBF1F32D49A9
:104FB8009B00C0E91013022380F8253013680569A7
:104FC80023F4FF4323F070031360D0E90243234323
:104FD8002B43456911682B4385692B43C5692B43CE
:104FE800056A2B430B431360FFF7AEFFB4F5804F00
:104FF80004BF002343604268816C02F07F030B60AA
:10500800D0E91314013A032A4C6020D8164A1749EC
:1050180081651A44013B9200012103F0030301FA60
:1050280003F300214265C3651160114A53640023EC
:105038000122C36380F8243080F82520184638BD43
:105048000C4B1344B3FBF1F30B499B00B1E700236E
:10505800C0E91533C365EAE70120F0E70704024019
:10506800F8FFFDBF000002403F82001040090240E7
:1050780000090240F8FBFDBF0004024038B50028D3
:1050880041D00268136823F0010313601F4B9A4252
:105098004FF0140130D81E4B1344B3FBF1F31D49F4
:1050A8009B00C0E91013012403F01C0304FA03F366
:1050B800002515604B60FFF747FF836C41681D6052
:1050C800D0E913325A604A1E032A06D8124B0B4401
:1050D8009B0094401D60114B5C640023C363C0E9CE
:1050E8001533C0E90B33C0E90D33C36580F82530AB
:1050F80080F82430184638BD094B1344B3FBF1F34C
:1051080008499B00CDE70120F5E700BF07040240EE
:10511800F8FFFDBF000002403F8200100009024076
:10512800F8FBFDBF0004024070B590F82450012D33
:1051380004463BD090F825600125AE4280F8245003
:105148004FF000062CD1022580F825500568C6636B
:105158002E6826F001062E60FFF7DCFE036BBBB15C
:105168002B6843F00E032B60A36C1A68D20342BF6E
:105178001A6842F480721A60636D1BB11A6842F4AF
:1051880080721A602B6843F001032B60002070BD09
:105198002B6823F004032B602B6843F00A03E2E733
:1051A8008023C36380F824602846F0E70220EEE7F6
:1051B800034640B190F82520022A06D00422C26393
:1051C800002280F82420012070470268806C116852
:1051D80021F00E011160016821F4807101601168ED
:1051E80021F001011160D3E9100202F01C01012233
:1051F8008A404260D3E9132151605A6D32B1116877
:1052080021F480711160D3E9162151600122002038
:1052180083F8252083F82400704710B590F82530CE
:10522800022B03D00423C363012010BD03681A684E
:1052380022F00E021A601A6822F001021A60826CCB
:10524800136823F480731360D0E9101303F01C0271
:10525800012393404B60D0E913325A60436D33B158
:105268001A6822F480721A60D0E916325A60012353
:1052780080F82530836B002480F8244013B19847C8
:105288002046D2E71846D0E770B4426C046C036835
:1052980026681D6802F01C020421914031420FD09B
:1052A80015F0040F0CD01A6892065EBF1A6822F037
:1052B80004021A60036B6160002B33D070BC18477E
:1052C80002219140314217D015F0020F14D01A680C
:1052D800940606D41A6822F00A021A60012280F89D
:1052E8002520114A93428CBF104B114B5960002363
:1052F80080F82430C36ADFE708219140314211D099
:1053080029070FD5196821F00E011960012303FA46
:1053180002F26260C36380F82530002380F82430ED
:10532800436BC9E770BC704780000240000402402C
:10533800000002400A4A536943F4802330B55361A0
:10534800EFF3108472B60023CD58C5500433B3F57B
:10535800807FF9D11369DB03FCD484F3108830BD56
:1053680000400058064B5A69002ABFBF054A9A6098
:1053780002F188329A60BABF5869C00F002070479E
:105388000040005823016745044B5A6942F0004227
:105398005A615869C043C00F704700BF00400058A9
:1053A80070B50546FDF786FB124E04463369D903EE
:1053B80013D43369DA0744BF012232614CF2FA325E
:1053C800134011D10B4E306910F480200BD0FDF73B
:1053D80071FB001BA842F6D304E0FDF76BFB001B32
:1053E800A842E3D3032070BD024A1361024A012098
:1053F8005360F8E700400058F80600202DE9F04116
:10540800184D98462B78012B06460C46174626D091
:1054180001232B704FF47A7000236B60FFF7C0FFF5
:10542800A0B9012E16D1104A536943F00103536104
:105438002760BFF36F8FC4F804804FF47A70FFF7CA
:10544800AFFF094A536923EA0603536100232B700F
:10545800BDE8F08139462046FFF76CFFEDE70220F2
:10546800F6E700BFF806002000400058054A5369D7
:1054780023F47E7343EAC00040F4803040F0020019
:1054880050617047004000582DE9F041234F3B78A8
:10549800012B054688463FD001233B704FF47A70B4
:1054A80000237B60FFF77CFF044688B92B68042B38
:1054B80013D11B4A536943F4803343F00403536107
:1054C8004FF47A70FFF76CFF0446154B1A681B6897
:1054D80000233B702046BDE8F0814FF0FF33C8F849
:1054E80000306E68D5E901321344B3420AD9304618
:1054F800FFF7BCFF4FF47A70FFF752FF50B1C8F8BE
:1055080000600446064A536923F47E7323F00203BD
:105518005361DAE70136E5E70224DBE7F806002005
:10552800004000582DE9F04F524C00234FF00F096E
:105538000A6832FA03F501D1BDE8F08F012505FAB2
:1055480003F818EA020200F08E804E68032706F07E
:1055580003054FEA430E07FA0EFC6F1E012F6FEA90
:105568000C0C32D8876807EA0C0ACF6807FA0EF7DE
:1055780047EA0A078760476827EA0808C6F300175A
:105588009F4047EA08074760C76807EA0C088F6822
:1055980007FA0EF747EA0807022DC76017D14FEA46
:1055A800D30800EB880803F0070AD8F820704FEA00
:1055B8008A0A09FA0AFB27EA0B0B0F6907FA0AF7A6
:1055C80047EA0B07C8F8207001E0032DDCD1076813
:1055D80005FA0EF507EA0C073D4316F4403F05604F
:1055E80041D023F0030707F1804707F5803703F020
:1055F800030CBD684FEA8C0C4FF0070E0EFA0CFE38
:10560800B0F1904F25EA0E0E2FD01B4DA8422ED098
:1056180005F58065A8420CBF0225072505FA0CF59B
:1056280045EA0E05BD602568D74316F4801F0CBFF8
:105638003D4015432560656816F4001F0CBF3D40CA
:1056480015436560D4F8805016F4803F0CBF3D4088
:105658001543C4F88050D4F88450B60354BF3D4075
:105668001543C4F88450013362E70025D6E70125C5
:10567800D4E700BF0008005800040048374A2DE965
:10568800F04F00234FF0010A4FF0070B4FF00F09BE
:1056980031FA03F401D1BDE8F08F0AFA03FC1CEAE1
:1056A800010654D023F0030404F1804404F5803447
:1056B80003F00307A568BF000BFA07F8B0F1904F95
:1056C80008EA050E45D0264DA84244D005F5806568
:1056D800A8420CBF02250725BD40754517D1D2F851
:1056E800805025EA0605C2F88050D2F8845025EA91
:1056F8000605C2F88450156825EA06051560556840
:1057080025EA06055560A56825EA0805A560056827
:1057180003265C0006FA04F423FA06F6254300EB98
:105728008606056003F00705376AAD0009FA05F536
:1057380027EA05073762856825EA04058560456814
:1057480025EA0C054560C56825EA0404C4600133F0
:105758009EE70025C0E70125BEE700BF0008005806
:10576800000400480369194214BF01200020704753
:105778000AB181617047816270470000044AD168AC
:10578800014208B502D0D060FDF7FCFF08BD00BF9C
:105798000008005810B5044600284AD090F8413057
:1057A80003F0FF021BB980F84020FCF771FE2423A8
:1057B80084F8413023681A6822F001021A6062688E
:1057C80022F070621A619A6822F400429A60D4E961
:1057D8000221012924D142F400429A605A6842F019
:1057E800007242F400425A60DA6822F40042DA6039
:1057F800D4E904210A43A16942EA0122DA60D4E922
:1058080007210A431A601A6842F001021A60002050
:105818002023606484F84130206384F8420010BD7E
:1058280042F4044202299A6004BF4FF400625A60AD
:10583800D4E70120F3E710B590F84120202A034669
:10584800D4B21CD190F84020012A18D0242280F824
:1058580041200268106820F001001060106820F4F0
:10586800805010601068014311601168002041F0F9
:105878000101116083F8414083F8400010BD022007
:10588800FCE710B590F84120202A0346D4B21BD17A
:1058980090F84020012A17D0242280F8412002687D
:1058A800106820F001001060106820F4706040EA71
:1058B800012111601168002041F00101116083F895
:1058C800414083F8400010BD0220FCE7024A1368FB
:1058D80043F4807313607047000400580D4B10B5F3
:1058E8005B690C4628B99A0507D500F027F820B15E
:1058F80010BD9B0501D400F019F8074A1369012C63
:1059080023F00403136101D130BFF1E740BF20BF8A
:1059180020BFEDE70004005800ED00E0024B1868D6
:1059280000F4C060704700BF00040058024A1368C2
:1059380043F4804313607047000400580C4A13680E
:1059480023F4804313600B4B1B6832214B430A49F5
:10595800B3FBF1F35169890500D533B9536913F4E1
:10596800007F14BF032000207047013BF2E700BF0F
:1059780000040058B800002040420F000B4A13688A
:1059880023F0070343F002031360094B1A69012847
:1059980042F004021A6105D130BF1A6922F00402EC
:1059A8001A61704740BF20BF20BFF6E700040058C7
:1059B80000ED00E04FF0B0431868C0F34040704776
:1059C8004FF0B0431868C0F3400070474FF0B04242
:1059D800536823F47F4343EA0023536070474FF032
:1059E800B0431868C0F34060704700007FB54FF0BF
:1059F800B0432C4AD3F80831C0F3031003F00F0367
:105A080052F82040284A52F82330B4FBF3F4FFF749
:105A180085FF264B054693E80700B5F5007F04ABE4
:105A280003E9070010D0224B9C4218D303F5B703B3
:105A380003F67F539C4229D903F5741303F51063C9
:105A48009C4225D802230BE01A4B9C4207D91A4BDB
:105A58009C421BD903F5370303F5D853F0E700231D
:105A680004AA02EB830353F80C4C144D2B6823F063
:105A7800070323432B60FDF71DF806462B6803F048
:105A880007039C4206D1002004B070BD0123E7E75C
:105A98000024EAE7FDF70EF8801B0228EED9032060
:105AA800F2E700BFD41B0108741B01085813010852
:105AB800C0CF6A00BFEA21013F933402004000587A
:105AC8004FF0B04310B59A68D96812F00C0205D0AF
:105AD8000C2A4AD101F00303012B50D14FF0B041F9
:105AE8002B480B6813F0080306D00B6813F0080363
:105AF80037D1D1F8941007E00C68240756BFD1F8C5
:105B080094300968C3F3032350F82330002A0CBFEC
:105B1800184600204FF0B0418A6802F00C020C2AA7
:105B28001ED1CA6802F00302022A2ED0032A06D127
:105B38000B68184A13F4801F174B18BF13464FF011
:105B4800B042D068D168D268C0F306205843C1F388
:105B580002130133B0FBF3F0530F0133B0FBF3F042
:105B680010BD0B68C3F30313CEE7042A0AD0082A32
:105B780005D11B6813F4801304D10748CAE7002332
:105B88001846C7E703480023C4E7024BD7E700BF1E
:105B9800D41B01080024F4000048E80108B5FFF709
:105BA8008FFF4FF0B043044A9B68C3F3031352F8C6
:105BB8002330B0FBF3F008BD741B01082DE9F04158
:105BC8000446002853D04FF0B0439D68DE68036850
:105BD8009B0605F00C0506F0030668D5026A1DB1A0
:105BE8000C2D46D1012E44D1002A40D04FF0B043AD
:105BF800A16A1A68170756BFD3F894301B681B09A7
:105C080003F0F00399421FD90846FFF7EFFE00287A
:105C18002DD14FF0B042136843F0080313601368A6
:105C2800A16A23F0F0030B431360606AFFF7CEFE0E
:105C3800FFF7B4FFAB4B1860AB4B1868FCF738FFA5
:105C4800002834D0BDE8F0814FF0B042136843F02B
:105C580008031360136823F0F0030B431360606AB2
:105C6800FFF7B4FE0846FFF7C1FE0028E0D0012088
:105C7800E8E74FF0B043002A54D01A6842F0010216
:105C88001A60FCF717FF0746FFF79AFE002842D074
:105C98004FF0B042136843F0080313601368A16A19
:105CA80023F0F0030B431360606AFFF78FFE23684D
:105CB800D80748D42368990700F18C8023681E0709
:105CC80040F1FA80A3694FF0B046002B00F0E18064
:105CD800D6F89430E16903F01002914200F0C480D4
:105CE80003F00302022AC2D0D80740F1B380D6F8E5
:105CF800943023F00103C6F89430FCF7DBFE074626
:105D0800D6F89430990740F1A580FCF7D3FEC31B61
:105D1800112BF5D904E0FCF7CDFEC01B0228B3D93E
:105D280003208FE71A6822F001021A60FCF7C2FE0E
:105D38000746FFF745FE0028B9D0FCF7BBFEC01B9D
:105D48000228F6D9ECE7082D03D00C2D05D1032E37
:105D580003D16368002BADD189E74FF0B043A16848
:105D68001A6822F480120A431A606268B2F5803F0A
:105D780010D11A6842F480321A60FCF79BFE07467D
:105D8800FFF718FE002895D1FCF794FEC01B642885
:105D9800F6D9C5E7B2F5041F04D11A6842F4001217
:105DA8001A60E6E7196821F480311960196821F44E
:105DB80000111960002AE0D1FCF77CFE0746FFF7C6
:105DC800F9FD00283FF476AFFCF774FEC01B642889
:105DD800F5D9A5E7042D236903D00C2D0ED1022E89
:105DE8000CD1002B3FF443AF4FF0B04261695368C8
:105DF80023F0FE4343EA016353605FE74FF0B04688
:105E0800BBB1336843F480733360FCF753FE074635
:105E180033685A0507D57368626923F0FE4343EA7D
:105E2800026373604AE7FCF745FEC31B022BEFD9F8
:105E380076E7336823F480733360FCF73BFE07464C
:105E480033685B057FF53AAFFCF734FEC31B022BC2
:105E5800F6D965E74FF0B042E169D2F8943023F003
:105E680010030B43C2F894304FF0B047D7F8943082
:105E780043F00103C7F89430FCF71CFE0646D7F838
:105E880094309A0718D4FCF715FE831B112BF6D90A
:105E980046E7D6F8943023F00103C6F89430FCF7AF
:105EA80009FE0746D6F894309B0705D5FCF702FE95
:105EB800C31B112BF6D933E72368580754D50B4F6A
:105EC8003B68D90514D4FFF701FDFCF7F3FD06463E
:105ED8003B68DA050CD4FCF7EDFD831B022BF7D9E0
:105EE8001EE700BFB8000020BC00002000040058D6
:105EF800E3684FF0B046002B58D023F08003052B01
:105F080002BFD6F8903043F00403C6F890304FF043
:105F1800B046FCF7CFFDD6F8903043F001030746B2
:105F2800C6F8903041F28838D6F890309B0705D4EF
:105F3800FCF7C0FDC31B4345F6D9F1E6E36823F03F
:105F48000403812B1BD1FCF7B5FDD6F8903043F044
:105F58008003C6F8903007464FF0B04641F28838C3
:105F6800D6F89030180504D5E06A00284AD10020F8
:105F780068E6FCF79FFDC01B4045F1D9D0E6FCF769
:105F880099FDD6F8903023F08003C6F89030074684
:105F98004FF0B04641F28838D6F890301905E3D56D
:105FA800FCF788FDC01B4045F6D9B9E6FCF782FD31
:105FB800D6F8903023F080030746C6F8903041F2B7
:105FC8008838D6F890301A0516D4FCF773FDD6F841
:105FD800903023F00103C6F8903007464FF0B048E0
:105FE80041F28836D8F890309B07BDD5FCF762FDA2
:105FF800C31BB342F6D993E6FCF75CFDC01B4045D2
:10600800DFD98DE60C2D4ED04FF0B04302281A6828
:1060180022F080721A6033D1FCF74CFD0546FFF779
:10602800DEFC38BBD4E90C314FF0B0420B43D068EA
:106038002D4901400B43E16B0B43216C0B43616C11
:106048000B43A16B43EA0123D360136843F08073C9
:106058001360D36843F08053D360FCF72BFD0446EC
:10606800FFF7BDFC002882D1FCF724FD001B0A289D
:10607800F6D955E6FCF71EFD401B0A28CFD94FE696
:10608800FCF718FD0446FFF7AAFC30B94FF0B04200
:10609800164BD1680B40D360D4E5FCF70BFD001B11
:1060A8000A28F0D93CE601283FF4CCAD4FF0B043C4
:1060B800226BDB6803F0030191427FF4D8AD616B7A
:1060C80003F070028A427FF4D2ADA16B03F4FE4262
:1060D800B2EB012F7FF4CBAD626C03F060439342C7
:1060E8003FF445AFC3E500BF8C80C111FCFFFEEE55
:1060F8002DE9F0410D46044610B90120BDE8F081B4
:10610800684E336803F007038B4216D323689A0757
:1061180027D54FF0B047A268BB6823F0F0031343BC
:10612800BB60FCF7C7FC0646BB68DB0319D4FCF769
:10613800C1FC831B022BF7D911E0336823F0070356
:106148000B433360FCF7B6FC0746336803F00703DC
:10615800AB42DBD0FCF7AEFCC01B0228F5D903200C
:10616800CCE72368580617D54FF0B0476269D7F8CF
:10617800083123F00F0343EA1213C7F80831FCF77C
:1061880099FC0646D7F80831D90305D4FCF792FCE8
:10619800831B022BF6D9E2E723685A0713D54FF081
:1061A800B047E268BB6823F4E0631343BB60FCF7C5
:1061B80081FC0646BB689B0305D4FCF77BFC831B6C
:1061C800022BF7D9CBE72368180714D54FF0B0474F
:1061D8002269BB6823F4605343EAC203BB60FCF73F
:1061E80069FC0646BB68590305D4FCF763FC831BAE
:1061F800022BF7D9B3E72368DA070FD4294C2368B1
:1062080003F00703AB4239D8FFF7C8FC264B1860E8
:10621800264BBDE8F0411868FCF74ABC6268022AC0
:106228001DD1FFF7C7FB00283FF467AF4FF0B0461A
:1062380041F28838B36823F003031343B360FCF7D3
:1062480039FC0746B368626803F00C03B3EB820FAE
:10625800D4D0FCF72FFCC01B4045F3D97FE7032AB5
:1062680002D1FFF7BCFBDEE712B9FFF7A9FBDAE7BB
:106278004FF0B0431B685B05D8D43EE7236823F092
:1062880007032B432360FCF715FC0646236803F03D
:106298000703AB42B8D0FCF70DFC801B0228F5D9E8
:1062A8005DE700BF00400058B8000020BC00002097
:1062B80008B5FFF773FC4FF0B043044A9B68C3F37B
:1062C800022352F82330D84008BD00BFB41B010890
:1062D80008B5FFF763FC4FF0B043044A9B68C3F36B
:1062E800C22352F82330D84008BD00BFB41B0108B0
:1062F8004FF0B043D3F89000C0F3400070474FF020
:10630800B0410209D1F8883002F47F22000123EA63
:10631800020300F47F200343C1F8883070474FF030
:10632800B041020CD1F88830120423EA020343EA90
:106338000040C1F88800704770B5066816F48036CA
:10634800044638D0FFF7C2FAFCF7B4FB614E0546A5
:106358003368DB0529D54FF0B043616BD3F8902043
:1063680002F44072914214D0D3F89010D3F89020E0
:1063780042F48032C3F89020D3F8902021F4407082
:1063880022F480328D07C3F89020C3F8900000F102
:1063980090804FF0B042616BD2F8903023F4407394
:1063A8000B43C2F89030002605E0FCF783FB401B46
:1063B8000228CDD903262568E8070AD54FF0B04151
:1063C8006268D1F8883023EA124392B21343C1F8C5
:1063D8008830A9070AD54FF0B041A268D1F88830B3
:1063E80023EA124392B21343C1F88830AA0609D5AA
:1063F8004FF0B0422169D2F8883023F440630B4350
:10640800C2F88830AB0502D5206AFFF788FF680517
:1064180002D5606AFFF783FF290502D5A06AFFF756
:106428007EFF6A0602D56069FFF769FF2B0602D571
:10643800A069FFF764FFE80502D5E069FFF75FFF91
:10644800E90610D54FF0B042E168D2F8883023F45D
:1064580040730B43C2F88830B1F5807F02BFD36820
:1064680043F08073D3602A040ED54FF0B042216BFD
:10647800D2F8883023F040430B43C2F8883019B96A
:10648800D36843F08073D3606B0410D54FF0B042EB
:10649800E16AD2F8883023F040530B43B1F1005F32
:1064A800C2F8883003D1D36843F48033D3603046D0
:1064B80070BDFCF7FFFA41F288360546FFF718FF72
:1064C80001283FF466AFFCF7F5FA401BB042F5D956
:1064D80070E700BF0004005830B590F82C30012B4D
:1064E80002464FF0020022D0174B82F82D00CA2432
:1064F800012582F82C505C6253245C62B1F5807FE0
:10650800146B996914D121F488519961596C24F05C
:10651800010421F0004159641463DD650A4BFF2131
:1065280059620020012382F82D3082F82C0030BDFA
:1065380021F408519961D96C24F0020421F000413A
:10654800D9641463D865E9E70028004070B50B4E9C
:10655800036B756D1D40EA07044603D50123F365F7
:10656800FCF719FCAB0704D50223F365204600F0BD
:10657800CBF9012384F82D3070BD00BF00280040FE
:1065880038B50A4CE36823F02003E360FCF792FA7D
:106598000546E3689B0601D5002038BDFCF78AFA5A
:1065A800401BB0F57A7FF4D90320F6E700280040B5
:1065B8002DE9F041114DEC6814F0400407461AD15A
:1065C800EB6843F08003EB60FCF774FA4FF00308C4
:1065D8000646EB685B0601D4032C02D12046BDE8D1
:1065E800F081FCF767FA801BB0F57A7F84BF87F8E3
:1065F8002D800324EDE70024F0E700BF00280040C9
:1066080038B50F4CE36823F08003E360A3699B0669
:10661800054606D4FFF7B4FF10B1032085F82D0016
:1066280038BDA36923F02003A361FFF7A9FF10B1C8
:10663800032085F82D00A36943F02003A361EFE749
:106648000028004038B5044600284BD090F82D307B
:1066580003F0FF021BB980F82C20FCF729F802236D
:10666800214D84F82D30EB68DB0632D4CA236B62E7
:1066780053236B622046FFF79BFF78BBAB6923F07F
:106688008E6323F04003AB6121696368AA690B43F9
:106698001343A2691343AB61D4E9022343EA0243DB
:1066A8002B61D4E90931EA680B4322F4F852134309
:1066B800EB602046FFF7A4FF80B9D4E90713AA6965
:1066C8000B4322F06042134362691343AB61FF231B
:1066D8006B62012384F82D30002002E0024BFF2278
:1066E8005A6238BD0120FCE7002800400023092831
:1066F80003D840EA0310C0B270470A380133C0B269
:10670800F5E700002DE9F04790F82C30012B0546FD
:106718004FF0020069D0012385F82C304E4B85F8E4
:106728002D00DE6806F44076B6F5807F78D04C6997
:10673800087891F8019091F802A091F82470002A45
:1067480055D19B6913F0400308BFCB70FFF7CEFF0C
:1067580080464846FFF7CAFF02465046FFF7C6FF85
:1067680081463846FFF7C2FF0B6ACF78234343EAD6
:10677800875343EA090343EA084343EA022343EA07
:106788000063354ACA205062532050628C6A886977
:10679800B4F5807F946945D124F488549461012428
:1067A800D465B6F5807F09BFCB691364034353648E
:1067B80018BF5064284B4A681A672A6B42F00102D6
:1067C8002A639A6942F488529A61244AD2F880303E
:1067D80043F40033C2F880301F4BFF225A62002076
:1067E800012385F82D3085F82C00BDE8F087B4F139
:1067F800803F07D0B4F5000F04D09B6913F0400325
:1068080008BFCB700B6ACA781C4344EA0A0444EAFE
:10681800004343EA092343EA825343EA0763B0E7A4
:106828000023AEE724F4085494610224D465B6F535
:10683800807F09BFCB6993640343D36418BFD064D6
:10684800054B4A685A672A6B42F002022A639A6922
:1068580042F40852B8E700BF00280040000800587A
:1068680090F82C20012A03464FF0020012D00A4A61
:1068780083F82D00CA21516253215162916941F078
:1068880020019161FF2151620020012283F82D200F
:1068980083F82C00704700BF0028004090F82C2097
:1068A800012A03464FF0020019D00D4A83F82D0043
:1068B800CA2151625321516291690A4841F080010D
:1068C8009161D0F8801041F48021C0F88010FF2138
:1068D80051620020012283F82D2083F82C00704794
:1068E8000028004000080058064B5A6D520610B5A3
:1068F800044603D54022DA65FCF750FA012384F8F0
:106908002D3010BD002800407047890001F18041FA
:1069180001F531410A607047890001F1804101F5B4
:106928003141086870470000034AD2F8903043F4B8
:106938000043C2F89030704700040058034AD2F868
:10694800903023F40043C2F8903070470004005898
:10695800074B1A6822F040021A6040F441704FF465
:10696800B85218605A601A6842F040021A607047BC
:106978000000015837B5054600284ED0837903F04A
:10698800FF046BB1032C0BD0254B4FF400629A61C6
:106998002868FFF7DDFF002401232B71AC602FE08E
:1069A80000236B712846FBF79DFF1E4AD2F89030F2
:1069B80043F48053C2F89030002CE5D102234FF005
:1069C800B042AB71D2F8943023F40043C2F894304B
:1069D800154B1B681C214B43DB0C64214B43019373
:1069E800019B93B90124AC60FFF79EFF0C4B9A689A
:1069F80042F400629A604FF400629A61002CC7D09A
:106A08000123AB71204603B030BD019B013B0193CC
:106A1800D2F894305B04E3D4E6E70124F2E700BF40
:106A28000004005800080058B800002037B5174D7A
:106A38002B6802461C204343DB0C64204343144864
:106A48000193019B93B901209060114C21732B682D
:106A58001C214B43DB0C64214B430193019B6BB915
:106A6800012090600A4BDB6803B030BD019B013BFD
:106A7800019383689C07E4D50020E6E7019B013B6E
:106A88000193A368DB07E9D5ECE700BFB800002055
:106A98000000015837B5184D2B6802461C204343A7
:106AA800DB0C6420434315480193019BA3B90120E3
:106AB8009060124CFF2323732B681C256B43DB0C5F
:106AC80064256B430193019B73B9012090600B4BC4
:106AD800DB680B7003B030BD019B013B01938368F9
:106AE8009C07E2D50020E4E7019B013B0193A368E2
:106AF800DB07E8D5EBE700BFB8000020000001582D
:106B08000F4B13B51B680F4C182253431B0D6422FF
:106B18005343014601936269019B02F0040223B9C1
:106B280002238B60012002B010BD019B013B019341
:106B3800606910F00200F6D0002AECD11046F2E7A6
:106B4800B80000200004005807B50379012B0FD1C5
:106B58000A4B1B68182253431B0C0193FFF7EEFEE8
:106B6800019B013B0193019B002BF9D1FFF7DCFE50
:106B780003B05DF804EBFFF7C3BF00BFB800002007
:106B8800F8B51E468379012B154604460F46DAB23E
:106B98002DD14379012B2AD0022342718371FFF74B
:106BA800D3FF0D212046FFF7C9FEFFF73FFF390A43
:106BB8002046FFF73BFFF9B22046FFF737FF2E4488
:106BC800B5420ED12046FFF7AFFEFFF799FFA06848
:106BD80001230038A3714FF0000318BF012063712F
:106BE800F8BD15F8011B2046FFF720FFE8E7022053
:106BF800F6E7F8B51E468379012B154604460F467D
:106C0800DAB22FD14379012B2CD04271FFF79CFFC8
:106C18001D212046FFF792FEFFF708FF390A20469C
:106C2800FFF704FFF9B22046FFF700FF00212046D6
:106C3800FFF7FCFE2E44B5420ED12046FFF774FE46
:106C4800FFF75EFFA06801230038A3714FF000032F
:106C580018BF01206371F8BD29462046FFF71AFFC7
:106C68000135E8E70220F6E7F8B51F468379012BDE
:106C7800154604460E46DAB22CD14379012B29D0A9
:106C88004271FFF761FF06F0EF03A3F1840253425C
:106C98005341237131462046FFF750FEFFF7C6FEE9
:106CA8002F44AF4210D1FFF73FFE842E02D020467A
:106CB800FFF726FFA06801230038A3714FF00003F7
:106CC80018BF01206371F8BD15F8011B2046FFF7B6
:106CD800ADFEE6E70220F6E7F8B51E468379012BFC
:106CE800154604460F46DAB227D14379012B24D042
:106CF8004271FFF729FF39462046FFF71FFEFFF7CD
:106D080095FE00212046FFF791FE2E44B5420ED194
:106D18002046FFF709FEFFF7F3FEA06801230038BD
:106D2800A3714FF0000318BF01206371F8BD294615
:106D38002046FFF7AFFE0135E8E70220F6E737B552
:106D48000023ADF8043001AA022312210546FFF7FB
:106D5800C3FFBDF80440022364BA01AAA4B21946CD
:106D68002846FFF781FFE20702D5284609F076FB9F
:106D7800A30702D5284609F077FB600702D5284605
:106D880009F09CFB210702D5284609F09DFBE20685
:106D980002D5284609F09EFBA30602D5284609F02D
:106DA80087FB600602D5284609F064FB210606D554
:106DB80014F4807118BF0121284609F061FBA2056F
:106DC80002D5284609F06CFB630402D5284609F071
:106DD80087FB03B030BDF8B51E468379012B1546F5
:106DE80004460F46DAB227D14379012B24D04271E9
:106DF800FFF7AAFE0E212046FFF7A0FDFFF716FEBB
:106E080039462046FFF712FE2E44B5420ED12046E1
:106E1800FFF78AFDFFF774FEA06801230038A3710D
:106E28004FF0000318BF01206371F8BD15F8011B6E
:106E38002046FFF7FBFDE8E70220F6E7F8B51E4617
:106E48008379012B154604460F46DAB22BD14379D4
:106E5800012B28D04271FFF777FE1E212046FFF74D
:106E68006DFDFFF7E3FD39462046FFF7DFFD002102
:106E78002046FFF7DBFD2E44B5420ED12046FFF732
:106E880053FDFFF73DFEA06801230038A3714FF0C2
:106E9800000318BF01206371F8BD29462046FFF79B
:106EA800F9FD0135E8E70220F6E7026852E8003FFD
:106EB80023F0C00342E8003102680029F5D102F14D
:106EC800080353E8003F23F4000302F1080C4CE8E0
:106ED80000310029F3D12023C0F888307047000022
:106EE80010B5026852E8003F23F4907342E800317D
:106EF80002680029F5D10F4C02F1080353E8003F5E
:106F0800234002F1080C4CE800310029F4D1C36E8B
:106F1800012B07D152E8003F23F0100342E800316B
:106F28000029F7D12023C0F88C300023C3664367BB
:106F380010BD00BFFEFFFFEFF8B504461346D4F8B6
:106F48008850202D32D1F1B1EAB1E06FA4F8562073
:106F5800A4F8542000262122C4F890602165C4F8C2
:106F68008820226888B1124FC762124F0763124FF8
:106F78002832C0E90D76FEF7D7F830B11023C4F8EF
:106F88009030C4F8885001200FE0236840221A622C
:106F9800226802F1080353E8003F43F0800302F13E
:106FA800080141E800300028F3D1F8BD0220FCE7D1
:106FB800C56F00080D7000081970000808B5034671
:106FC800806A1B681B6813F0200317D1A0F856309D
:106FD800026802F1080353E8003F23F080030832F7
:106FE80042E8003102680029F2D152E8003F43F03C
:106FF800400342E800310029F7D108BDFCF724F826
:10700800FBE7704708B5806AFFF7FBFF08BD7047CC
:10701800806A38B50468D0F88830D0F88C50A268F7
:10702800120606D5212B04D10023A0F85630FFF70D
:107038003CFFA3685B0606D5222D04D10023A0F8E7
:107048005E30FFF74DFFD0F8903043F01003C0F8E2
:107058009030FFF7DCFF38BD08B5806A0023A0F840
:107068005E30A0F85630FFF7D2FF08BD7047000029
:107078000368D9691A682DE9F04140F60F063142D4
:107088009D68044610D18E0640F1978002F02006D4
:1070980005F080573E4300F09080436F002B00F0CE
:1070A8008580BDE8F0411847AB4EAC482E401040F3
:1070B800304300F08280CF0709D5D00507D50120DD
:1070C8001862D4F8900040F00100C4F890008F07CF
:1070D80009D5E80707D502201862D4F8900040F0D7
:1070E8000400C4F890004F0709D5E80707D5042025
:1070F8001862D4F8900040F00200C4F890000F071E
:107108000BD502F02000304307D008201862D4F8CD
:10711800900040F00800C4F890000E050AD5500110
:1071280008D54FF400601862D4F8903043F020037B
:10713800C4F89030D4F89030002B37D08B0609D59E
:1071480002F0200205F080552A4303D0636F0BB18B
:10715800204698472668D4F89020B36802F02802A1
:1071680003F0400353EA0205204621D0FFF7B8FE9A
:10717800B3685F0617D5226802F1080353E8003F99
:1071880023F04003083242E800310029F3D1D4F853
:10719800800040B1724B8363FEF73FF830B1D4F8FA
:1071A8008000836B7DE72046FFF731FFBDE8F08163
:1071B800FFF72DFFC4F89050F8E7E06E012840F083
:1071C8008980CE0640F18680D00640F18380102267
:1071D8001A629A6851064BD5D4F8802011684A681B
:1071E80092B2002AE2D0B4F85C009042DED9A4F84A
:1071F8005E200A6892062FD453E8002F22F480728A
:1072080043E800210029F7D103F1080252E8002FD2
:1072180022F0010203F1080040E800210029F3D11F
:1072280003F1080252E8002F22F0400203F108009F
:1072380040E800210029F3D12022C4F88C20E1661F
:1072480053E8002F22F0100243E800210029F7D16B
:10725800D4F88000FDF7ACFF02232367B4F85E3052
:10726800B4F85C10C91A89B22046FFF7FFFE9DE703
:10727800B4F85E20B4F85E00B4F85C1080B292B244
:10728800002893D0891A89B200298FD053E8002F9B
:1072980022F4907243E800200028F7D1314D03F121
:1072A800080252E8002F2A4003F1080646E80020A9
:1072B8000028F4D12022C4F88C206067E06653E8E7
:1072C800002F22F0100243E800200028F7D1022303
:1072D8002367C9E7CF0209D56E0207D54FF480129C
:1072E80020461A62BDE8F04100F0A0BD08060BD5A3
:1072F80002F0800005F40005284305D0A36F002B99
:107308003FF454AF2046CCE64F0611D556060FD5AC
:1073180053E8002F22F0400243E800210029F7D16A
:107328002023C4F88830A1672046FBF78DFE3DE78F
:107338000D0206D5500004D52046BDE8F04100F006
:1073480077BDCB017FF532AF002ABFF62FAF2046BD
:10735800BDE8F04100F06BBD010000102001000401
:1073680061700008FEFFFFEFD0F88C20B0F86010C5
:10737800222A08B5036855D15B6A826D0B401370E9
:10738800836D01338365B0F85E30013B9BB2A0F892
:107398005E30B0F85E309BB2002B42D1026852E8F2
:1073A800003F23F4907342E8003103680029F5D1C7
:1073B80003F1080252E8002F22F0010203F1080C41
:1073C8004CE800210029F3D12022C0F88C20184A6B
:1073D80041679342016705D1C26E012A0ED0FBF7BF
:1073E80041FE1EE05A681102F6D553E8002F22F03C
:1073F800806243E800210029F7D1EDE70022C26648
:1074080053E8002F22F0100243E800210029F7D1A9
:10741800DA69B0F85C10D20644BF10221A62FFF78E
:1074280025FE08BD9A6942F008029A61F9E700BF93
:1074380000800040D0F88C20B0F86010222A08B5EF
:10744800036852D15A6A1140826D22F8021B826584
:10745800B0F85E20013A92B2A0F85E20B0F85E2043
:1074680092B2002A40D153E8002F22F4907243E8E8
:1074780000210029F7D103F1080252E8002F22F079
:10748800010203F1080C4CE800210029F3D1202265
:10749800C0F88C20174A41679342016705D1C26E34
:1074A800012A0ED0FBF7DEFD1EE05A681102F6D560
:1074B80053E8002F22F0806243E800210029F7D129
:1074C800EDE70022C26653E8002F22F0100243E8DD
:1074D80000210029F7D1DA69B0F85C10D20644BF60
:1074E80010221A62FFF7C2FD08BD9A6942F008022D
:1074F8009A61F9E7008000402DE9F74F0368B0F87A
:107508006080DF691A689D68D0F88C100192222982
:10751800044640F0B480B0F86890DFF86CA1DFF85A
:107528006CB10026B9F1000F01D0BB0621D4B4F824
:107538005E309BB2D3B1B4F868209A4216D922685B
:1075480002F1080353E8003F23F08053083242E871
:10755800003122680029F2D14D4B636752E8003FA1
:1075680043F0200342E800310029F7D103B0BDE819
:10757800F08F2368A26D5B6A03EA08031370A36D9A
:107588000133A365B4F85E30013B9BB2A4F85E30CA
:107598002368DF6978072CD0F9070AD5019AD20544
:1075A80007D501211962D4F8901041F00101C4F8FF
:1075B8009010B80709D5E90707D502211962D4F850
:1075C800901041F00401C4F890107A0709D5E80733
:1075D80007D504211962D4F8903043F00203C4F8A7
:1075E8009030D4F8903023B12046FFF710FDC4F84E
:1075F8009060B4F85E309BB2002B93D1216851E8BB
:10760800003F23F4807341E8003023680028F5D157
:1076180003F1080252E8001F01EA0A0142E80010DB
:107628000028F5D120215B45C4F88C1060672067DD
:107638000AD05968090207D553E8001F21F0806174
:1076480043E800100028F7D1E16E012913D1E6665E
:1076580053E8001F21F0100143E800100028F7D17B
:10766800D969CA0644BF102119622046B4F85C10D3
:10767800FFF7FCFC56E72046FBF7F4FC52E79A6953
:1076880042F008029A6171E7FEFFFFEF00800040B8
:10769800717300082DE9F74F0368B0F86080DF695F
:1076A8001A689D68D0F88C1001922229044640F08F
:1076B800B280B0F86890DFF868A1DFF868B10026FA
:1076C800B9F1000F01D0BB0621D4B4F85E309BB2EB
:1076D800D3B1B4F868209A4216D9226802F1080397
:1076E80053E8003F23F08053083242E80031226813
:1076F8000029F2D14C4B636752E8003F43F0200366
:1077080042E800310029F7D103B0BDE8F08F2368C3
:10771800A26D596A08EA010122F8021BA265B4F8B1
:107728005E20013A92B2A4F85E20DF6978072CD077
:10773800F9070AD5019AD20507D501211962D4F8AB
:10774800901041F00101C4F89010B80709D5E90775
:1077580007D502211962D4F8901041F00401C4F849
:1077680090107A0709D5E80707D504211962D4F8DB
:10777800903043F00203C4F89030D4F8903023B12D
:107788002046FFF744FCC4F89060B4F85E309BB222
:10779800002B95D1216851E8003F23F4807341E81C
:1077A800003023680028F5D103F1080252E8001FD1
:1077B80001EA0A0142E800100028F5D120215B45C2
:1077C800C4F88C10606720670AD05968090207D589
:1077D80053E8001F21F0806143E800100028F7D12A
:1077E800E16E012913D1E66653E8001F21F010016C
:1077F80043E800100028F7D1D969CA0644BF102110
:1078080019622046B4F85C10FFF730FC58E72046B0
:10781800FBF728FC54E79A6942F008029A6173E77B
:10782800FEFFFFEF008000403D74000838B50446B5
:1078380003682169A2681D68C0690A4361690A432F
:107848007D49024329400A431A605A68E16822F4D4
:1078580040520A435A60794AA16993421CBF226A7E
:1078680011439A6822F06E4222F430620A439A6009
:10787800DA6A616A22F00F020A43DA62704A9342B6
:107888001CD14FF0B043D3F8883003F0030343F41E
:107898004033A3F54033013B022B00F2C780694A0D
:1078A8009B5CB0F5004F40F08980082B24D8DFE8B6
:1078B80003F061C08323802323236500624A934237
:1078C80009D14FF0B043614AD3F8883003F00C0374
:1078D80043F44023E4E7594A93420DD14FF0B043B3
:1078E800D3F8883003F44063B3F5006F1AD005D895
:1078F80053B1B3F5806F12D0012009E0B3F5406FA2
:10790800FAD14FF400400EE0FEF7D2FC58B900203F
:107918004FF00113A3660023C4E91D3338BDFEF7F9
:10792800CFF8F3E74A4865684A4B626A05EB4501B8
:1079380033F81220B0FBF2F39942DDD8B3EB053FE0
:10794800DAD800231946FAF7DFF8090241EA10618C
:107958006B080002C0182A464FF0000341F10001ED
:10796800FAF7D2F83C4BA0F540729A42C4D8236883
:10797800D860CCE7FEF79CFC0028C8D06168354B7E
:10798800626A33F81220B0FBF2F24B0803EB4203B1
:107998004FF6EF72B3FBF1F3A3F110019142ABD8AC
:1079A80023F00F02216892B2C3F342031343CB6062
:1079B800ADE7FEF785F8DFE72548DFE7082B9BD81A
:1079C80001A252F823F000BF197A0008257A0008AE
:1079D800317A0008017900082B7A0008017900083B
:1079E8000179000801790008F57900084FF4004092
:1079F8006368616A174A32F81120B0FBF2F000EBB5
:107A08005300B0FBF3F04FF6EF73A0F11002ACE7B0
:107A1800FEF74EFC00283FF47AAFE9E7FEF758FC82
:107A2800F8E7FEF74DF8F5E70948E1E7B0F5004F4C
:107A3800F4D1FEF74DFC9FE7F369FFCF00800040CB
:107A480000380140141C010800440040171CF507C9
:107A58000024F400241C0108FFFC0F00836ADA07E5
:107A680010B506D50168C46A4A6822F40032224378
:107A78004A609C0706D50168046B4A6822F4803284
:107A880022434A60590706D50168446B4A6822F4C4
:107A9800802222434A601A0706D50168846B4A6827
:107AA80022F4004222434A60DC0606D50168C46B12
:107AB8008A6822F4805222438A60990606D50168B2
:107AC800046C8A6822F4005222438A605A060FD551
:107AD8000168446C4A6822F480122243B4F5801F7E
:107AE8004A6005D14A68846C22F4C00222434A6085
:107AF8001B0606D50268C16C536823F400230B43A8
:107B0800536010BD2DE9F041DDF8188004460E469B
:107B180015461F462268D36936EA03030CBF0123C2
:107B28000023AB4201D0002027E0B8F1FF3FF2D09C
:107B3800FAF7C0FFC01B4045206802D8B8F1000F13
:107B48001DD150E8003F23F4D07340E80032002AEA
:107B5800F7D100F1080353E8003F23F0010300F1D7
:107B6800080141E80032002AF3D12023C4F8883004
:107B7800C4F88C3084F884200320BDE8F0810368C1
:107B88005A07C7D5C3691B05C4D54FF40063036200
:107B980050E8003F23F4D07340E80032002AF7D1C0
:107BA80000F1080353E8003F23F0010300F1080146
:107BB80041E80032002AF3D12023C4F88830C4F801
:107BC8008C30C4F89030D5E773B504460026C0F869
:107BD8009060FAF76FFF23681B681A07054619D4E7
:107BE80023681B685B070AD56FF07E430093002269
:107BF8002B464FF480012046FFF784FFB0B90020E0
:107C08002023C4F8883084F88400C4F88C30E066F7
:107C180020670CE06FF07E430093324603464FF432
:107C280000112046FFF76EFF0028D9D0032002B0CC
:107C380070BD10B5044650B3D0F888301BB980F831
:107C48008430FBF7EDF822682423C4F888301368E1
:107C580023F0010313602046FFF7E8FD012816D042
:107C6800A36A13B12046FFF7F9FE23685A6822F485
:107C780090425A609A6822F02A029A601A6842F082
:107C8800010220461A60BDE81040FFF79DBF0120A1
:107C980010BD000030B581658168A0F85C20002324
:107CA800B1F5805FA0F85E20436735D10369002BEA
:107CB80040F2FF1318BFFF23A0F860300023C0F87C
:107CC80090302223C0F88C30016801F1080353E892
:107CD800003F43F00103083141E800340368002CF9
:107CE800F2D1456E84680169B5F1005F34D1B0F80E
:107CF8006850954230D8B4F5805F1DD1254A264C8E
:107D0800002918BF22464267C1B153E8002F42F448
:107D1800807243E80021F7E729B90369002B14BFF3
:107D28007F23FF23C8E7B1F1805FC5D10369002B2A
:107D38000CBF7F233F23BFE7174AE4E703F108029C
:107D480052E8002F42F0805203F1080040E8002179
:107D58000029F3D1002030BDB4F5805F0FD10F4A60
:107D68000F4C002918BF2246426751B153E8002F33
:107D780042F4907243E800210029F7D1EAE7084A63
:107D8800F2E753E8002F42F0200243E800210029DF
:107D9800F7D1DFE79D760008017500083D740008FB
:107DA80071730008D0F88C30202B30B415D1B9B1DC
:107DB800B2B100230468C3660A4B9C420AD06368C8
:107DC8001B0207D554E8003F43F0806344E80035C0
:107DD800002DF7D130BCFFF75DBF022030BC7047E3
:107DE8000120FBE700800040436E30B52BB901232A
:107DF800A0F86A30A0F8683030BD0368094D9A6869
:107E08009968094C490FC2F342626B5C615CDB0004
:107E1800B3FBF1F3A0F86A30AB5CA25CDB00B3FB08
:107E2800F2F3E7E7441C01083C1C0108704770475F
:107E380070471FB504AB03E9060090F88430012BA6
:107E480004463AD0012380F884302423C0F88830CF
:107E580003681A6822F001021A609A6822F4401234
:107E68000A439A6071B95A68BDF80C009DF80E1063
:107E780022F0100202435A605A6822F07F4242EA16
:107E880001625A601A6842F001021A60FAF712FE9B
:107E98006FF07E42034600924FF480010022204694
:107EA800FFF730FE38B92023C4F88830002384F85F
:107EB800843004B010BD0320F8E70220F9E790F8F9
:107EC8008430012B0FD0012380F88430016851E8F9
:107ED800002F42F0020241E80023002BF6D180F87F
:107EE8008430184670470220704710B590F88430E7
:107EF800012B044617D02423C0F8883003681A6879
:107F0800196821F00101196042F000524FF0005148
:107F180041661A60FFF768FF2023C0F88830002008
:107F280084F8840010BD0220FCE770B590F8843016
:107F3800012B044617D005682423C0F888302E6822
:107F48002B6823F001032B60AB6823F060431943CF
:107F5800A960FFF749FF20232E60C0F88830002071
:107F680084F8840070BD0220FCE770B590F8843076
:107F7800012B044617D005682423C0F888302E68E2
:107F88002B6823F001032B60AB6823F0606319436F
:107F9800A960FFF729FF20232E60C0F88830002051
:107FA80084F8840070BD0220FCE7000038B5084D55
:107FB800052455F8043B2BB9013C14F0FF04F8D113
:107FC800204638BDDB6898470028F5D0F9E700BFA0
:107FD8002C080020034BD870034B1B681B6C03B1A3
:107FE800184770474008002028080020034B1874E1
:107FF800034B1B685B6C03B11847704740080020AF
:1080080028080020F0B5314D314B95F90420314E48
:1080180091B00C46012795F905108DF804700228D7
:108028008DF809208DF80A1010D18DF80800D87144
:108038001C7202F09FFD337803B114B101A803F05C
:1080480003FA254B059A1A6011B0F0BD59714FF427
:1080580080711A71D9801C7233788DF8087053BBFF
:108068001F2306A88DF81C208DF8183002F064FF35
:1080780020238DF8183006A82B798DF81C3002F0D3
:108088005BFF22238DF8183006A86B798DF81C3019
:1080980002F052FF21238DF8183006A86B798DF86D
:1080A8001C3002F049FF29238DF8183006A80B4B25
:1080B800079302F041FF02F05DFD012306A88DF849
:1080C80018308DF81C3002F037FFB4E74008002064
:1080D800C00000201C080020200800200004000127
:1080E8007FB5092301A88DF8043003F0ADF90038F5
:1080F800044B059A1A6018BF0120404207B05DF88A
:1081080004FB00BF2008002070B504460B46134945
:1081180062784A700020A2780A7208701A884A7237
:108128009A788A72DB780B746368CB600C4B1B6897
:10813800DA6A2AB1237803F0FB030A2B00D09047B0
:10814800084E052556F8043B1BB15B6A0BB1204667
:108158009847013D15F0FF05F4D170BDCC00002013
:10816800280800202C08002070B504461048012378
:10817800037063784370A3788372E368C360E3781D
:10818800037623694376237943720A4B1B689B6AFB
:1081980003B19847084E052556F8043B1BB19B6967
:1081A8000BB120469847013D15F0FF05F4D170BD8D
:1081B800E0000020280800202C080020014B186847
:1081C800704700BF2008002000B58BB00123684627
:1081D8008DF8003002F088FD38B99DF804000038A9
:1081E80018BF01200BB05DF804FB0020FAE700007F
:1081F80008B501F073FE48B9FFF7E6FF012806D07D
:10820800054BD879197AFFF7FDFE012008BDBDE8B6
:108218000840FFF7CBBE00BFC00000202DE9F041A9
:1082280086B005460E46174601F058FE00287FD155
:1082380001F06CFE044640B9FFF7C6FF012807D0DD
:108248003D4B197AD879FFF7DDFE6FF0020462E042
:10825800DFF8E88088F80860003E18BF01268DF82E
:108268000460374E687833798DF81230694602F029
:10827800D9FC00283ED08DF804400394ADF8104096
:108288006FF0060495E803002E4B83E8030033796A
:1082980088F80A30394601A803F0DAF92A4B059A1A
:1082A8001A60112841D801A353F820F0138300085D
:1082B80039830008338300083383000833830008B8
:1082C800338300083383000853820008338300088F
:1082D80033830008338300082D83000833830008A4
:1082E800338300083983000839830008398300087C
:1082F800278300082B788DF808306B78ADF810309C
:108308006B6803934FF0FF34BCE7104B00221A70E0
:10831800E31D18BF1446204606B0BDE8F0816FF093
:108328000404F8E76FF00504F5E74FF0FF34F2E7CF
:108338006FF00104EFE700BFC0000020E00000205C
:1083480040080020F0000020200800202408002019
:1083580037B501F0E5FD144D052455F8043B5BB134
:108368001B694BB155F8043C9B682BB1984718B171
:1083780055F8043C1B699847013C14F0FF04ECD104
:10838800FFF714FE68B9094D2B7853B1084BADF8C7
:108398000040D978019422466846FFF73FFF00B9AC
:1083A8002C7003B030BD00BF2C080020240800202A
:1083B8004008002030B58BB0054601F08FFD04461B
:1083C800002839D1FFF700FF012838D168468DF819
:1083D800004002F089FC10B14FF0FF3004E09DF836
:1083E8000430AB4202D100200BB030BD012DF3D0D8
:1083F800022D11D0002DF7D1002BF4D068468DF84E
:10840800045002F099FD0028E6D10E4B1B681B6B47
:10841800002BE8D09847E6E7002BDDD168468DF8B9
:10842800045002F089FD0028D6D1064B1B681B6B4F
:10843800002BD8D02846EDE76FF00100D4E76FF0A5
:108448000200D1E72808002010B504468AB018B900
:108458004FF0FF300AB010BD002368468DF8003099
:1084680002F042FC0028F3D19DF804302370F1E7B4
:108478007FB500220B4620498DF8072001220A709B
:1084880042784A700446002A33D102790A721A885F
:108498004A729A788A72DB780B740369CB60C37866
:1084A800164D8DF80830037B8DF8093083680393E7
:1084B8002B68DB6A0BB102A898472B689B6B13B13A
:1084C800227E02B198470E4E052556F8043B1BB193
:1084D800DB690BB120469847013D15F0FF05F4D143
:1084E8000DF10700FFF7B0FF637913B1054B0122C7
:1084F8001A7004B070BD00BFCC000020280800200E
:108508002C0800202408002010B504468AB018B9A9
:108518004FF0FF300AB010BD202368468DF80030B8
:1085280002F0E2FB0028F3D1024A9DF904302370DF
:108538001371EFE74008002000B58BB023230190AA
:1085480068468DF8003002F0F7FC003818BF0120AB
:1085580040420BB05DF804FB70B5654C01468EB027
:108568001822204606F0ECF8624B00221A70FBF73E
:1085780047FF23784068012202FA03F1014004D141
:108588005D4B084608F0D2F8FEE75C495C481A469D
:1085980002F032F918B14FF0FF300EB070BD27234A
:1085A80004A88DF8103002F0C7FC564E564D00282E
:1085B80070D1012333702B68DB690BB10020984719
:1085C800272304A88DF8103002F08EFB059B93F842
:1085D8004820227093F8182193F81A316270A3701A
:1085E800464BD3E9020105F09DFF05460028D2D18C
:1085F800464E062304A88DF8103002F075FB059B43
:10860800736104A802F098FC022304A88DF81030C6
:10861800059602F069FB0836032304A88DF810308C
:10862800059602F061FB0F2606F040F8012304A826
:108638008DF814308DF8106002F07EFC10230DEBDD
:1086480003008DF810308DF8145002F075FC0423E7
:108658008DF8103004A8A3788DF8143002F06CFC63
:108668003A238DF8103004A86369059302F064FC7E
:1086780002A920788DF8086004F0E4F8003818BFE3
:108688000120E0711420FFF757FFE07903F0A4F907
:10869800284682E728238DF810302B681B6943B1E0
:1086A80004A802F021FB2B6805981B6940F2C4510D
:1086B8009847272304A88DF8103002F03DFC50B9E4
:1086C800012304A88DF8103002F00EFB9DF8143039
:1086D800002B7FF46EAF3378002B7FF46CAF05224C
:1086E80004A88DF81020059302F026FC78E700BF57
:1086F80040080020240800204C1C010868080020BD
:10870800800800201C0800202808002004080020F9
:1087180037B500230D4601930446D0B900F0A8FBF5
:108728000190019BD3B10F4A42F824300E4A9A6255
:108738000E4A1268916B1963916C596392690C49DE
:10874800D9625A6128465B680A49F2229847002094
:1087580006E001A900F092FB0028E2D04FF0FF30BC
:1087680003B030BD2C0800200D8000082808002028
:10877800E980000810070020194B07B51860194B4D
:10878800194A1A60194A5A60194A9A60194ADA60ED
:10879800194B02681A6042685A6082689A60C26817
:1087A800DA60164A1A6182695A61154BC26B5A60BF
:1087B800144A019119609A601946134ADA60002038
:1087C800FFF7A6FF48B901A800F056FB003818BF0C
:1087D8000120404203B05DF804FB4FF0FF30F9E799
:1087E800280800208008002071810008798400088A
:1087F800918800081181000868080020FDC700085A
:1088080058080020DD7F0008F57F000851B118B135
:10881800012804D000207047044B0B607047044BBC
:108828000B60F7E74FF0FF30704700BF000400010E
:108838000100010208B503F0EBF8002814BF6FF03F
:108848000100002008BD08B502F0BCF9002814BFDB
:108858006FF00100002008BD10B504468AB018B9B1
:108868004FF0FF300AB010BD212368468DF8003064
:1088780002F03AFA0028F3D1024A9DF90430237035
:108888005371EFE7400800202DE9F0412E4D2F4F9E
:1088980000232B7043786B703B689B6A8AB0044650
:1088A8000BB128469847DFF8A880052658F8043BFE
:1088B8001BB11B6A0BB120469847013E16F0FF0614
:1088C800F4D12378052B2FD00B2B35D0012B25D1B4
:1088D800204C062368468DF8003002F005FA01990D
:1088E800E07905F065FE10B91B4B019A5A611B48E7
:1088F800FFF70AFE1A48FFF7AFFF6B788BB9A37131
:10890800184B5878FFF756FD3B685B6A0BB1114866
:1089180098476B7813B9E07905F0DAFE0AB0BDE83C
:10892800F081FF23A371EFE70F4B01225A74227ADB
:108938009A74627ADA74F1E76378002BEED00AB0A1
:10894800BDE8F041FFF7CCBBE0000020280800207C
:108958002C080020C000002004080020C4000020CB
:10896800C500002040080020CC00002030B58BB0A6
:10897800FFF769FF0446F0B903F044FF831C1DD0DC
:10898800F8B9134D2B685B69DBB1272368468DF86E
:10899800003002F0A9F92B6801985B694FF4B961BE
:1089A800984703F041FF78B92CB9094B1B68DB697C
:1089B8000BB10120984720460BB030BD6FF007047B
:1089C800EFE74FF0FF34ECE74FF0FF34F3E700BF79
:1089D80028080020014B1878704700BF9408002031
:1089E800014B5878704700BF94080020704700007A
:1089F800044B9A7A0AB101225A70034B5B6903B19E
:108A08001847704794080020FC00002073B5224CDA
:108A18006378002B33D008F073F966680546FFF7D2
:108A2800CDFB0644AE4214D2A37A93B1E0228DF86E
:108A380000208DF80130217AE3680193012268460D
:108A4800FFF7ECFB08B1073010D100236370A37265
:108A5800656094F83430EBB1002384F834300F4B60
:108A68005B6BBBB102B0BDE87040184740F2DC5107
:108A78000B4808F011FA0A4808F0D4F9E8E794F826
:108A88003520002AE5D094F8360084F83530FFF711
:108A980091FCDEE702B070BD94080020FC000020C5
:108AA800CC08002037B5104D104CC8B1C1B1012316
:108AB800627200222860E16023700D480D4B00921D
:108AC8004FF0FF3108F002F900250B4825822022DB
:108AD800294605F049FE6570A574A58603B030BD2A
:108AE80000232B602370EFE79008002094080020F3
:108AF800CC080020F9890008A80800202DE9F047D3
:108B08008E4C23788CB0002B56D0C2780AB9837B60
:108B180013B1238A01332382437B002B4CD0E02AF4
:108B28004AD10023A372876897F80080B8F1220F12
:108B380027D8B8F1220F30D8DFE818F04100FB0041
:108B480052005A0061006E0075008E009D00B4004E
:108B5800C7002F002F002F002F002F002F002F00FD
:108B68002F002F002F002F002F002F002F002F0085
:108B78002F002F002F002F002F002F00C900D0003A
:108B8800D400B8F17E0F00F0CC80B8F17F0F00F070
:108B9800DF80B8F17D0F00F0AB80A57A002D00F0E2
:108BA8005B81674C637A3BB94FF47A71204608F0D1
:108BB80073F9204608F036F90CB0BDE8F087E36891
:108BC80001220021A2721970A37AE1689818A07294
:108BD8000620C854A37AE1689818A072CA54DCE742
:108BE800584B9B6A002BD8D0012102209847D4E724
:108BF8007B7884F83630012384F83530CDE70423B8
:108C08008DF804307B78003B18BF012301A88DF84C
:108C1800083002F091F9C0E77878003818BF0120D1
:108C280002F0DAFEB9E7484E0FCE01AD0FC50FCE00
:108C38000FC596E8070085E807007B780A2BACD8B3
:108C4800424A12685268002AA7D00CA901EB830394
:108C580053F82C0C9047A0E77878431E012B9CD83A
:108C68003A4B01381B6818BF012020729B68002B03
:108C780093D0984791E7E26801230821A372117005
:108C8800627A057BA17AAA4228BF2A46934284D2F7
:108C980085685A1CEB5CE56801334E1CA6726B5460
:108CA800D3B2EDE7E3680122A27209221A70A37A0F
:108CB800E268218A581CA072D154A27A238AE168FA
:108CC8001B0A501CA0728B5467E7238265E70523B3
:108CD8008DF8043001A802F0B7FB5EE7194BDB6A98
:108CE80098475AE7194B78781B686075DB68BEE7C8
:108CF800037B072B7FF451AF06238DF80430B7F8B8
:108D08000130ADF808307B793A791B0443EA022335
:108D1800FA781343642253430393BB798DF81030D8
:108D2800D8E73B2201A88DF804208DF8083002F01E
:108D380003F9012384F834302FE700BF940800209A
:108D4800CC080020FC0000206413010890080020D3
:108D58002A2301A88DF8043001F0C6FF94F80A9080
:108D6800E6689DF808009DF809509DF80A709DF87E
:108D78000BC09DF80D309DF80E209DF80F109DF842
:108D88000CE009F1010A84F80AA006F80980354EBA
:108D980094F80A903668D4F80C8009F1010A84F82E
:108DA8000AA096F803A008F809A094F80A90D4F845
:108DB8000C8009F1010A84F80AA096F802A008F8C4
:108DC80009A094F80A90D4F80C8009F1010A84F8F3
:108DD8000AA096F801A008F809A094F80A9009F1E9
:108DE800010A84F80AA096F80080E66806F8098067
:108DF80094F80A80E66808F1010984F80A9006F8F0
:108E080008C094F80AC0E6680CF1010884F80A80E2
:108E180006F80C70A77AE66807F1010C84F80AC016
:108E2800F555A57AE6686F1CA7727055A07AE568B3
:108E3800461CA6722954A17AE0684D1CA5724254BA
:108E4800A27AE168501CA0728B54A37AE268591C7C
:108E5800A17202F803E0A0E6034807F095FF6570E9
:108E6800AAE600BF90080020CC0800207047000048
:108E780000487047FC000020002070474FF0FF308A
:108E880070470000044B054A93F81831022B18BFAD
:108E9800062382F890347047A80E00207014002032
:108EA800034BD3F8483313B15B6903B118477047D4
:108EB80070140020034A137843F004031370FFF77B
:108EC800EFBF00BF6C1400201FB50A4B8DF80900D6
:108ED80093F87C208DF80A2093F88C2093F84800AA
:108EE8000D3202A98DF8082003F0ACFCC0B205B021
:108EF8005DF804FBA80E002010B5074C04F580604F
:108F080007F042FF94F81A3413B1012384F8193496
:108F1800BDE81040FFF7C4BF7014002010B50C4C1A
:108F2800D4F8403343F08003C4F8403394F81A343B
:108F380013B10020FFF7E0FF94F8913423F01203F7
:108F480043F0120384F89134BDE81040FFF79ABF4C
:108F5800701400202DE9F041DFF8AC8098F8183142
:108F6800022B06460D4602D0284BDB6A984702F0D2
:108F7800E9FD044628B1022002F0DAFD002002F0E3
:108F8800DCFD98F81831012B17D102F0DDFD0746FA
:108F980030B1002002F0CDFD002002F0CFFD3C46AC
:108FA80002F0D4FD48B1002002F0C4FD002002F018
:108FB800C6FDBDE8F041FFF765BF002CF9D1144CA0
:108FC80094F8902494F81A34BAB90BB184F841642F
:108FD800304602F065FFD8F82C0007F09BFED4F865
:108FE800B4339842E5D30B4807F0CEFE94F8913499
:108FF80043F0100384F89134DBE70BB184F8415453
:10900800284602F04DFFF1E7A80E0020CC23010806
:10901800701400200818002073B5164C164D04F57E
:109028007A76EB6C95F8502095F9781095F8480009
:10903800009603F02DFC95F8303184F8FC3395F850
:10904800480040F2012304F224423146A4F8FA33DE
:1090580003F02AFC58B194F8243484F86A34074B96
:1090680000205B6B984794F8FB3384F8903402B087
:1090780070BD00BF70140020A80E0020CC2301088A
:10908800074A10B5137843F002031370FFF708FF7F
:10909800BDE81040034B01220021022007F046BB27
:1090A8006C140020951C0108074A10B5137843F08A
:1090B80008031370FFF7F4FEBDE81040034B0122CC
:1090C8000021022007F032BB6C140020A51C010807
:1090D8002DE9F0410F4616461D46804607F010FE62
:1090E8000B4A0C4C1378278123F0110343F011032A
:1090F8001370C4E9000866812573FFF7D1FEBDE847
:10910800F041054B01220021022007F00FBB00BFF0
:109118006C1400201C1A0020B51C010813B507F0B8
:10912800EFFD0D4B6C461860204607F03DFD94E8B6
:1091380003000A4A0A4B83E80300137843F020032C
:109148001370FFF7ADFE074B01220021022002B089
:10915800BDE8104007F0EABA2C1A00206C14002071
:10916800A8170020C21C0108F8B5334D95F818411E
:10917800012C06464BD0022C51D064B938B9D5E938
:109188001B0105F1740383E803002046F8BD01289C
:109198003DD0022801D00324F7E7284F85F81801AD
:1091A80007F5747EBEE80F0007F57A7CACE80F007F
:1091B8009EE8030095F8E9308CE8030087F8FB6324
:1091C800E3B195F80031022B18D1D5F804316B675B
:1091D800C7F8EC3395F87D3095F8082187F8F8330F
:1091E80095F88C3085F8782087F8F93397F81B24A0
:1091F80087F8E82340F20133A7F8FA33002387F809
:109208001A340F4BDB6A9847FFF706FFBDE702F0F9
:10921800A4FC04460028B8D185F81861B5E70028F1
:10922800B9D1064B85F81801062283F89024044B1F
:10923800DB6A98473446A8E7A80E0020701400207F
:10924800CC2301082DE9F04192B0064602F07AFCE1
:10925800002840F05981AD4D95F81831012B09D0FF
:109268002B6BAB4C93B194F80431BBB1042B6FD08A
:10927800032003E002F068FC18B10F2012B0BDE82B
:10928800F08102F063FC0028EAD0F6E7B5F8203157
:10929800D4F81C24013B53432B63E4E79D4803F0B7
:1092A80008FA002840F02C8194F80C3123802B6BAD
:1092B8000C930DF1180895F839308DF83830404680
:1092C80095F81C318DF83A3007F094FCD5F8283120
:1092D800009302AF98E80600D5F82431384607F025
:1092E80020FC97E803000FAB83E80300EB6A0D93BB
:1092F80000238DF844302388ADF8463095F8303196
:1093080001228DF839201BB98DF844208DF83930A9
:10931800814B0093814B95F84800A3F179020CA981
:1093280003F005FBC0B10B28A8D1D4F8941499B167
:10933800002EA3D0D4F84033794843F02003C4F872
:10934800403307F0A9FD764807F06CFD002095E74B
:10935800704803F0E2F9A4E795F8487095F9693088
:1093680095F9392095F87D106E4E384603F0ECFAE1
:10937800009641B2EB6C95F850203846183603F049
:1093880087FA0096EB6C95F8502095F9701095F8CF
:10939800480003F07DFAD4F8C413AB6DD4F8DC238D
:1093A8000B44C4F8B033EB6D1344C4F8B43394F8E9
:1093B8000431042B07D02B6E0B44C4F8B0336B6E0A
:1093C8001344C4F8B4330023089395F8303183B1BB
:1093D80008A802F095FC00284ED195F9390094F8B8
:1093E80037629DF82070FFF76FFD3E4480B2B042AF
:1093F80040D300238DF8133095F839308DF821309B
:1094080095F838308DF82230D5F880300993D5F8A2
:1094180084300A932388ADF82C3095F8303194F8CD
:109428001B648DF82E3095F848003F4B8DF820606E
:109438000DF1130208A903F03FFA012384F841341F
:1094480095F8393084F842349DF8133084F8433461
:10945800D4F81C34C4F85064C4F84834C4F85834F8
:1094680002F076FB50B1D4F81C0402F083FB28B15B
:10947800102003E7082001E71320FFE695F81831CC
:10948800012B01D102F078FB02F065FB0023059364
:1094980094F8043195F9395094F81B649BB1042B66
:1094A8007FF4E6AE05A802F067FE58BB94F81834BE
:1094B80013B1059B013B0593164B05983246E9B25B
:1094C80002F0BCFE02E0134802F090FEC0B9D4F8E6
:1094D800403394F80C11218043F00203C4F8403360
:1094E80094F8183411480133DBB284F8183484F83E
:1094F80045340F4B00259B6AC4F89854984725E7D4
:109508001120BBE61220B9E60E20B7E6A80E00200F
:109518007014002078150020D80E002004190020AF
:10952800D8170020281800208C180020721400205A
:10953800CC230108F0B5504C504EB4F8DC202287FB
:10954800D4E92D0194F8B12084F8692004F16C0263
:1095580082E80300D4E92F0104F1740282E80300D1
:10956800B4F8C420A4F87C2091B0D4F8CC20D4F866
:10957800C810C4F884200025D4F8D020C4F8882066
:109588000123A4F82031C4F8801084F83051A56272
:1095980084F81B5184F83A5084F81D5184F81E5100
:1095A800C4F83451C6F89854A6F8185486F81A54D2
:1095B800A4F838518DF8183004F50973039304F5AD
:1095C8000A7394F84800A4F84651049303A92C4B55
:1095D80084F84551C4E94F55059303F041F9E36E0A
:1095E800C6F8D43394F87D3086F8E03394F88C309C
:1095F80086F8E1334FF48073A6F8E23386F8D05347
:1096080094F8303186F8E43306F574770FCF06F511
:109618007A740FC497E8030040F2012384E803003A
:10962800A6F8FA33D6F8483386F81B54CDE9015525
:109638001BB15A685B6901920293124B0793A3F11D
:1096480048020892A3F1140209920F4A0B92293397
:109658000A93A2F19C030C93A2F198030D93131D96
:109668000E9301A902F14C0307A802F599620F9322
:1096780002F05DFA11B0F0BDA80E002070140020B1
:109688008C190020D81800208C0F0020F8B50D4F39
:109698000D4C0E4E0D4607F077FB3B6B984796F83E
:1096A800480004F22442294603F0FEF848B194F831
:1096B800243484F86A34706D7B6B9847EB7C84F8AB
:1096C8009034F8BDCC23010870140020A80E0020A7
:1096D8000F4890F81B3480F8B8330E4B93F8692084
:1096E80080F8BB2393F87D2080F8C82393F88C205A
:1096F80080F8C92393F8303180F8CC330022A0F8E1
:10970800CA2300F56E7100F56070FFF7BFBF00BF98
:1097180070140020A80E0020114890F89034EBB186
:1097280090F81B3480F8D0330E4BDA6EC0F8D4238F
:1097380093F87D2080F8E02393F88C2080F8E123CB
:1097480093F8303180F8E4334FF48072A0F8E223C4
:1097580000F5747100F56670FFF798BF704700BF99
:1097680070140020A80E002070B5344C2421204627
:1097780004F0FCFF636A984218BF60624FF01C0156
:109788002F4814BF0125002504F0F0FF636C9842B0
:1097980018BF60644FF480712A4818BF45F002056D
:1097A80004F0E4FFD4F84831984218BFC4F84801DF
:1097B8004FF0D401244818BF45F0040504F0D6FF43
:1097C800D4F82032984218BFC4F820024FF00001A4
:1097D8001E4818BF45F0080504F0C8FFD4F8243225
:1097E800984218BFC4F824024FF46071184818BF93
:1097F80045F0100504F0BAFFD4F8A835984218BF10
:10980800C4F8A8054FF01401124818BF45F0200508
:1098180004F0ACFFD4F8C03598420F4B18BFC4F819
:10982800C005D3F8483318BF45F040052BB11B6974
:109838001BB12846BDE87040184770BDA80E00202F
:10984800D00E0020F00E0020F40F0020CC100020D5
:10985800D010002054140020701400202DE9F04F7F
:1098680091B04FF00008012B05460F4602928DF883
:109878001580ADF8188003D8C84EC146B94502D343
:1098880011B0BDE8F08F15F8090002F077FA4844E6
:10989800B842F5DC15F8093009F10104023BE4B2DD
:1098A800112BEDD801A252F823F000BFFD98000853
:1098B8002F9900082F9A0008599A0008E19A000881
:1098C800099B00087B9B0008AD9B0008299C0008A9
:1098D8008998000889980008879C000889980008DA
:1098E80089980008459D00086D9D0008B19D0008F5
:1098F800EF9D0008052002F0EDFA90B10521002047
:1099080002F0ACFA2A5DA64B09F1030409F1020939
:109918005FFA89F983F85C2415F8092083F85D2437
:10992800E4B2A146AAE700238DF816308DF8173067
:109938008DF81C308DF82030B8F1000F6CD14FF045
:10994800050896F87C208DF83920631E96F8392092
:109958008DF83B202B4496F838200D938DF83C2049
:1099680096F81A3196F868208DF83D20D6F82C2103
:109978008DF83A300C9273B37B1C1B1BDBB28DF84D
:10998800383008AB019307AB009396F848000DF107
:1099980017030DF116020CA902F09AFF8DF81500B5
:1099A80000F00700072813D196F939209DF91630E1
:1099B80086F839309A429DF8173086F83830B8BFA3
:1099C80001229DF81C30B8BF86F81D2186F8683042
:1099D8004FF0000909E00523D1E701220DF1150137
:1099E800032002F0DBF809F101095FFA89F29DF81A
:1099F8002030B3FBF8F19142EFD82344DCB2631E68
:109A0800DBB29F420DD9EA5C032A9AD0A74288BFED
:109A18001C464FF0010884E709F105095FFA89F44B
:109A2800F7E71C46F5E72B5D012203F00F0309F168
:109A3800020986F81B3102FA03F35FFA89F9A6F8DE
:109A48002031002206A9042002F0A8F84C4668E755
:109A580007238DF815302B5D96F84800C3F30212E2
:109A680003F00F038DF8303009F10303DBB28DF8F2
:109A78003120EA5C09F10403DBB209F10504EB5C6F
:109A880009F102095FFA89F91B0443EA022315F870
:109A980009201343642253430CA90D9302F027FFB6
:109AA80000F00703072BE4B28DF815000CD19DF8E0
:109AB800303086F8703086F878300D9BF36673671F
:109AC8009DF8313086F869308DF81800012206A912
:109AD800052002F063F824E7314BD3F848336BB123
:109AE8001B685BB19847029B8DF8180003F03F0391
:109AF8008DF81930022206A90620EAE7FF20F2E7CE
:109B080003238DF815302B5D8DF824300CAB0893AA
:109B180009F10303DBB209F10604EA5C96F8480090
:109B280009F10403DBB208A9EB5C1B0443EA022336
:109B380009F10202D2B209F10509AA5C13436422B1
:109B480053435FFA89F90C9300230D9315F80930F4
:109B58008DF8383002F0D1FEC3B20028E4B28DF897
:109B68001530FFF6DEAE8DF81830012206A9072061
:109B7800AFE72B5D03F00F03012B4FF47A7238BF68
:109B88000123534309F10209B36513445FFA89F9C4
:109B9800F365002206A9082056E700BFA80E00209A
:109BA800701400202B5D96F84800C3F340128DF81E
:109BB8001D2007A9C3F3001203F00F038DF81C2022
:109BC8008DF81E3002F09FFE09F1020901305FFA9C
:109BD80089F93FF43BAFBDF81C30914AA6F87C30B8
:109BE8009DF81E309DF81C40D05CF7F70FFF02234C
:109BF800C6F880000CA996F848008DF830308DF82A
:109C0800324002F01FFE96F93930089040B298426F
:109C1800B8BF184686F83900002206A9092013E7BC
:109C280003238DF815302B5D8DF8303009F10303CF
:109C3800DBB209F10504EA5C96F8480009F104036F
:109C4800DBB209F10209EB5C5FFA89F91B0443EA0C
:109C5800022315F809201343642253430CA90D93DA
:109C680002F057FEC3B20028E4B28DF81530FFF6B3
:109C780058AE8DF81830012206A90A2029E70920D4
:109C880002F028F9DFF89CA1002854D0092100200F
:109C980002F0E4F80023ADF8263009F10203DBB244
:109CA8004FF47A71EA5C09F10303DBB20DF1300B72
:109CB800EB5C1B0443EA02232A5D134309F1040207
:109CC800D2B209F1060409F10509AA5C5FFA89F91B
:109CD80043EA026315F8092003934A4312125846CF
:109CE800ADF8242006F060FF039B03F1965303F5BB
:109CF800A91303F5EC530893DAF83C3300930DF1FC
:109D0800200999E80600DAF838330AA806F009FFAE
:109D18000B9B00939BE806000A9B484606F0E6FE6C
:109D280099E8030006F018FF01F021FF0123E4B2CF
:109D38008AF83834F5E58AF83804F2E50C2002F0A0
:109D4800C9F800283FF4EDAD0C21002002F086F898
:109D5800344B93F89034043B012B7FF6E2AD01F0CD
:109D680002FFDEE509F10203DBB22A5DE95C09F1D5
:109D78000303DBB209F10504EB5C09F104095FFA9E
:109D880089F91B0415F8090043EA012313436421E8
:109D9800594300F00F0001F0E7FEE4B28DF8180017
:109DA800012206A9112094E60D2002F093F800285C
:109DB8003FF4B7AD0D21002002F050F809F102037D
:109DC800DBB2194AE85C2B5D126809F1040409F159
:109DD80003095FFA89F943EA002015F80910E4B28B
:109DE80001F0C4FE9DE52A5D09F1020309F10404AE
:109DF80009F10309DBB25FFA89F9E95C15F8093062
:109E08001B0443EA012313436420584301F0B0FEC6
:109E1800E4B28DF81800012206A9132059E600BF04
:109E2800CF1C0108701400201C1A00200E4B93F858
:109E38009124920703D593F88F24012A08D90B4956
:109E480091F81A2122B18A6A501C18BF01328A621D
:109E58000022A3F8182483F81A24D3F8402322F008
:109E68000202C3F84023704770140020A80E002097
:109E780070B5184C184D04F55A7006F085FFD4F8E3
:109E88004033D4F89804D5F8906023F02003C4F840
:109E9800403338B106F03EFF864203D2002385F8EE
:109EA8003A3070BD0120FFF7CDF90028F9D00B2812
:109EB800F7D095F8393084F84234092094F81834EA
:109EC80084F8453484F8410401F0EAFFBDE87040A5
:109ED800FFF7ACBF70140020A80E0020094BD3F880
:109EE8004023012A0AD008490978C90708D43AB991
:109EF80093F89204013818BF01207047002070477A
:109F080001207047701400206C140020034BD3F814
:109F18004003431E58425841704700BF7014002048
:109F28002DE9F04FA9B0EFF3108272B6DFF8F48292
:109F38000021D8F80030C8F8001082F31088BA4C15
:109F4800002B00F0E480DAB29B06039264D5B74D8B
:109F580095F81831022B02D0B54BDB6A9847EFF31E
:109F6800108972B6B34F06F0CBFE3E68D4F8B01332
:109F7800361A3144B04806F08FFFAF4806F052FF5A
:109F8800D4F8B413AD48314406F086FFAB4806F068
:109F980049FF89F3108894F81A34002B00F06D817A
:109FA800152312A995F848008DF8483002F04AFCAC
:109FB800D4F8B4130F900144A14806F06DFFA048EF
:109FC80006F030FF3B6894F81B24EB620DAF38466F
:109FD8008DF870201D9306F00DFED5F828310093FA
:109FE80006AE97E80600D5F82431304606F099FD0C
:109FF80096E803001FAB83E80300D4F81C341E93D3
:10A0080095F8303195F84800003B18BF01231CA98A
:10A018008DF8713002F01FFC039BDF064BD5834D92
:10A02800DFF820A2D5F8E420BAF90A30059298F8AA
:10A0380000200493002363F300020A9388F80020A9
:10A0480084F84434049AA4F8223484F82534C4F8F3
:10A058002834A4F82C3484F82E34C4F8303484F826
:10A068002034C4F8343484F83834C4F83C34704BA1
:10A078009AF90C90A4F88C2494F89024DB6A84F85C
:10A088008E9484F88F24DAF80470BAF80860984738
:10A0980094F88F3413B9694806F076FE314638468D
:10A0A80001F04EFD8346002800F0EA80049BA4F8E6
:10A0B8007E3484F88094039B19071AD55B4B93F878
:10A0C8001831022B02D05A4BDB6A98470220FEF760
:10A0D800D9FE84F8410401F0E3FE94F81A3413B170
:10A0E800012384F8193494F8913443F0100384F868
:10A0F8009134039B5A0703D506210520FEF72AFF52
:10A10800039B9B0703D504210320FEF723FF01F0DF
:10A1180035FD94F89124D7065FD5002384F892344E
:10A12800D4F840331E0644BF23F08203C4F84033FA
:10A1380012F0050F00F0FC820B2001F0CBFE002886
:10A1480000F0F68294F89134DD0700F1F1825807A7
:10A1580040F10883D4F8403323F00203C4F84033B5
:10A16800D4F8402382BB94F8915415F001011EBF26
:10A178002B4662F3000384F8913494F891345E0717
:10A1880044BF6FF3820384F89134012384F8923436
:10A1980021B1D4F844332C481B6898476D070BD578
:10A1A8002A4801F0A3FE01F0D1FE28B194F89134B9
:10A1B80043F0040384F8913401F0CEFC94F8913410
:10A1C8006FF3041384F89134012384F8923494F8DB
:10A1D800913443F0200384F8913494F891341807AB
:10A1E8000AD56FF3C3031A4984F89134D4F8443379
:10A1F800A1F12400DB68984794F8913499070AD5AF
:10A208006FF34103124984F89134D4F84433A1F12F
:10A218006C005B68984794F89034022B1AD1FEF7CB
:10A22800FBFE17E06C14002070140020A80E00201C
:10A23800CC2301082C1A0020F01700200818002051
:10A24800701800201C1A0020B0180020C418002024
:10A25800FC18002094F891349A0640F1C6826FF3F6
:10A26800451384F89134D4F84033002B40F0BD8274
:10A2780029B0BDE8F04FFFF777BA84F84134A1E67A
:10A2880095F81821012A0CD101F05EFC804668B1CE
:10A29800584601F04EFC584601F050FC042384F85F
:10A2A8008F347EB9012384F8213450E101F04EFC4B
:10A2B8000028F6D0404601F03DFC404601F03FFC46
:10A2C8000523ECE73B7804935B09013B062B00F27E
:10A2D8001882DFE813F007001602950016029200B4
:10A2E80016020702102EDDD995F830311297F6B212
:10A2F8008DF84C60002BD5D11CA804F04BF912AA9C
:10A308001CA9FF2002F0AEF89DF85830C3F30303F0
:10A3180007468DF82C3095F8480095F87D308DF873
:10A328002D3007220BA902F0A0FA002F5DD10028DA
:10A338005BD09DF853309DF852201599C5F8E4106C
:10A348001B0443EA02239DF8512002201343C5F859
:10A35800E03004F02DF99DF8583095F8480085F85C
:10A368002E71C3F30212C3F3030385F8703085F826
:10A3780078309DF8593085F86920012B38BF0123C2
:10A388004FF47A725343AB651344EB650DF15A03EE
:10A398004FF001081093113E94F81B348DF83C30AF
:10A3A8000FA985F868808DF8446002F066FA0223E8
:10A3B800404685F8303101F08DFD18B141463846E8
:10A3C80001F04CFD94F88F34012B00F2A88194F829
:10A3D8001A34002B40F09B8194F8913443F0100319
:10A3E80084F89134FEF74EFD65E6012001F072FD18
:10A3F8000028E7D001210720E2E7012384F8203470
:10A4080095F87D308DF82E3094F824348DF82D3061
:10A4180095F88C3095F848000D330BA98DF82C3041
:10A4280002F010FAA6F10D031BB2099023EAE373B8
:10A4380000B283423FF736AF0B2E7FF633AFBB4BEC
:10A4480025931CA8FF231C978DF874608DF898300D
:10A4580002F0D4F8074600287FF424AF95F81831A5
:10A46800012B13D101F070FB002873D0384601F09E
:10A4780060FB384601F062FB04239DF87C101E98AF
:10A4880084F88F34C1F3001101F077FB9DF87C301C
:10A498001E99C4F8341413F00F0203D09DF89000ED
:10A4A800002863D19DF89800002862D0002A7FF424
:10A4B800F9AE9DF89020002A0CBF4FF002084FF02B
:10A4C800030800220A92D5F8EC20914254D195F85D
:10A4D800E910002950D0D5F80C1195F8EAB00968B0
:10A4E8000A9195F81811022902D1032184F88F14D2
:10A4F800B8F1030F7FF4D6AE13F0600F7FF4D2AE3D
:10A508000592012795F82E31BBF1000F37D0BBF12A
:10A51800010F38D1012B34D16FF0090646FA08F63D
:10A5280006F00106C6F10206F6B2BDF87E100AAAC8
:10A53800304601F02DFE40B307280CBF0823012345
:10A5480084F821340A9BC4F83034C4F86C34FEF71C
:10A55800E5FCB0E501F0FAFA002897D0384601F09A
:10A56800E9FA384601F0EBFA052386E74FF00008D0
:10A57800A7E74FF00108A4E74FF0010BC2E7042654
:10A58800D3E70326D1E70123DAE71CAB009305994B
:10A598000A9B3246584601F0B7FE20B102280CBF8C
:10A5A8000A230B237FE60A9BC4F83034C4F86C34C2
:10A5B8009DF87C3084F82104C3F3401384F82E34CA
:10A5C80084F8443494F88F3484F82274012B9EBFA5
:10A5D8000122A86285F81E21012FC4F8280484F8F6
:10A5E8002C0484F8410438D1022284F8202495F8F8
:10A5F8003A20002A4AD19DF87C20D60646D4012B61
:10A6080094F840149DF87C2005D8012901D19006C2
:10A6180001D501F05FFBB8F1020F94F88F3443D0F5
:10A62800B8F1030F0AD09DF87C10B8F1010F4A4623
:10A6380001F00F0120A83BD0FFF710F99DF89030EA
:10A6480084F82334259BC4F828349DF8983084F87E
:10A658002C34012384F82D3430E0049A02F0E0020F
:10A66800A02A1BD195F82E11012285F83A2009B9A4
:10A6780027996963012B84F8202407D9D5F89020FD
:10A68800C4F83C24DAF80020C4F8982495F8182176
:10A69800002AB4D1012284F82524B0E7002285F8E5
:10A6A8003A2084F82024A6E79DF8981025984A4671
:10A6B800FFF7D4F89DF8903084F823349DF8902063
:10A6C800E02A08D195F81F312BB984F82324C4F85F
:10A6D8002834A4F82C3494F8913443F0020384F815
:10A6E80091346FE6114D013EB2B2791C284604F050
:10A6F80027F80323A4F82034C4F8285484F82C64D9
:10A70800E9E7012384F82134FEF708FC5AE694F8B7
:10A718004434002B3FF460AE0020FEF7EDFB94F8C4
:10A728008F34022B3FF45EAE56E600BFA816002019
:10A7380094F89134590715D5012001F0CBFB60B18D
:10A74800012001F09DFB08B984F81804D4F84033BF
:10A7580023F00203C4F8403304E0062001F0BAFBFA
:10A768000028F3D194F89134DA077FF5F9AC94F81E
:10A7780040240AB1032A18D11D4A94F8181492F8F3
:10A788006820914205D29B0723D594F88F34012B7A
:10A798001FD8184806F0F8FAD4F8403323F02003FD
:10A7A800C4F84033FFF742FBDAE4012A11D194F8E8
:10A7B8001924002A3FF4D4AC0D4A94F8181492F8DE
:10A7C80068209142E5D29F0703D594F84434002BC2
:10A7D800DFD194F8913400206FF3041384F8913496
:10A7E80084F81904FFF744FBBAE429B0BDE8F08FF8
:10A7F800A80E0020D81700202DE9F04F89468DB00B
:10A8080090460746002800F08F81002900F08C81CF
:10A818000368002B00F088814368002B00F08481D6
:10A828008368002B00F08081C368002B00F07C81D6
:10A83800104602F003F8002800F07881BD4CBE4DA8
:10A84800384601F0C1FA40F2C4520021204603F014
:10A858008BFF40F21C520021284603F085FFB74BBE
:10A86800C4F82C3104F50973089304F50A7300261B
:10A878004046099308A9B24B84F848800A9384F8A3
:10A88800186184F88C608DF82C6001F0E9FF0F23C3
:10A8980006A994F848008DF8183001F0D3FF801B02
:10A8A80018BF01204FF00A0B84F81C0106A994F880
:10A8B80048008DF818B001F0C5FF4FF0060A84F87B
:10A8C800DC0006A994F848008DF818A001F0BAFF3A
:10A8D800102384F8DD0006A994F848008DF8183094
:10A8E80001F0B0FF1123C4F89C0006A994F84800B1
:10A8F8008DF8183001F0A6FF1223C4F8A00006A9AD
:10A9080094F848008DF8183001F09CFF1323C4F820
:10A91800A40006A994F848008DF8183001F092FFB9
:10A928001423C4F8A80006A994F848008DF8183034
:10A9380001F088FF1623C4F8AC0006A994F8480073
:10A948008DF8183001F07EFF172384F8B10006A9AE
:10A9580094F848008DF8183001F074FF18230DEBB7
:10A968000301C4F8B400C4F8BC0094F848008DF89A
:10A97800183001F067FFC0B21D2384F8B80084F8CE
:10A98800C00006A994F848008DF8183001F05AFF65
:10A998001E2384F8C40006A994F848008DF81830DE
:10A9A80001F050FF1F2384F8C50006A994F8480059
:10A9B8008DF8183001F046FF2023C4F8C80006A916
:10A9C80094F848008DF8183001F03CFF0B23C4F8C8
:10A9D800CC0006A994F848008DF8183001F032FF31
:10A9E8000C2306A9A4F8D00094F848008DF8183074
:10A9F80001F028FFD4F89C306365D4F8A030A36533
:10AA0800D4F8A430E365D4F8A83023664FF00108E1
:10AA1800D4F8AC300590A4F8D200636684F8B0800E
:10AA2800C4F894B084F898A0C4F84CB084F850A046
:10AA380084F8688084F81F81C5F84893FEF77AFD8A
:10AA4800404B009632464FF0FF3105F55A70C5F875
:10AA58004473C4E90B6684F8198185F89164C5F8D4
:10AA6800408306F033F9384B009632464FF0FF31F9
:10AA780005F5607006F02AF9344B009632464FF01F
:10AA8800FF3105F5667006F021F902AF304B0096EC
:10AA980032464FF0FF3105F5806006F017F9384669
:10AAA80006F0A8F897E8030004F5927383E803001A
:10AAB800284B294F1E60294BC5F84C33284BC5F845
:10AAC8005433284BC5F85C33274BC5F85033274B14
:10AAD800C5F8583305F553703B68984704F5A670D8
:10AAE80003F084FB20B1112630460DB0BDE8F08F8D
:10AAF800204601F01DFB0028F5D101F041F8B8B956
:10AB08001B4801F067FB06460028ECD17B69984793
:10AB180003F0F4FDBB6D94F819019847FB6A984758
:10AB2800012385F89234DFE70326DDE70926DBE712
:10AB38001326D9E7A80E0020701400200004000195
:10AB48008C190020799E0008D996000821970008E2
:10AB5800018F00086C140020CC23010825910008FF
:10AB6800D9900008BD8E0008B190000889900008AF
:10AB7800900F002008B5034B0020C3F84003FEF7F0
:10AB880081F908BD7014002010B5FFF7A7F90A4C29
:10AB980060B90A4B93F81831022B02D1084BDB6AD3
:10ABA80098470123C4F84033002010BDD4F840036F
:10ABB800013818BF0120F8E770140020A80E002003
:10ABC800CC23010838B5134C04F55A7006F0DCF8AC
:10ABD80004F5607006F0D8F804F5667006F0D4F84D
:10ABE80004F5806006F0D0F800F0B5FF0A4B0025A8
:10ABF800DB6A9847C4F84053FEF7B6FD0749084892
:10AC080040F2C45203F09CFD0123C4F840332846A7
:10AC180038BD00BF70140020CC230108A80E002006
:10AC2800E408002070B52E4B8AB0054693F8DD0085
:10AC38008DF8090093F8DC008DF80A0029489A6A13
:10AC480090F81804039200268DF80B0004960C4621
:10AC5800002940D00692D3F8882007921A8F93F8DB
:10AC68001A118DF8151052BAADF8202093F87C20EF
:10AC780093F848308DF8243003AB8DF822008DF816
:10AC8800232000930DF10A020DF10B030DF10901C8
:10AC980005A88DF8146000F0DDFE9DF90900FEF7A7
:10ACA80013F9607004A801F02BF8B0B9049A0F2AC0
:10ACB8000DD863789A420AD81544AB42A3EB020137
:10ACC8002CBF002001202170C0000AB070BD0023F5
:10ACD80023700820F9E70320F7E71320F5E700BF02
:10ACE800A80E0020701400201FB50446002800F0AC
:10ACF80012810078412800F20881DFE810F0420054
:10AD080048004D00520056005A005F000601060137
:10AD180006010601060106010601060166006A0031
:10AD28006E0079008000830086008B0089008D000A
:10AD38009100940097009A009D00A000AF00B30016
:10AD4800BB00B700BF00C200C600CF00CB00CD00DB
:10AD58000601D300060106010601060106010601E7
:10AD680006010601060106010601060106010601A3
:10AD78000601DB00DF00E300E800EC00F000F4006F
:10AD8800FD00674B93F81831237104B010BD644B74
:10AD980093F83031237102E0606803F0B5FB0020BE
:10ADA800F3E7606803F0F6FBF9E75D4B93F81A31B7
:10ADB800F0E75B4BD3F8E0306360F0E7584B211DB8
:10ADC80093F8300103F0FEFBE9E7554B93F819318E
:10ADD800E0E7534B93F88C30DCE71C238DF8083000
:10ADE8004F4B02A993F8480001F02CFD6060D6E7AC
:10ADF8004C4B043493E8030084E80300CFE74A4B44
:10AE08000434F7E7494B0434F4E7494B0434F1E7D9
:10AE18001A23E3E71923E1E7414B93F86830B9E7D0
:10AE28003F4B5B6DC8E73E4B9B6DC5E73C4BDB6D0D
:10AE3800C2E73B4B1B6EBFE7394B5B6EBCE7022397
:10AE48008DF80830364B02A993F87C2093F8480017
:10AE58008DF80A2001F0F6FC2071A0E7304B93F83A
:10AE6800DD3097E72E4B93F8393093E72C4B93F866
:10AE7800DC308FE72A4B93F838308BE7284BDB6CB4
:10AE88009AE7274B93F8503084E7254BD3F8843062
:10AE9800636084E7224B8FE7264B8DE7204BD3F87E
:10AEA800CC30F5E71E4BD3F82C31636001F058FD28
:10AEB800A06074E71A4BD3F890307DE7184B93F8ED
:10AEC8001F3167E7164BB3F88830A38067E7144B48
:10AED800B3F88A30F9E7124BB3F8D030F5E7104BE6
:10AEE800B3F8D230F1E70E4B93F848200AB1062A9E
:10AEF80013D1B3F8A035E8E7094B93F848200AB115
:10AF0800062A0AD1D3F8A43556E7204604B0BDE88E
:10AF1800104000F024BE032037E7182035E700BFB3
:10AF2800A80E0020140F00205C0F00201C0F00202A
:10AF3800640F0020E40800207FB5044610B9032000
:10AF480004B070BDA44DD5F840339A0700F1718262
:10AF58000278412A00F26A82DFE812F042004800D3
:10AF680056005C00600065006A0077008200880077
:10AF78008E0094009A00A000A600AC00B6006802FB
:10AF8800BB00DD00F000170139012A0144014D0121
:10AF98005101550159015D016802610173019B016D
:10AFA8008901AD01B301BA01BF01C40168022A02D7
:10AFB8006802680268026802680268026802680239
:10AFC8006802680268026802680268026802680229
:10AFD80036023B02400245024A024F0254025E0218
:10AFE8000079FEF7C1F80028AAD105E00379022B01
:10AFF800A5D07A4A82F8303195F8913443F020038D
:10B0080085F8913400209BE7406803F06FFA002828
:10B01800F2D094E7406803F0ADFAF8E76F4B027995
:10B0280083F81A21E8E76D4B4268C3F8E020E3E7AC
:10B038006A4E416896F8300103F0BAFA00287FF4A6
:10B048007EAF6368C6F8E430D6E7416800293FF46C
:10B0580076AF002001F0EAF90028CDD011206FE783
:10B06800416800293FF46BAF0120F3E741680029EC
:10B078003FF465AF0820EDE7416800293FF45FAF72
:10B088000920E7E7416800293FF459AF0C20E1E7C0
:10B09800416800293FF453AF0D20DBE741680029E0
:10B0A8003FF44DAF0E20D5E7416800293FF447AF84
:10B0B8000F20CFE74A4C494B007983F81901A36D5B
:10B0C8009847E36A984797E7444B027983F88C20BE
:10B0D80092E7424E037A8DF8043096F8480096F8C5
:10B0E8007D308DF80530072201A901F0BEFB00284C
:10B0F8003FF425AF636896F848000193002201A940
:10B1080001F0B3FB00283FF41AAF6C36D4E9010113
:10B1180086E8030070E7314E037A8DF8043096F81C
:10B12800480096F87D308DF80530072201A901F016
:10B138009CFB00283FF403AFB436E7E7274E037AB9
:10B148008DF8043096F8480096F87D308DF8053073
:10B15800072201A901F089FB00283FF4F0AED4E9E9
:10B16800010106F1740383E8030096F81831022BF5
:10B178007FF442AF96F83031002B3FF43DAF184BC7
:10B18800DB6A9847FDF748FF36E7144E037A8DF8D7
:10B19800043096F8480096F87D308DF8053007227F
:10B1A80001A901F062FB00283FF4C9AEBC36ADE747
:10B1B8004368029301238DF80C30084B02A993F8D9
:10B1C800480001F05FFB00287FF416AFB7E643683C
:10B1D80002930023EFE700BF70140020A80E0020A0
:10B1E800CC23010803795A1E0E2A3FF6A8AE934ACB
:10B1F80082F8683000E7914B42685A65FCE68F4B4D
:10B2080042689A65F8E68D4B4268DA65F4E68B4B3E
:10B2180042681A66F0E6894B42685A66ECE6874C43
:10B22800037994F848008DF80430062201A901F04A
:10B238001CFB00283FF483AE9DF8043084F8DD3011
:10B24800DAE67E4C03798DF8043094F8480094F8D7
:10B258007C308DF80630052201A901F006FB002894
:10B268003FF46DAE9DF8043084F83930C4E6734C71
:10B27800037994F848008DF804300A2201A901F0F6
:10B28800F4FA00283FF45BAE9DF8043084F8DC3013
:10B29800B2E66A4C037994F848008DF80430092224
:10B2A80001A901F0E2FA00283FF449AE9DF8043004
:10B2B80084F83830A0E6614B4268C3F89420DA6419
:10B2C8009AE65E4B027983F8982083F8502093E63B
:10B2D8005A4B4268C3F884208EE6584B4268C3F83C
:10B2E800CC2089E6012B40F0A480554C242120462F
:10B2F80003F03CFA636A984201D0172020E61C212B
:10B3080004F1280003F032FA636C9842F5D14FF447
:10B31800807104F1480003F029FAD4F848319842C2
:10B32800EBD1D42104F5A67003F020FAD4F820322A
:10B338009842E2D1002104F5097003F017FAD4F815
:10B3480024329842D9D14FF4607104F50A7003F0A1
:10B358000DFAD4F8A8359842CFD1142104F2AC5094
:10B3680003F004FAD4F8C0359842C6D1334E2146CA
:10B37800304640F2C45203F0E3F9204640F2C4528A
:10B38800002103F0F1F995F81B3485F8E833736F61
:10B39800C5F8EC3396F87D3085F8F83340F2012390
:10B3A800A5F8FA33274B96F819019B6D984723E6C1
:10B3B8008379012B3FF6C3AD204B42684068C3F840
:10B3C8002C2100F0D1FE47E61C4B4268C3F89020C0
:10B3D80012E61A4B027983F81F210DE6174B828873
:10B3E800A3F8882008E6154B8288A3F88A2003E68C
:10B3F800124B8288A3F8D020FEE5104B8288A3F870
:10B40800D220F9E50D4B93F848200AB1062A12D14B
:10B41800A288A3F8A025EFE5084B93F848200AB1C5
:10B42800062A08D16268C3F8A425E5E500F099FB6F
:10B43800D9E5012084E5182082E500BFA80E002088
:10B44800E4080020CC2301082DE9F04387B000234D
:10B45800ADF800300646002800F0ED800361FEF7E5
:10B468003DFD20B10124204607B0BDE8F08300F07F
:10B4780073FD0028F6D100F069FD014618B96F4840
:10B48800142203F071F96E4D95F89134012243F0BE
:10B49800040385F8552485F8913433788DF8043001
:10B4A8000021013B8DF80520ADF806100C2B00F2A9
:10B4B800BA80DFE803F007B8B8B87881B8B88FB8B1
:10B4C800AC99A800D5F8407317F02007CAD196F8B0
:10B4D8000480B8F1020F45D1DFF868815A4CFEF7B5
:10B4E80029F896F9051098F848003A4601F017FA35
:10B4F80088F83900B37988F83830384607238DF84A
:10B508000530FDF731FEFF2304F58670A5F80C31F0
:10B51800C5F8084185F8047103F03CF804F58A7011
:10B5280002F0F2FF3846FDF78DFE044640B196F969
:10B53800051098F84800012201F0F1F988F839005F
:10B54800D5F894343361002C71D000F0FFFC00284A
:10B5580089D195F8913485F81A0460F3820385F847
:10B56800913480E7B8F1010F4FF00204E8D1DFF819
:10B57800D4908DF8144099F8480089F81D7102A9F3
:10B5880001F06EF9337989F830318DF805708DF84E
:10B598000680FDF785FC95F8913443F0100385F893
:10B5A80091340024CCE700226946022000F0F6FA24
:10B5B8000028F6D01324C3E7244BB288DB6B96F936
:10B5C8000C10B0689847D5F8403343F00203C5F82B
:10B5D8004033E6E702A90D2000F060FB0028E0D028
:10B5E800002269460D20E1E7164B93F81831D3B9CC
:10B5F800347904F0070000F0ADFA8DF8004001221C
:10B6080069461020D2E7002269461220CEE78DF85D
:10B61800072000F090FA044638B900F089FA20466D
:10B6280000F08BFA8CE702248AE7012488E701A856
:10B6380000F0DEFB17E7032415E700BFC41800205D
:10B6480070140020A80E002072140020CC230108DA
:10B658002DE9F04F99B08046059118B9032019B02B
:10B66800BDE8F08F00230361FEF738FC064600288A
:10B6780040F0AB8045460FCD0EAC0FC45A4C98F83D
:10B6880000A0B8F80C7098F90EB0142204F5886080
:10B69800314603F069F8012284F84124534C94F8A8
:10B6A8003021022A35460BD194F81821022A07D1F5
:10B6B80094F81E2122B9BAF1010F38BF4FF0010AE0
:10B6C800BAF1010F2DD0BAF1030F2CD0BAF1000F47
:10B6D80035D102229DF83C30DDF84090029362F3A8
:10B6E8004715012694F87C108DF8321002220CA917
:10B6F80094F848008DF8302001F0A4F894F81A3135
:10B7080094F830C194F81D1140B20222002B6FD07A
:10B71800BCF1010F65D1002963D1002E6DD110460F
:10B7280027E00422D6E70023DDF83C90BDF84070FE
:10B738009DF942B0029365F01F050126D2E74FF04C
:10B74800000BD946CDF808B0CCE74FF0010084F8DB
:10B758001A04DDE005F29A420BA900F0DDFA002890
:10B7680000F020811320049B33871F4B002283F8AD
:10B778001A241D4BD3F89434C8F810306FE705F23B
:10B788009A452A460BA900F0C7FA0028EAD10B9B74
:10B7980084F82801C4F82C5184F8303102E1B9F159
:10B7A800000F00F0FF80002A00F0FC804946E01CF2
:10B7B80002F0C6FF94F8373201332380F2E01220FA
:10B7C800D1E70220CFE70720CFE7012047E7064B64
:10B7D80093F8912483F840A442F0010283F891245D
:10B7E800C7E7EEB90220C4E770140020A80E0020B5
:10B7F800002E94D05845B8BF584694F87C308DF840
:10B808002000052294F848008DF8223008A901F09C
:10B818002CF800283FF422AF9DF8203084F8393006
:10B82800694A6A4BD2F89804D3F8904038B105F0C9
:10B8380071FA664B84423CBF002283F83A20198F84
:10B848001A8F93F830010491996A099152BA002825
:10B85800B9D093F81B0100B9186393F81801ADF833
:10B868005820013893F87C2093F81A411491D0F1AC
:10B87800000BD3F888108DF85B204BEB000B93F886
:10B88800482093F83A0093F868308DF85A3009AB9D
:10B8980000934F4B03904FF001008DF84C00159129
:10B8A8008DF85C20A3F12F01A3F1300213A88DF8C5
:10B8B8004D4000F0CFF8039B4FEA0B1B4BEA431BAC
:10B8C80000264BEA801B4BEAC413B1453E4C039358
:10B8D80008BF37463A46494604F59C70CDE90A66E2
:10B8E8009B46268084F81A6402F02AFFE9B2A57004
:10B8F800C5F34215FAB2042D344E039B84F837225F
:10B908003FF423AF072D3FF44AAF022D7FF459AF20
:10B91800304D84F80D110420029984F80401FF20A9
:10B9280084F80C0184F8281184F81431D6F8E4104E
:10B93800C4F8085105F59B730AA8C4F8101184F8D7
:10B948003021C4F82C3100F017FC00287FF437AF01
:10B958000A9BA4F844040BA8A4F81631C4F84C3484
:10B9680000F0CEF900287FF4FDAE0B9BD3B196F919
:10B978003900FDF7A9FA94F83732002B3FF4FFAEEF
:10B988000B9B0F2B3FF6E6AE05F58B720BA90F202C
:10B9980000F0C2F900287FF4E5AE0B9B63F3030BBC
:10B9A80084F814B10598FDF74DFC00287FF4DBAE50
:10B9B800099B86F83A00B36200F07EF900283FF44C
:10B9C80006AF1320D1E600BF70140020A80E002097
:10B9D800100F00207214002037B50B4D8DF80400AD
:10B9E80004460F2295F8480001A900F03EFF40B137
:10B9F800064A85F81C4192F8913443F0200382F8F6
:10BA0800913403B030BD00BFA80E00207014002090
:10BA180010B5FFF7B9F8044688B90A4805F0B4F933
:10BA2800094805F0B1F9094805F0AEF900F093F8B6
:10BA3800FDF780FD064BDB6A9847204610BD0124C0
:10BA4800FBE700BFD8170020F017002008180020D7
:10BA5800CC2301082DE9F04F8BB047780093149B55
:10BA680090F90C8090F90D6090F80E908B46416823
:10BA7800196004469246002F57D002238DF81030E3
:10BA880004A9C37B007C8DF8123000F0DBFEB4F80B
:10BA980008C0618943B26068984545466144B8BFAB
:10BAA8001D46604534BF00270127884209D30A2173
:10BAB8008DF81010207C019304A900F0C3FE019BAF
:10BAC80046B2B4F808C0608961680CEB400E714555
:10BAD80020D3A1EB0C01B1FBF0FC00FB1C11C9B990
:10BAE80098450ADC237833B10223207C8DF8243072
:10BAF80006A900F0B5FE4FF0010921238DF810309A
:10BB0800207CE37B8DF8115004A98DF8123000F0E9
:10BB180099FE45B2009B8BF8005038468AF80060C1
:10BB280083F800900BB0BDE8F08F4546F2E7704708
:10BB380070477047704700207047704770477047DC
:10BB48000020704700207047002070470020704791
:10BB580000207047704770477047022070470220E6
:10BB68007047022070477047002070477047704741
:10BB780000207047002070477047704770470000EA
:10BB880010B5054C4FF403722046002102F0ECFD7D
:10BB98000020C4E9000010BD301A00202DE9F84348
:10BBA8008146174600293FD0244B002503F1010C9C
:10BBB8001A462801103312F8018FB8F1000F36D158
:10BBC8009A42F8D11E4E33680BB9C6F800C07368A4
:10BBD8000BB1C3F800C03318002401359C6083F80A
:10BBE8000C900D302B01BAB206EB05153044F75016
:10BBF800C6F804C002F0A4FDB9F1110F4FF000031C
:10BC080098BF104C6B71D6F8083298BF24FA09F423
:10BC180003F1010398BF04F001043B442C71C6F8FA
:10BC280008324046BDE8F8834FF00108F9E70135CE
:10BC3800202DBBD14FF00208F3E700BF371A0020D0
:10BC4800301A00202007020010B510B3124A1368FA
:10BC5800984204D103681360002304E00B4613B133
:10BC680019688842FAD15168884208BF53600BB1FD
:10BC780001681960D2F808328168013B00245B1A18
:10BC880004602146C2F80832102202F06DFD2046F9
:10BC980010BD0120FCE700BF301A0020054B1B68CF
:10BCA80013B11A798242FAD1002B0B600CBF032022
:10BCB80000207047301A002010B5054B186800B9ED
:10BCC80010BD037B04680BB9FFF7BEFF2046F6E7FB
:10BCD800301A002038B5084B084C186800B938BD30
:10BCE80003790568112B05D824FA03F3DB0701D57E
:10BCF800FFF7AAFF2846F1E7301A002020070200C4
:10BD080028B1044BD3F808320360002070470120A3
:10BD1800704700BF301A00202DE9F04107460E4653
:10BD280015463AB331B3144B1C6800232CB930467E
:10BD3800FFF7E6FF0020BDE8F081A268F91A01329A
:10BD4800914210D32279EA54581C22895FFA80F86C
:10BD5800611D55FA80F002F0F3FCA368246898444A
:10BD68005FFA88F3E2E720462468FFF76DFF002CAE
:10BD7800F9D1DCE70120DEE7301A00200238C0B232
:10BD880011289ABF014B185C00207047DF1C01087E
:10BD980030B50B4B93F820200446084672B10021B9
:10BDA8001C330578A54208D001319842CDB20CBFAA
:10BDB80004480430AA42F4D8002030BD1046FCE7FD
:10BDC8003C1C0020481C002010B5084C00232060B3
:10BDD800142204F10C00FF2184F82030C4E901008A
:10BDE80002F0C2FC012384F8213010BD3C1C002065
:10BDF80010B50E4A92F82010042915D893680478D3
:10BE08001C7044785C70C478807898700131DC705C
:10BE180082F8201002F11C018B4214BF043302F196
:10BE28000C039360012010BD0020FCE73C1C00209F
:10BE3800094B93F8200068B15A6803F11C018A4243
:10BE480000F1FF3014BF043203F10C0283F8200024
:10BE58005A600120704700BF3C1C002010B5074BFA
:10BE680093F820200446084632B15968FFF790FF3E
:10BE780010B101234470837010BD00BF3C1C00202A
:10BE880008B5064B93F820202AB15968FFF780FFC0
:10BE980008B1407808BD0120FCE700BF3C1C002029
:10BEA80030B50A4A92F82010536882F8210061B12F
:10BEB800916801241C32DD78587005B99C70934252
:10BEC8000CBF034B04339942F5D130BD3C1C002014
:10BED800481C002008B5044B5968FFF759FF003883
:10BEE80018BF012008BD00BF3C1C00202DE9F3410C
:10BEF8000422154E044600210DEB020096F820801E
:10BF080002F032FC0025EBB2984502D802B0BDE839
:10BF1800F0817368197821705A7862709F785FB1E0
:10BF2800336820469B689847FFF782FF17B901A836
:10BF3800FFF75EFF0135E6E7DB788DF804108DF832
:10BF480005208DF80730EFE73C1C0020014B93F8E3
:10BF5800200070473C1C0020034B93F82000042865
:10BF680094BF0020012070473C1C00201FB500240E
:10BF7800CDE90244C41F8DF800408DF801100C0A69
:10BF8800ADF80420090C120C8DF803108DF806206A
:10BF98008DF8073002461B0A012168468DF80240D9
:10BFA8008DF8083002F04BFA002818BF0E2004B0B4
:10BFB80010BD2DE9F04188B017460D460F9A064688
:10BFC80000284DD000240121CDE904448DF810103B
:10BFD8009DF838108DF81510ADF81630190CCDE90C
:10BFE80000441B0ECDE902448DF81930ADF81A2033
:10BFF800130C120E07948DF818108DF81C308DF85C
:10C008001D20E3B24FEA0318002D5FFA88F803DC1D
:10C01800002008B0BDE8F081013310218DF81F30F1
:10C028003A466B460DEB010002F09FF90346C8B98A
:10C03800102DAC46A8BF4FF0100CDAB2624503F1E0
:10C04800010303DB103D2DB20134DAE708EB0200EF
:10C0580020326A44315C12F8202C4A403254ECE712
:10C068000920D6E70E20D4E70138032815D8DFE8E1
:10C0780000F002080C100A4B1B681B690B600020BB
:10C088007047074B1B685B69F8E7054B1B689B69A2
:10C09800F4E7034B1B68DB69F0E70520704700BF36
:10C0A800601C00202DE9F041C4B00C464A9E17469A
:10C0B8001D468046B8B3B1F5807F36D84FF48872F4
:10C0C8000021684602F050FB492300934FF4807327
:10C0D800ADF804302B0C8DF80830330CADF8065051
:10C0E800ADF80A608DF80C3022460023414604A8BA
:10C0F8002D0E360E8DF80E308DF809508DF80D6026
:10C108008DF80F4002F01CFB04F110014B9A3B46DE
:10C1180089B2684602F013F910B1012818BF0E2041
:10C1280044B0BDE8F0810920FAE70D20F8E70000E7
:10C1380010B590B10A4C28220021206002F014FBAF
:10C148002368084A1A6000204FF0FF32C3E903024F
:10C15800C3E90522C3E9072210BD0820FCE700BF98
:10C16800601C002000010101024B1B6818600020C0
:10C17800704700BF601C002030B1044B1B68DB68AF
:10C18800013303600020704709207047601C0020BD
:10C1980013B500230C460193D2B101A9FFF764FF40
:10C1A80018B9019B591C02D1146002B010BD99B294
:10C1B800611A002902DD0B441360F6E702D113600F
:10C1C8000720F2E71B0C1B0403F580332344F3E735
:10C1D8000920EAE728B1044B1B681C33436200209E
:10C1E80070470920704700BF601C002013B5044643
:10C1F800D8B1114B1A68938801339BB29380C382DC
:10C2080000F057FA98B904F1180300932168012344
:10C21800132202F08BF860B9204600F04AFA003881
:10C2280018BF0120000102B010BD0920FBE7102053
:10C23800F9E70E20F7E700BF601C0020F0B50546BF
:10C2480087B01C463BB32F4E3368DB68834257D810
:10C2580094F82020002A14BF09220822834205D31B
:10C26800204600F05AFA70B110200AE0002301902D
:10C278000093A36894F82810606AFFF79AFE0028D4
:10C28800EED007B0F0BD23792168B4F808C0A768DC
:10C29800043B9AB209B90920F3E7B2F5807F2DD89B
:10C2A800ADF80EC08DF817304FEA174C04F12C0387
:10C2B8003F0E8DF8117000932F0C08234FF0490E94
:10C2C800ADF80C008DF814708DF816002F0E0DEBDC
:10C2D8000300CDF808E08DF810C0ADF812508DF8C5
:10C2E800157002F023F808B10E20CAE7204600F0C6
:10C2F80014FA0028B8D13368DD60C2E70D20C0E722
:10C308000620BEE7601C00202DE9FF410A9D8046FB
:10C318000F4616461C46002D5AD0002303A9104686
:10C328000393FFF7A1FE18B1062004B0BDE8F08121
:10C33800039B9C4201D80133F6D1284600F05EF9F0
:10C34800002847D1264B1A78424503D01A7942452E
:10C3580042D10120AA68BA4240D103EB8002EB6ABD
:10C3680092F801802979CDE9004304399278286848
:10C378003B4689B2FFF796FE0028D6D195F82030C3
:10C388000194002B4FF00103009314BF424608228A
:10C3980095F82810686A3B46FFF70BFE0028C4D1C1
:10C3A800013E032EC1D8DFE806F002070B0F0D4B44
:10C3B8001B681C611C62B8E70A4B1B685C61F9E7E3
:10C3C800084B1B689C61F5E7064B1B68DC61ACE712
:10C3D8000920AAE70F20A8E70B20A6E70220A4E778
:10C3E80034010020601C00201FB50A460B2A4FF0BC
:10C3F8000001CDE90011CDE9021107D00C2A13D0B4
:10C408000A2A0FD00A2005B05DF804FB012802D1E2
:10C4180020238DF80030684602F011F8002818BF74
:10C428000E20F0E73023F4E70B21F4E738B5054692
:10C4380002F000F8044678B97DB9094B1B680B2156
:10C448009878FFF7D1FF38B90C21FFF7CDFF18B95D
:10C458000A21FFF7C9FF00B10E24204638BD00BFEE
:10C46800601C00202DE9F04380468FB00C4617462B
:10C47800002A6BD0002969D0002529461D2206A86C
:10C48800059504F093FE8DF81350344D2B680DF18B
:10C4980014099E88CDF804900DF1130302933B799B
:10C4A80000933B6832462146404601F0E4FF0028ED
:10C4B8004ED138683A79494602F042F9384600F0D8
:10C4C8004FF8002846D13C7AFA79BB79240444EA2B
:10C4D80002241C432B689A6894423DD99C609DF8BD
:10C4E80013000B21FFF780FF034658BB0C21FFF711
:10C4F8007BFF034630BB0A21FFF776FF034608BBE4
:10C508007B7ABA7AFF7A3F0447EA02271F433A4602
:10C51800334621460920FFF729FD034690B93346E3
:10C528003A4621460820FFF721FD034650B92A68FC
:10C538009DF8131091700021D1604FF0FF31C2E9CE
:10C548000411916118460FB0BDE8F0830923F9E79B
:10C558000E23F7E70F23F5E70323F3E7601C00201A
:10C5680010B50446002845D00168002942D011F8CA
:10C57800013B43710322063002F0E2F82046032211
:10C5880050F8091B043102F0DBF82168CB79E3602D
:10C598000A7A43EA0223E3604A7A43EA0243E36001
:10C5A8008A7A43EA0263E360CB7A23740B7B637471
:10C5B8002379212B1AD110220D3104F1120002F037
:10C5C800BFF81D222168501C8B5C6362085C43EA3B
:10C5D8000023901C6362085C033243EA00436362F1
:10C5E8008A5C43EA02636362002010BD112B03DCFE
:10C5F8000D22E7E70220F8E70120F6E710B5044628
:10C60800002854D00168002951D00B7843714B7829
:10C6180083608A7843EA02238360CA7843EA024344
:10C6280083600A7943EA026383604B7903738B79E9
:10C63800C381CA7943EA0223027BC38102F00F0255
:10C648000831103002F07CF8237B002203F00F033E
:10C6580084F8202084F82820227903F10800111A90
:10C6680004290DDD21680933043AD21A085C84F8DC
:10C678002000D2B2606A84F82820194402F060F8D9
:10C68800237922681A44002012F8043CE36212F865
:10C69800031C43EA0123E36212F8021C43EA014344
:10C6A800E36212F8012C43EA0263E36210BD022040
:10C6B800FCE710B5044660B3036853B30279162A41
:10C6C80029D942791A700146082251F8060B01301F
:10C6D80002F040F82146082251F80E0B093002F00A
:10C6E80039F82368E28A5A74E38A22681B0A937429
:10C6F8002368A269DA74A36922681B0A1375236880
:10C70800628B5A752368E27E9A751723237100207D
:10C7180010BD0120FCE70220FAE738B504460028DE
:10C7280063D00168002960D0037B90F8282003F0CB
:10C738000F03002A57D10833207904321344984252
:10C7480055D363790B702368A2685A70A36822686E
:10C758001B0A937023686289DA702368E27A1A7177
:10C768002368227B5A712368E2899A71E3892268D7
:10C778001B0A2146D371227B51F8100B02F00F02DD
:10C78800083001F0DDFF237B94F8282003F00F0325
:10C7980003F108052AB1226894F82010515503F1D5
:10C7A8000905206894F82820616A284401F0C8FF28
:10C7B80094F828302268E16A2B44D1545A1CE16A63
:10C7C800206892B2090A81549A1C2168E08D92B2BD
:10C7D8008854DA1C216894F82F0092B204338854E4
:10C7E8002371002038BD0933A6E70120FAE70220AB
:10C7F800F8E70000024B1A8810431880704700BF02
:10C80800641C002008B5074B1B883BB1FEF7BCF938
:10C8180000280CBF00206FF0020008BD6FF0010077
:10C82800FBE700BF641C002010B5034B00241C80EC
:10C83800FEF7A0F9204610BD641C0020B0FA80F075
:10C848004009704782B018B9084602B000F0CAB86B
:10C85800002002B0704710B9084600F077B9704759
:10C8680010B9084600F08EB97047034608461146CD
:10C878000BB900F0E5B90020704710B9084600F080
:10C8880071BD704710B9084600F006BA002070471D
:10C8980010B40446084611461A46019B14B910BC48
:10C8A80000F018BA10BC70470346084611460BB989
:10C8B80000F042BA0020704710B4044608461146FA
:10C8C8001A4614B910BC00F0AFBA002010BC70476B
:10C8D80030B40546084611461A46DDE902341DB94A
:10C8E800029430BC00F02EBB002030BC704710B959
:10C8F800084600F0DFBB0020704710B9084600F07A
:10C908006FBD0020704710B9084600F0EEBB00204C
:10C91800704710B9084600F0EBBB0020704703468B
:10C92800084611460BB900F005BC0020704710B44A
:10C938000446084611461A46019B14B910BC00F07B
:10C94800FBBB092010BC704710B4044608461146CA
:10C958001A4614B910BC00F063BDC8B210BC7047C9
:10C968000048704701000102064B10B51B6A0446D7
:10C97800984730B10448054B204498428CBF0020AA
:10C98800012010BDCC23010840C220C980B92A006B
:10C99800F0B5114B85B00C4610491F56054601F0FD
:10C9A80049F80F4BE4B25E6A072D4FF00103CDE959
:10C9B800024301460AD105220023CDE900234FF4A2
:10C9C8007A727A431846B04705B0F0BD08220020B5
:10C9D800CDE900203A46F5E71B1D0108F41C0108C3
:10C9E800CC2301081FB5002300930378013B372BA4
:10C9F80021D8DFE803F01C242020201E202020203E
:10CA08004143454E2055585B5E6164206C1E6E7331
:10CA1800787A20207D812620202020202020202098
:10CA28002020202083858A2020838A208C90C37828
:10CA38000BB102230093009805B05DF804FB8378DE
:10CA4800F6E743788DF8043005238DF805308378B0
:10CA5800003B18BF01235B008DF8063010238DF8CA
:10CA68000730304B1B6801A803F55872CDE9022343
:10CA780000F0C0FF0090DEE74023DBE72023D9E782
:10CA8800827890F9013012B9274AD35CD2E7274A55
:10CA9800FBE7827890F90130002AF8D1244AF4E7BC
:10CAA80040F6B833C6E74FF47A73C3E74FF4FA6336
:10CAB800C0E741F28833BDE741F27073BAE71D4819
:10CAC8004FF47A7101F020FE00F5FA60D2E71A4BB4
:10CAD800B0E7144B1B6803F55873ABE7114B1B68A1
:10CAE80003F55B73A6E71023A4E70E4B1B68A1E7C9
:10CAF8004FF0834300939EE7104BFBE7104B99E7F9
:10CB080040F21113ADF8003095E7032392E790F94E
:10CB180001300C4AB9E70C4990F9010000F08AFF8E
:10CB2800A8E700BF6C1C0020A31D0108AB1D01086D
:10CB3800B31D010818FCFFFF00EA06379A9909405F
:10CB480040F709371B1D0108F41C010837B50B4BCA
:10CB580002781B680C2101FB02335B7A03EB430468
:10CB6800074B1D6803690093C3684278816805EB29
:10CB7800C40000F0DFFC03B030BD00BF6C1C002017
:10CB8800681C002070B586B0027B6423ADF80030C5
:10CB9800012A4FF00003CDE90133CDE903338DF8C5
:10CBA80002308DF8143030D0022A39D05ABB0368CD
:10CBB8004BB343683BB31F4D80682B601E4B182254
:10CBC8006946186001F0BCFD1C4B2C6893E807000F
:10CBD8000C3384E8070093E8070004F10C060323EC
:10CBE80086E80700A4F86C33012204F55B7104F5AC
:10CBF800587000F090FC2B684FF6B072A3F87823B9
:10CC08000522C3F87C2306B070BD0A490868436052
:10CC1800036100F55B7100F5587000F07CFCF2E7E9
:10CC2800044B1B68B3F86023B3F86C130A43A3F8EA
:10CC38006023E8E76C1C0020681C002090130108A2
:10CC480008B503460A2924D8DFE801F00623232380
:10CC5800230B161B23212100BDE808400068FFF7BD
:10CC680083BE90F900009978052271B900F013FC91
:10CC7800003818BF012008BD052293F900000021E3
:10CC8800F4E790F900005978EEE70221EEE7072271
:10CC9800F3E70020EFE7000010B504791CB1012C80
:10CCA8000BD0002010BD0A4B01681B68012203F558
:10CCB800587000F030FC0120F4E7054B01681B6850
:10CCC800224603F55B7000F026FC2046EAE700BF29
:10CCD8006C1C0020F7B50528144D1C46A8BF05207C
:10CCE80058700E462946174600F0A4FE94F9013004
:10CCF800A070072B13D1322000F09CFD0C4BDB6D8C
:10CD08000546984704F10C02083403460192009442
:10CD18003A463146284600F092FD03B0F0BD054A78
:10CD280055F82310D05C00F07DFDE7E7F41C0108FE
:10CD3800CC2301081B1D01082DE9F04F344F90F951
:10CD480001607B68D0F804908BB004468846984709
:10CD58000546002859D1E37C73B92E4A2378126816
:10CD680003EB4303990002EB8303D3F80490B9F172
:10CD7800000F01D152F80190274B484613F906B02D
:10CD8800FB689847A37CD7F818A022890993072E37
:10CD980028D100230121CDE90223204A0693CDE9B9
:10CDA8000431CDE907330521CDE900214FF47A722A
:10CDB80002FB0BF24CF250311846D047637C13B398
:10CDC800174B995D7B6D0D31C9B228469847E07CB9
:10CDD8003246494600F040FE88F8006001200BB05A
:10CDE800BDE8F08F002101250823CDE90013CDE926
:10CDF8000715CDE90511CDE903110292A1782B465B
:10CE08005A462846D9E7074BDBE70020E7E700BF8B
:10CE1800CC2301086C1C00201B1D0108854501005E
:10CE2800B31D0108A31D01082DE9F04F8DB090F93D
:10CE38000130DFF8FCA0DFF8FC90CDE90A123E4A89
:10CE480012F903B00278DAF800300C2505FB02333A
:10CE58003A4A5B7A126803EB430302EBC3030446C6
:10CE680093F9021090F9020000F0DFFD34490646FC
:10CE780094F9010000F0DEFDA26861688046304642
:10CE880000F005FD2178DAF80020D9F80C30694364
:10CE9800074650589847D9F81C309C4694F90130F9
:10CEA8000025072B4FF47A63CDE90753CDE90555E3
:10CEB8002DD10123CDE903530523CDE901534FF4C7
:10CEC8007A7303FB0BF300933946434646F2A812E4
:10CED80028466746B8472378DAF800200C214B43E8
:10CEE80094F90110D05800F0D9FDA18994F90100F6
:10CEF800FFF74EFD0B9B217B1860D9F8543028466C
:10CF080098470A9B01201E700DB0BDE8F08F0120E4
:10CF18000823CDE90350CDE901032A46CDF800B036
:10CF2800654643463946A84701200546D3E700BF72
:10CF38006C1C0020CC2301081B1D0108681C002064
:10CF4800F41C01082DE9F04F8FB0002405468A46ED
:10CF5800914698460494ADF81440ADF8024007266F
:10CF68004FF0010B2B7AA34206D9686804A9204424
:10CF780000F0F2FB00285ED102238DF8083002A8E9
:10CF88006B7A8DF80A30FFF72DFDAB7A8DF81D30DE
:10CF98009DF811308DF81E309DF812308DF81F3035
:10CFA8009DF810308DF82030EB7A8DF821302B7BEE
:10CFB8008DF822306B7B8DF8233010238DF81C60A0
:10CFC8008DF824303A4E8DF82C000DF102030A93A7
:10CFD80005238DF82D3033680C930723ADF83430D2
:10CFE8002B6806930DF1120204AB0DF1110106A88E
:10CFF80000F0CCFB072805460BD130680C22002135
:10D0080000F5587001F0B0FB3368BDF80220A3F8B2
:10D0180060239DF811308AF800309DF8123089F8A5
:10D0280000309DF8103088F80030189B28461C7096
:10D038000FB0BDE8F08F9DF81330BDF81470ADF84F
:10D0480002702044C4B2F3B917B3194A002011681A
:10D05800072602464FF00C0C062B1BD10CFB00FEDA
:10D0680051F80EE0BEF1000F04D00BFA00F23A437B
:10D0780097B2012201301028EED1002A3FF472AF96
:10D08800ADF802706EE75A1E042A01D9062BDCD0CF
:10D09800062667E747FA00FE1EF0010FEAD00CFBF0
:10D0A80000FE51F80EE0BEF1000F08BF0626E1E7CA
:10D0B8006C1C002038B505464068FFF755FC052272
:10D0C800841D002195F90000E4B200F0E4F908B9E4
:10D0D80004F0FD0495F901000722002100F0DBF9B6
:10D0E80008B904F0FB04204638BD00207047000052
:10D0F80010B503780F2B044618D84068FFF734FCA6
:10D1080022780B4902EB42020968831C01EB82007A
:10D1180051F82220DBB21AB903F0FD0358B210BD52
:10D12800032B06BF626842600223F7E70020F6E798
:10D138006C1C0020022070472DE9F04FDFF8388181
:10D148000446D8F8000099B08946174600211E46C3
:10D158000122032300F55870CDE90611CDE9081125
:10D168008DF814108DF81510ADF8163000F0B5F9DB
:10D1780038B9D8F80020B2F8603343F00303A2F8B6
:10D188006033D8F80020637A8DF8283002F558719A
:10D19800CDE90B12394A94F9083012680D920DF155
:10D1A80016020F922268109262681192D4E9030164
:10D1B800A27A8DF8482001228DF8492013AA82E826
:10D1C80003001025227DE18A8DF8293018468DF854
:10D1D8005420ADF83850FFF7DBFB0AAB17930DF17D
:10D1E8001503169000933146019705AB06AA10A8BF
:10D1F80000F0BCFB064698BB9DF81410204F01397F
:10D2080001F082FA1F4B1B690393C4B24FF00C0B59
:10D2180004F160036B44D8F8000013F848AC9DF89B
:10D2280014300BFB0AFC01343946B4FBF3F203FB60
:10D238001244D0F87C33B0F9782350F80C00DDF8AC
:10D248000CC0E4B2E04728B189F800A0304619B014
:10D25800BDE8F08F013D15F0FF05D9D10D26F5E7A2
:10D268000C2801BFD8F80020B2F8603343F003035C
:10D27800A2F86033EAE700BF6C1C0020681C00209D
:10D28800400D0300CC230108F8B50679012E0546A8
:10D2980001D80620F8BD0F2E2BD80368187A40F362
:10D2A80003000522002140B200F0F5F82B6804467F
:10D2B800187A40F303100522002140B200F0EBF881
:10D2C800A8B1B4FA84F4640929680B7A086843F3AE
:10D2D800030243F3031352B25BB29A42C8BF01245C
:10D2E800FFF742FB48B9002CD3D10420D2E7012430
:10D2F800EAE70320CEE70520CCE7002CFBD10C4F52
:10D3080029683B6806EB460003EB80000C2201F01D
:10D3180017FA3A680C2303FB062320465C72B2F81E
:10D3280060130123B3400B43A2F86033B2E700BF98
:10D338006C1C002010B4017801290ED9084B18681C
:10D348000C234B43C4180022C250C4E9012200F543
:10D35800587010BC102200F0A7B8002010BC70470D
:10D368006C1C00202DE9F04186B050238DF8143054
:10D37800037A102B074630D14368DD7B6DBB02244E
:10D38800A8466426062C14D87A68535D03932A4469
:10D39800517843EA01230393927843EA02437343A3
:10D3A800CDE9033863B968468DF80040FFF7C2FF3E
:10D3B8000DE0CDF80C808DF81480CDF81080F2E7E0
:10D3C80003AB01A801938DF80840FFF75DFF013416
:10D3D800E4B2102C05F10305D4D106B0BDE8F08104
:10D3E8001FB502680379116851B901A88DF8043096
:10D3F800FFF7A0FF78B9002040B205B05DF804FB44
:10D4080002A802928DF80C30FFF73EFF0628F2D8EA
:10D41800024B185CF0E70320EEE700BF141D01087B
:10D42800C90020B9034B0B449856C0B27047024B51
:10D43800F9E700BF231D0108631D0108F0B59A42F2
:10D44800069D03DB9DF914309A4220DD0020F0BDD3
:10D4580003EB430331F814C005EB830300264CFAB1
:10D4680006F7FF0707D51F7A07F00F0E724502DB94
:10D47800B2EB171F0DDD0136102E03F10C03EED1B0
:10D488000134E4B22301DBB29842E1D8DEE700249C
:10D49800F8E70120DBE7884204DB9042CCBF00209C
:10D4A800012070470020704710B51409B4EB111F14
:10D4B80003464FEA11100ED391420CD202B201F08A
:10D4C8000F0133F81240012000FA01F124EA0101AA
:10D4D80023F8121010BD0020FCE7F0B528B100EBCE
:10D4E800410501270020914200D3F0BD002435F802
:10D4F80002CB234607FA04F636EA0C0608BF0133C6
:10D5080004F1010408BFDBB2102CF3D11844013137
:10D51800C0B2C9B2E7E710B500B149B910BD31F8DA
:10D52800134020F813400133DCB2A242F7D8F5E7E4
:10D538000023F9E782B030B5048804936AB9B3F5DB
:10D54800616F18D349F6AF2542F21072AB4298BF0B
:10D558004FF47A72944238BF1446012C38BF012424
:10D568006143BDE83040C3688B428CBF5B1A00231F
:10D57800C36002B070476422ECE700002DE9F04F69
:10D5880091B01546DDF86C8004939DF868300993D6
:10D598000C46064603F0B4FB684ADFF8A4B10590D0
:10D5A800A8F5F633303BB3FBF2F3534303F5F632F9
:10D5B80003F5A83303F5C0730393182313FB05433E
:10D5C80030320692089300254FF0FF3A089BA34299
:10D5D80007D1002D14BF50464FF0FF3011B0BDE801
:10D5E800F08FBDF97030ADF82C300B99CDF86C8008
:10D5F8004046CDF8288003F013FBB4F800906EB9CC
:10D60800B8F5616F5BD349F6AF2242F210739045CB
:10D6180098BF4FF47A73994538BF99464B46012B0A
:10D6280038BF01230793002E52D1B9F1640F48D1B6
:10D63800A0605F46A1680EA803F014FB0F9B00933F
:10D64800DDE90A120E9B0CA803F06BFA049B0C9AF6
:10D658000BB9099B2BB12369BB4202D1394B9A42C2
:10D668000DD9394BE760984509D90023ADF8343016
:10D67800069B0D990C93184603F0D2FAA0606068D7
:10D6880000B9E760276126B103F044FBE36803446F
:10D69800E360D4E903329342059B1D996360079BBD
:10D6A80088BFE2604B43E168994202D20498A8B966
:10D6B800A6B101231D442375EDB2183486E764230F
:10D6C800A9E7B9F57A7F0ABF204F214FA060B1E7DB
:10D6D800049B0BB9C4F80CB05F46D0E70020934216
:10D6E800207506D85B1A9A4505F1010528BF9A46A8
:10D6F800EDB2002EE1D1B9F1640F164AADF83460ED
:10D7080019D049F6B023B9F57A7F18BF134690456A
:10D7180084BF039A9B180C931C9B00930CAF97E84B
:10D7280006001B9B384603F0FCF997E8030003F05A
:10D7380077FA8246C1E74FF46163E8E78051010058
:10D7480040771B007F5101002FEC010080A81201D7
:10D75800002E930230EC01000378032B14D1437898
:10D7680003F00F021B098A704B7083788B80C27894
:10D7780043EA02238B800379C3F3021203F00F03F9
:10D78800CA700B7005207047002070472DE9F347D9
:10D7980098464379057990F907609146044690F9CF
:10D7A80006208A4683B190F9087075B30F2A12D102
:10D7B80094F909200F2E1ED194F90A60072D24D15F
:10D7C800002F08BF012720E090F90B7090F909207D
:10D7D80090F90A60E9E7A369019394F91530009379
:10D7E800216994F91430207BFFF728FE0028E1D145
:10D7F80005F0FD05DEE794F91D30B3420FDC94F91E
:10D808001C30B342DADA05F0FB0528468AF8002016
:10D8180089F8006088F8007002B0BDE8F0871E46FD
:10D82800CCE70000024B03FA00F0B0FBF1F07047C0
:10D8380040420F004FF4FA53B3FBF0F0704730B595
:10D848004FF47A750C1F6A4300FB042252001EBF76
:10D8580000F1FF341219B2FBF0F2914238BF1146C1
:10D86800039A1160820048431CBF013040084FF4FE
:10D878007A71121A01FB1323002BCABF03F2E73394
:10D8880093FBF1F1B3FBF1F1049B196030BD38B59E
:10D89800400014460D46F4F7B9F801462846F4F757
:10D8A80003F82146F4F700F8F3F7F2FE03F0C4FC9E
:10D8B800F3F7CEFF40B238BD2DE9F74F01930023AF
:10D8C8001F469C461C01058A5FFA84FE04F0F0049A
:10D8D800A54206D8019B82F800C01F7003B0BDE8BE
:10D8E800F08F0EEB4E054FEA4309AD000024466861
:10D8F80036F809602641F60727D5866806EB050A3B
:10D90800765916B3067836B9466926B136F80960ED
:10D918002641F60719D59AF8086090F901B046F340
:10D9280003084FFA88F8D8450FDC46F3031676B299
:10D938005E450ADB9AF8096006EB4608C66806EBFE
:10D94800C806367D4EB90137FFB20134102C05F1F7
:10D958000C05CCD10133DBB2B4E70CF101060EEBB8
:10D96800040801F80C805FFA86FCEEE72DE9FF4712
:10D9780004464068DDE90C671D468A46914603F077
:10D98800C9F923681B1A3B604FF000080123337064
:10D9980085F80080636813B12368834224D8CAF8E5
:10D9A8000080D4F81CC0A3699CF800E00393D4E974
:10D9B800030101AB83E80300237D0093DCF80C101E
:10D9C800237A627A7046FFF7D9FD334638602A46D3
:10D9D800E0694946FFF770FF2B782BB1C7F8008044
:10D9E800002004B0BDE8F0873378002B14BF0B206B
:10D9F8000C20F6E737B590F9002090F902509542CF
:10DA080004460FD0013A52B295420BD0A368019355
:10DA180094F9013000936168E0782B46FFF70EFD1A
:10DA28000028EFD0104603B030BD8842B8BF084682
:10DA38007047000051F82000054B984205D0054B6F
:10DA4800C31A58425841400070470120704700BF30
:10DA580090D0030020A1070005281FB50ED80C4B55
:10DA680053F820300093CDE901120A4B012200211E
:10DA7800022002F05BFE05B05DF804FBCDE9001260
:10DA8800054B01220021022002F050FEF3E700BFFF
:10DA9800241E0108BB1D0108DA1D010807B5054B46
:10DAA800CDE9000101220021022002F03FFE03B06F
:10DAB8005DF804FBF61D010810B51022044600218C
:10DAC800F13000F051FE0021C4F814112046F02274
:10DAD800BDE8104000F048BE02460846102100F09C
:10DAE800A5B92DE9F0430446D0F8140185B00E46D7
:10DAF800154604F2011988B3C0F11008904547464D
:10DB080028BF1746BAB2484400F01AFED4F81431B8
:10DB18003B440F2BC4F814312DD9A8452BD204F15E
:10DB2800F00304F5807113F8012F187C8B4282EA08
:10DB380000021A70F7D104F1F10810224146684634
:10DB480000F0FEFD22466946684600F0E9F9102219
:10DB58006946404600F0F4FD3E44ED1B04F580782C
:10DB680004F1F107102D09D8AAB23146484600F051
:10DB7800E7FDC4F8145105B0BDE8F08304F1F003E3
:10DB8800711E13F8012F11F8010F434582EA0002B4
:10DB98001A70F6D110223946684600F0D1FD2246A7
:10DBA8006946684600F0BCF910226946384600F01C
:10DBB800C7FD1036103DD5E7F0B589B00C461022E8
:10DBC80000210546684600F0CFFD224669466846B2
:10DBD80000F0A6F99DF90030002B6A464FF00001CD
:10DBE80043DA137812F8010F01315B0043EAD013CE
:10DBF8000F2902F8013CF4D19DF80F305B0083F047
:10DC08008703D4F81401DBB210288DF80F303BD10C
:10DC180004F58073694604F5887013F8016F11F8EC
:10DC2800012B984282EA06021A70F6D104F1F00339
:10DC380004F5807113F8012F187C8B4282EA0002E8
:10DC48001A70F7D110220DEB020004F1F10100F077
:10DC580077FD2246294604A800F062F91022002127
:10DC6800684600F081FD09B0F0BD137812F8010F85
:10DC780001315B0043EAD0130F2902F8013CF4D1CB
:10DC88009DF80F305B00BCE79DF90030002B6A4619
:10DC98004FF0000137DA137812F8016F01315B0099
:10DCA80043EAD6130F2902F8013CF4D19DF80F304E
:10DCB8005B0083F08703471CDBB28DF80F30102F11
:10DCC80004EB0003C0F10F064FF0800288BF002666
:10DCD80000F5817083F801210021324620443E443A
:10DCE80003F064FAC4F8146104F58073694604F516
:10DCF800887013F8016F11F8012B984282EA060226
:10DD08001A70F6D192E7137812F8016F01315B00AF
:10DD180043EAD6130F2902F8013CF4D19DF80F30DD
:10DD28005B00C8E70A780378534003704A78437861
:10DD3800534043708A78837853408370CA78C37895
:10DD48005340C3700A790379534003714A79437980
:10DD5800534043718A79837953408371CA79C3796F
:10DD68005340C3710A7A037A534003724A7A437A5A
:10DD7800534043728A7A837A53408372CA7AC37A49
:10DD88005340C3720A7B037B534003734A7B437B34
:10DD9800534043738A7B837B53408373CA7BC37B23
:10DDA8005340C373704710B50B7814786340037001
:10DDB80054784B786340437094788B7863408370D1
:10DDC800D478CB786340C37014790B7963400371BE
:10DDD80054794B796340437194798B7963408371AB
:10DDE800D479CB796340C371147A0B7A6340037298
:10DDF800547A4B7A634043728B7A947A6340837285
:10DE0800D47ACB7A6340C372147B0B7B6340037371
:10DE1800547B4B7B63404373947B8B7B634083735E
:10DE2800CB7BD27B5340C37310BD0000A1F110031C
:10DE3800DBB2102B2DE9F04704D8374C24FA03F352
:10DE4800DB0705D4002382F8F030FF20BDE8F08717
:10DE5800531E4418A0424ED101F11C039B005FFAE7
:10DE680083F9C3F30313013B2C4D82F8F0300124EE
:10DE78000B46D618B3FBF1F001FB103010F0FF0091
:10DE880016F804AC16F803EC16F802CC16F8017C68
:10DE980036D115F80E8015F80CE015F807C015F8FE
:10DEA8000A70E00900EB400084EA080800EBC000B3
:10DEB8006400C0B2E4B24440C246581AC0B212F874
:10DEC80000808AEA080A02F803A01044043390F894
:10DED80001808EEA080E86F801E090F802E08CEAEC
:10DEE8000E0C86F802C0C078DBB247409945F7703F
:10DEF800BFD80020AAE710F8015B03F8015FA9E783
:10DF08001829DAD9102801BF15F80AA015F80EE06B
:10DF180015F80CC0EF5DD0E7010101003C200108B5
:10DF28002DE9F04FA3B092F8F0301D911B920193A8
:10DF3800002B00F0538101461EA8FFF734FF1B9BFE
:10DF4800A74CA84DA84E10330293002303939DF8C5
:10DF58007C0004909DF886000590205C06909DF852
:10DF68007B000790205C089004989DF881C0205C95
:10DF7800099014F80C000A909DF880000B909DF809
:10DF880085009DF878809DF87DE09DF882A09DF839
:10DF980087900C909DF87A00029B1C9314F80A2035
:10DFA80014F8093014F8081014F80E700D90205C5D
:10DFB8000E909DF87F000F90205C10900B98205CCD
:10DFC80011900C98205C12909DF8840013909DF895
:10DFD800790014909DF87E001590205C16909DF8AD
:10DFE80083001790205C18901398205C199014985F
:10DFF800205C1A900398013003900298DDF804B071
:10E00800103002909DF80C00834536D88DF87810B2
:10E018008DF87A2009990E9A8DF87C108DF8822057
:10E028001199069A8DF880108DF87E201999169A04
:10E038008DF884108DF886200A99189A8DF87D102D
:10E048008DF887201299109A8DF87B301B9B8DF8DC
:10E0580081108DF883201A99089A1D988DF88510DB
:10E068008DF87F201EA903EB0B128DF87970FFF74E
:10E078009AFE002023B0BDE8F08F15F808B082EAB8
:10E0880003008BEA000016F80EB080EA0B008DF84A
:10E09800780015F80E004B40434016F80A0043403C
:10E0A8008DF8793081EA070315F80A10594016F8F7
:10E0B8000930594016F808308DF87A107A405340E4
:10E0C80015F8092053408DF87B30089A069B534079
:10E0D800049AAA5C534016F80C2053408DF87C3003
:10E0E800DDE908325A4015F80C305340059AB25C05
:10E0F80053408DF87D30DDE909325A40059BEB5CD1
:10E108005340079AB25C53408DF87E30069B0A9ABA
:10E118005340049AB25C5A40079BEB5C5A408DF816
:10E128007F200E9B109A53400B9AAA5C53400C9A7E
:10E13800B25C53408DF88030DDE910325A400C9BB8
:10E14800EB5C53400D9AB25C53408DF88130DDE9A9
:10E1580011325A400D9BEB5C53400F9AB25C53400E
:10E168008DF88230129A0E9B53400B9AB25C5A403B
:10E178000F9BEB5C1C995A408DF88320169B189ACC
:10E188005340139AAA5C5340149AB25C53408DF8DA
:10E198008430DDE918325A40149BEB5C5340159AE1
:10E1A800B25C53408DF88530DDE919325A40159B31
:10E1B800EB5C5340179AB25C53408DF886301A9A3C
:10E1C800169B5340139AB25C5340179AAA5C1EA838
:10E1D80053408DF88730FFF7A5FDB8E6FF2049E7E3
:10E1E8003C2001083C1E01083C1F010808B538B155
:10E1F800044A05491060D82200F0A2FA002008BDA0
:10E208000220FCE7701C00206C2501080A4B1A68E4
:10E2180070B5002302F1180503EB03142E5D864246
:10E2280004D1183422440A60002070BD01330B2B3E
:10E23800F2D10320F9E700BF701C00202DE9F0415E
:10E24800CCB00646DDF8488117461C460D4631B36A
:10E25800B8F1000F23D006A8FFF72EFC204601A92D
:10E26800FFF7D4FF0446B0B9019906A80131FFF7BA
:10E2780033FC26B11022314606A8FFF732FC3A4695
:10E28800294606A8FFF72DFC06A902A8FFF794FC6B
:10E29800029BC8F8003020464CB0BDE8F08102244B
:10E2A800F9E7000030B595B013A90446FFF7AEFFB3
:10E2B800002830D11B490C2303FB00F2555CA54212
:10E2C8002BD1139B187C1090D87B0F90987B0E90C5
:10E2D800587B0D90187B0C90D87A0B90987A0A90FE
:10E2E800587A0990187A0890D87907909879069002
:10E2F8005879059018790490D87803909878029006
:10E308000A445B780193936800930022064B1146F8
:10E31800022002F00BFA15B030BD01300B28CBD12A
:10E32800F9E700BFB42201083C2101080B2B10B407
:10E3380002D810BCFFF782BF032010BC704730B56D
:10E348000D4685B01446014668B103AA0020009224
:10E358002A460390FFF772FF18B90398001B18BFED
:10E36800012005B030BD0220FBE72DE9F0430D4642
:10E37800BFB014469946804620B31BB311F00F0175
:10E3880022D1F02201A800F0EFF920466946FFF7F4
:10E398003DFF044648B9009801AA10210130FFF753
:10E3A80045FD2E46AF1BFFB21EB920463FB0BDE863
:10E3B800F08301AA09EB070108EB0700FFF7B0FD9E
:10E3C800103EEFE70224F0E70524EEE7F0B5184E1B
:10E3D8003468024685B00846002304F1180103EBAF
:10E3E80003154F5D97421ED10D2A05F1190513D16A
:10E3F8000023CDE90033CDE902330C2210216B460E
:10E40800FFF7B3FF0446306810226946284400F03D
:10E4180097F9204605B0F0BD01461022601900F0BA
:10E428008FF90024F5E701330B2BD8D10324F0E74B
:10E43800701C002009B1FFF7C9BF022070471FB543
:10E448001446A0B10C2A01D10B2912D10023CDE921
:10E458000033CDE902330A466B461021FFF785FFEA
:10E4680018B969462046FFF7B1FF04B010BD022075
:10E47800FBE70320F9E7F8B51E46DDE907479DF8F5
:10E4880018505BB354B34FB3212D29D819462A46E7
:10E49800204600F055F90122631C691EB018FFF7E9
:10E4A80064FFF8B9E37ADB093B70EBB963192046DE
:10E4B80013F8012C13F8021C120642EA014213F861
:10E4C800041C0A4313F8031C012342EA0122291FF2
:10E4D800FFF735FF003818BF0120F8BD0220FCE720
:10E4E8000520FAE70720F8E70420F6E708B5014613
:10E4F80030B1044B0822186800F022F9002008BD4A
:10E508000220FCE7701C002008B530B1044B08223B
:10E51800196800F015F9002008BD0220FCE700BFCB
:10E52800701C00207FB5124E0023044602A80193F8
:10E538000D46FFF7E9FF33685B6901936CB102AAE6
:10E54800082312F8011B41B9013B13F0FF03F8D16E
:10E5580002A8A04702A8FFF7C9FF35B1019B23B95C
:10E5680001A8A8473368019A5A61002004B070BD19
:10E57800701C002008B5014638B1054B1868082200
:10E58800104400F0DDF8002008BD0220FCE700BFC1
:10E59800701C002008B538B1044B196808221144D2
:10E5A80000F0CEF8002008BD0220FCE7701C002017
:10E5B800034B1B6802280CBF196159610020704782
:10E5C800701C002041B1054B1B6802280CBF1B6959
:10E5D8005B690B600020704702207047701C0020A8
:10E5E80030B58FB0002405460CA80994FFF78CFFBE
:10E5F8009DF8373007939DF8363006939DF83530EF
:10E6080005939DF8343004939DF8333003939DF8B7
:10E61800323002939DF8313001939DF830300093E9
:10E62800224621461E4B022002F080F80AA8FFF776
:10E63800B1FF9DF82F3007939DF82E3006939DF873
:10E648002D3005939DF82C3004939DF82B300393BF
:10E658009DF82A3002939DF8293001939DF82830BF
:10E66800009322460F4B2146022002F05FF809A9C9
:10E678002846FFF7A7FF9DF8243003939DF825301F
:10E6880002939DF8263001939DF827300093224687
:10E69800054B2146022002F049F80FB030BD00BFFB
:10E6A80098210108D62101081422010808B5002084
:10E6B800FFF7F8FD0120FFF7F5FD0920FFF7F2FD50
:10E6C8000820FFF7EFFD0020FFF78AFF002008BDB4
:10E6D80010B504460B20FFF7E5FD0C20FFF7E2FD1F
:10E6E8000920FFF7DFFD0820FFF7DCFD0A20FFF710
:10E6F800D9FD2046FFF774FF002010BD014B1860BC
:10E70800704700BF3C0100200B4A30B514680B4D20
:10E7180043F2390305FB04331360091A6FF0004212
:10E72800B3FBF2F2C2EBC27201319B1A93FBF1F216
:10E7380001FB1233184430BD3C0100206D4EC64128
:10E7480001380A44914200D1704711F8013B00F8A2
:10E75800013FF7E710440A44914200D1704711F88D
:10E76800013B00F8013DF7E702F020BD30B530B1BC
:10E778000A4D01444FF0FF33814201D1D84330BDE7
:10E7880010F8012B5340082243F30004013A2C40AF
:10E7980092B284EA5303002AF6D1EDE72083B8ED5C
:10E7A80001207047054B4FF400529A62044B1B68D6
:10E7B80013B15B6803B11847704700BF00040048F5
:10E7C800741D0020054B4FF480529A62044B1B685D
:10E7D80013B1DB6803B11847704700BF0004004855
:10E7E800741D0020012070470120704701F048B9CE
:10E7F80001F036B910B501F019FE0E21044640F6B5
:10E808001F1001F02DF92046012101F0F9FDBDE8A6
:10E81800104001F0D7BA000070B50C4E01EB400370
:10E828000D46B3654FF6FF71002304461A460846A5
:10E8380001F05EFB96F85600002101F0E1FD294643
:10E848002046BDE8704001F095BA00BF901D002039
:10E8580010B5044601F0AAFE01281CD101F0AEFE55
:10E8680034B11248214602F017FB104802F0DAFAD8
:10E878000F4C104B00214FF48052A1659A6194F817
:10E88800560001F0BDFD63786BB16FF07F40BDE8C5
:10E89800104001F053BA002340F262211A4608469C
:10E8A80001F026FBDCE7A0688001F0E7781D002076
:10E8B800901D002000040048002001F0BFB90000AE
:10E8C80008B501F0C7F80438C0B2032896BF024B58
:10E8D8000020185C08BD00BFC823010808B501F076
:10E8E800BAFD033008BD01F049B901F009B908B50E
:10E8F80001F000FD00B208BD38B50D46144601F020
:10E908005DFB284601F092FD0E21054640F61F10DA
:10E9180001F0A6F828460121074D01F071FD01F02C
:10E9280051FA4FF47A716143284602F0B5FA284645
:10E93800BDE8384002F076BAEC1D002001F03EBB7D
:10E9480008B5084B002193F8560001F059FD002343
:10E958004FF4C0711A46084601F0CAFABDE80840EB
:10E9680001F024BA901D002010B5044601F01EFEE7
:10E9780001281CD101F022FE34B11248214602F0D0
:10E988008BFA104802F04EFA0F4C104B00214FF44E
:10E998008052A1659A6194F8560001F031FD6378C0
:10E9A8006BB16FF07F40BDE8104001F07DB90023E6
:10E9B80040F262211A46084601F09AFADCE7A0689C
:10E9C8008001F0E7781D0020901D00200004004819
:10E9D80008B54FF0040001F017F9BDE8084002201F
:10E9E800F4F770B808B500231A461946184601F01E
:10E9F8007FFABDE8084001F06DB900001D4B73B502
:10EA08001D4D186000241D486C70C5E90144AC65B3
:10EA180001F098FAAC8101F003FA2146204601F092
:10EA28004BFC21460422012001F0FCFA144E154D3E
:10EA38004FF6FF7123462246084601F059FAFFF7C0
:10EA4800C7FF2246104B00944FF0FF31304602F0CA
:10EA58003DF90E4B009422464FF0FF31284602F054
:10EA680035F9304602F090F9284602B0BDE870400A
:10EA780002F08AB9741D0020901D00204DFA00088C
:10EA8800EC1D0020781D0020ADE70008CDE7000848
:10EA98000128084805D1084BC17719700E3001F0DC
:10EAA800A7BB437D012B03D1034B81751970F5E793
:10EAB800704700BF901D0020400100200D4B10B58D
:10EAC800044618735873012000F016F85CB134211D
:10EAD8004FF4E86000F0C4FF4421BDE8104040F264
:10EAE800417000F0BDBF14214FF4E86000F0B8FF9A
:10EAF8002421F2E7901D002038B5114C05462070FE
:10EB080001F061FD052D04D8DFE805F0090B0317B6
:10EB18001709032001F070FA0023637338BD002041
:10EB2800F8E7012001F068FA207B637B8342F5D087
:10EB38006073BDE83840FFF7C1BF0220EAE700BFB5
:10EB4800901D00202DE9F0431E4687B0002305469E
:10EB5800CDE901330C46174601F027FD032D61D896
:10EB6800DFE815F07B00C3000E010400A27C082A30
:10EB780004D94FF0FF3007B0BDE8F083A16801A8C1
:10EB880001F0DCFE21680029F3D042F210729142B4
:10EB9800E37C864D51D80322AA7385F83820E963AF
:10EBA80085F844304FF002086368A17DDB002B82B2
:10EBB8000423AB74A37CDB00EB7402294FF0000341
:10EBC8002B75637D02D0227D022A42D103F10F0208
:10EBD800D2B2012A01D9012BCBD1754B754A1968DC
:10EBE80003944FF0010903A88DF8149001F0DAFCA2
:10EBF8000028BED1287685F817906875FFF75CFE67
:10EC08004046FFF779FF6C4801F086FA6B4801F03F
:10EC1800EFFA01A800F084FF208A00F055FFA089D0
:10EC280000F09AFF384601F001FC604C84F8560069
:10EC380001F0C0FC666000209DE74FF00008E96322
:10EC4800890885F80E8085F8388085F8443029646D
:10EC5800AAE7EB7529766A75D0E72368002B88D078
:10EC6800A27C082A85D8514DA16801A801F066FE4A
:10EC7800002385F838302268EA63E27C85F844206E
:10EC8800A269AB732A646268A17DD2002A82042239
:10EC9800AA74A27C2B75D2000229637DEA7402D083
:10ECA800227D022A1DD103F10F02D2B2012A02D914
:10ECB800012B7FF45EAF3E4B3E4A196803944FF038
:10ECC800010803A88DF8148001F06CFC00287FF47B
:10ECD80050AF287685F817806875FFF7EDFD00209E
:10ECE8008FE7EB7529766A75F7E7304D012185F8CE
:10ECF8003810227885F85020637885F85130A37849
:10ED080085F85230E3788B4202D0022B03D03BB90E
:10ED180085F8533004E00B3A012A29D885F85310B6
:10ED28004FF0010885F80E80A388AB83A379AB77F1
:10ED3800E37985F82030237A85F82130FFF7BCFD88
:10ED48004046FFF7D9FE1C4801F0E6F91B4801F0E0
:10ED58004FFA95F85130062B40F689000AD100F099
:10ED68008FFE00F0FB0140F6890000F079FE59E7BC
:10ED78000023CDE700F084FE40F00401C9B2F2E7B9
:10ED88002368013BB3F57A7FBFF4F3AE0320FFF7A6
:10ED9800B3FE0648022380F83830236883641623BC
:10EDA80080F84C30383001F0B7F93BE7901D00206F
:10EDB800741D0020EC1D0020C81D00209E1D002091
:10EDC8002DE9F041002686B01F461446CDE90166BC
:10EDD80080460D4601F0E9FBB442764C16BF01238C
:10EDE800334637466370B8F1000F06D0B8F1010F0B
:10EDF8007CD0002006B0BDE8F081AB68002B00F0A5
:10EE0800D680EB68002B00F0D280AA7F082A00F297
:10EE1800CE80296901A801F091FD2868003818BF43
:10EE2800012000F0D9FF84F83880AB68E36395F8D7
:10EE3800203084F84430686801F05AFB84F80E806A
:10EE480084F84500EB68DB002382EB7FA374AB7F7B
:10EE5800DB00E37495F82130237595F82230002BF8
:10EE68003ED12A7D95F82410A275022995F8232011
:10EE780001D0022B36D102F10F03DBB2012B02D9EC
:10EE8800012A40F0948000238DF814304A4B4B4AF5
:10EE98001968049503A801F085FB002840F08780D5
:10EEA80001232076E3756075FFF706FD0020FFF764
:10EEB80023FE434801F030F9424801F099F901A8CE
:10EEC80000F02EFEA88B00F0FFFD288B00F044FE1A
:10EED8004FF4FA53AA687B43B3FBF2F3A36088E7C5
:10EEE800FF22BFE7E27521766375DDE72B8E002BE5
:10EEF8005DD095F83230A86A012B0CBF95F81480C4
:10EF08004FF0FF08003818BF012000F065FFF8B285
:10EF180000F06EFF012184F8381095F82C2084F851
:10EF2800502095F82D3084F8513095F82E3084F81B
:10EF3800523095F82F308B4202D0022B03D03BB9C8
:10EF480084F8533004E00B3A012A28D884F8531087
:10EF58002B8EA38395F83230A377AB8E23840126BA
:10EF6800A67384F81F80FFF7A7FC3046FFF7C4FD9F
:10EF7800134801F0D1F8134801F03AF994F8213018
:10EF8800B34240F236700CD100F07AFD00F0FB017C
:10EF980040F2367000F064FD4FF6FF739EE70023E1
:10EFA800CEE700F06DFD40F00401C9B2F0E74FF084
:10EFB800FF301FE7901D0020741D0020781D0020E1
:10EFC800C81D00209E1D00202DE9F04F85B0824607
:10EFD8000E9DBDF840B09DF844709DF84890019290
:10EFE80088461E4601F0E1FABAF1010F524C54D09E
:10EFF800BAF1040F00F09180BAF1000F3AD10B2258
:10F00800304684F8442084F838A0E56301F070FAAB
:10F01800019B23644FEACB03B9F1000F238241F629
:10F028000403638214BFF2230123E37587F0010709
:10F038000123237684F8450084F80EA084F814A0F0
:10F048006775FFF739FC5046FFF756FD04F13800A5
:10F0580001F062F804F10E0001F0CAF8374A1068AE
:10F06800516802AB03C302A800F05AFD40F2FF103A
:10F0780000F02AFD404601F0D9F90E2184F8560027
:10F0880040F61F1000F0ECFC94F8560001F092FADC
:10F09800169B636005B0BDE8F08F294984F838A055
:10F0A800EAB2895D84F8502076BB0B3D012D8CBFF8
:10F0B80000250125053A012A04D8BBF10C0F38BFF9
:10F0C8004FF00C0B1F4B9DF83C201B7884F85350D5
:10F0D800E37701259DF8543084F8511084F85220C4
:10F0E80084F82130A573A4F81CB0A77784F8209081
:10F0F800FFF7E2FB2846FFF7FFFC134801F00CF886
:10F10800124801F075F8B5E7012E04D1A5F10C03FA
:10F118005D425D41CEE70025CCE75046FFF7ECFCA9
:10F12800022384F8383004F138001623A56484F8E3
:10F138004C3000F0F1FF9DE7901D0020A813010856
:10F148009623010840010020C81D00209E1D0020B4
:10F158002DE9F04F87B0DFF8B4B29DF864A09DF8B0
:10F168004C90029314469DF854309DF85020BDF8F9
:10F178004880039205468BF801A0BDF844600193CE
:10F188000F4601F012FABAF1000F18BF4FF000084D
:10F19800DFF87CA2039AB9F1000F08BFFF22012D06
:10F1A8008AF8002000F0C880052D48D0002D40F0D6
:10F1B800C080284600F010FE0B2238468BF8442009
:10F1C8008BF83850CBF83C4001F092F9019B8BF852
:10F1D800450041F60402002BABF812209AF80020F3
:10F1E8008BF8162014BFF22201228BF81720F600A4
:10F1F800012289F001098BF818208BF80E50ABF822
:10F2080010608BF814508BF81590FFF755FB2846C3
:10F21800FFF772FC0BF1380000F07EFF0BF10E00D7
:10F2280000F0E6FF7B490868496804AA03C204A8FD
:10F2380000F076FC40F2FF1000F046FC71E001207F
:10F2480000F0CAFD09224FF000098BF84420384627
:10F258004FF44872CBF840208BF83890CBF83C40FC
:10F2680001F046F94FF48052ABF812209AF80020CA
:10F278008BF845008BF8162028460122F6008BF8FB
:10F2880017208BF80E90ABF81060ABF814908BF841
:10F298001890FFF731FC0BF1380000F03DFF0BF13F
:10F2A8000E0000F0A5FF5B498868C96804AA03C27C
:10F2B80004A800F035FC40F2FF1000F005FC40F611
:10F2C800B80000F0DDFB00F0EF0140F6B80000F0F8
:10F2D800C7FB042140F6B90000F0C2FB40F69B00D2
:10F2E80000F0CEFB00F0E30141F0080140F69B007E
:10F2F80000F0B6FB40F2D16000F0C2FB40F018010C
:10F30800C9B240F2D16000F0ABFB40F2AC6000F053
:10F31800B7FB00F08F0141F0500140F2AC6000F003
:10F328009FFB4FF4FA5202FB08F2B2FBF4F2CBF85F
:10F33800082007B0BDE8F08F002000F04DFD3649E9
:10F348008BF83850E2B2C95D8BF85020002F4DD1B0
:10F358000B3C012C8CBF00240124053A012A02D859
:10F368000C2E38BF0C26029B9AF800208BF85230DE
:10F378008BF85340019B8BF81F2001249DF86020D7
:10F388008BF821208BF851108BF820308BF80E4029
:10F39800ABF81C608BF81E90FFF78EFA2046FFF73B
:10F3A800ABFB1E4800F0B8FE1D4800F021FF5FFAD5
:10F3B80088F000F01DFD40F6A30000F061FB00EAB4
:10F3C800040140F6A30000F04BFB9BF82120A24269
:10F3D80040F2367013D100F053FB00F0FB0140F20D
:10F3E800367000F03DFB4FF6FF72A0E7012F04D105
:10F3F800A4F10C035C425C41AFE70024ADE700F0E8
:10F408003FFB40F00401C9B2E9E700BF901D0020AE
:10F4180040010020A813010896230108C81D0020F8
:10F428009E1D0020F0B58BB00D46044617461E46BB
:10F43800FFF742FA0020FFF75FFB204600F0BEFD11
:10F4480000240123CDE9084303234FF4167229460B
:10F458002046CDE90644CDE90444CDE90244CDE98E
:10F4680000532346FFF774FE2046FFF77DFAFFF7A7
:10F4780035FAF3F727FB01F043FC0446204601F078
:10F4880049FCB04205D30124FFF716FA20460BB019
:10F49800F0BD00F02FFF00B28742EFDA0024F3E757
:10F4A800F7B500230C4640F201211A4606460846E5
:10F4B80000F01EFD644B654D4FF400529A6195F8BB
:10F4C8005600012100F09CFF2B78012B40F68900A3
:10F4D80013D195F85130062B0FD100F0D1FA00F076
:10F4E800FB0140F6890000F0BBFA2B78042B6CD89E
:10F4F800DFE803F0524B527F090000F0C1FA40F0F8
:10F508000401C9B2EDE7524A731E1046C6F101075D
:10F518004FF0000CF9188C426FDC0022E70013460C
:10F52800BA4271D19A0142EAC3125B0183F0200307
:10F538001343661C0355F6B202234648AB73AE76F6
:10F5480000F056FE0021F12000F08AFA0021F02098
:10F5580000F086FAAB6C642B70D17021F32000F0B8
:10F568007FFA1D21F22000F07BFAE1008C1CF420C8
:10F57800090A00F075FA04F0FE01F52000F070FAAF
:10F5880033486FF07F4231461DE0EC77314800F098
:10F598002FFE0022214615E001F008F80128074651
:10F5A80025D121460DF10702304601F004F8044642
:10F5B800A0B99DF807302748AB7500F019FE9DF8F3
:10F5C80007102246304600F065FB6968224801F0C2
:10F5D80063FC214801F026FC002006E01F4B3A4658
:10F5E8000021022001F0A2F8032003B0F0BDAC75A1
:10F5F800CCE70223AB73AC76C8E713F8011FC94305
:10F60800197002F801CB85E7D1106FEA020C715C22
:10F618000CF0070C013241FA0CF101F001014FEA3C
:10F62800E20C4B40D14310F80CE001F0070103FA5B
:10F6380001F141EA0E0100F80C1071E7E121F32015
:10F6480000F00EFA04218DE700040048901D002008
:10F65800741C00209E1D0020EC1D0020382301088A
:10F66800F0B5BDF814409DF818709DF81CE09DF8A1
:10F67800205040B1012814D00122002398180138E5
:10F68800B0FBF2F0F0BD87F00107E30003EBC7031E
:10F6980018330EEB450503EBC5034FF47A714B4362
:10F6A800ECE7501F012803F1040302D80C2C38BFE3
:10F6B8000C24D1B9A2F10B0CBCF1010F8CBF4FF097
:10F6C800000C4FF0010C2801002F00EBCE0014BFF6
:10F6D80000251425A0EB8200062A4FEA820628445A
:10F6E800A2F102070DD8354610E0012906D1A2F192
:10F6F8000C00D0F1000C4CEB000CE4E74FF0000CD0
:10F70800E1E70830BCF1000FEDD0BD000028ACBF28
:10F718002E182E1C701E90FBF5F003FB0044094BBD
:10F72800062A5A5C8CBF0C340E340A2A09D8A30066
:10F7380001334FF47A71BB404B43034951F82220FF
:10F748009CE7FFDE962301089C23010808B5094BB6
:10F75800012193F8560000F053FE4FF4D7602D2195
:10F7680000F07EF900F033FBBDE80840024800F0E5
:10F778007BBA00BF901D0020FFFF0F0073B5A44C9B
:10F78800B4F854300025202B8DF80350019500F073
:10F798001B8114D8082B0DD87BB1013B072B0CD843
:10F7A800DFE813F042005B000B00CD000B000B00FC
:10F7B8000B00FD00102B00F0008102B070BDB3F506
:10F7C800807F00F0988011D8402B00F01081802BAA
:10F7D800F3D1284600F032FA8E4B1B68002BECD090
:10F7E8009B69002BE9D028469847E6E7B3F5007FE8
:10F7F800E3D1894B01222946022000F097FF00F04F
:10F8080029F9042840F08580844B85484FF400523C
:10F818009A6201F0B9FA284600F010FA7D4B1B688D
:10F82800002BCAD05B6814E07C4B7D484FF4005233
:10F838009A6201F0A9FA002000F000FA00F0B8FE80
:10F84800012801D100F0BDFE724B1B68002BB4D01B
:10F858001B68002BB1D09847AFE7704B71484FF445
:10F8680080529A6201F090FA657895B9284600F0BE
:10F87800E5F9294640F6021000F0F2F840F6441087
:10F8880000F0FEF840F00201C9B240F6441000F062
:10F89800E7F8FF220DF1030163485E4D00F05AFDC1
:10F8A800624800F071FD2B68002B86D09E68002E00
:10F8B80083D094F82430012B08D194F9313094F98D
:10F8C80030209DF803105848B04776E7E06B01A94F
:10F8D80000F022FE019B9DF8031053484FF47A7202
:10F8E80003F5FA7393FBF2F32A685BB2956894F90F
:10F8F8002920A84761E7284600F0A0F9454B1B6876
:10F90800002B3FF45AAF9B69002B3FF456AF012000
:10F918006AE700F09FF805287FF44FAF3F4B414856
:10F928004FF480529A6201F02FFA284600F086F9C7
:10F93800384B1B68002B3FF440AFDB6889E7002198
:10F948003B4B0122022000F0F1FEA16D00293FF49B
:10F9580034AFC1F3074140F6031000F081F894F882
:10F96800591040F6041000F07BF894F8581040F64F
:10F97800051000F075F840F6021000F081F840F02C
:10F988000101C9B240F6021000F06AF8002340F203
:10F9980062211A460846A36500F0AAFA0DE7254B2E
:10F9A80001220021022000F0C1FE00F0FFFD012825
:10F9B8007FF403AF00F006FEFFE61F4B0122002193
:10F9C800022000F0B3FEF8E6164801F0DDF9607891
:10F9D80008B900F033F90F4B1B68002B3FF4EDAE6C
:10F9E800DB68002B3FF4E9AE9847144BE6E7144B6D
:10F9F80001222946022000F099FE607808B900F03B
:10FA08001DF9044B1B68002B3FF4D7AE1B6920E798
:10FA1800901D0020741D00204D230108000400489B
:10FA2800EC1D0020781D0020741C0020B41D00204F
:10FA3800612301086A230108742301087D23010852
:10FA480086230108024BA3F85400FFF797BE00BFB6
:10FA5800901D0020014B1878704700BF0A1E002037
:10FA680007B501238DF807100DF107020146034879
:10FA7800F7F786F803B05DF804FB00BF4C030020DD
:10FA880007B5012301460DF107020448F7F7B1F85D
:10FA98009DF8070003B05DF804FB00BF4C0300208D
:10FAA80010B50446F4F716FD01280CD140F62310D2
:10FAB800FFF7E6FF00F0F901214340F62310BDE807
:10FAC8001040FFF7CDBF10BD10B50C4B1B78044696
:10FAD8009BB94FF4D760FFF7D3FFC4F3002100F0C0
:10FAE800FE0001434FF4D760FFF7BAFFE1B240F2DE
:10FAF800B960BDE81040FFF7B3BF10BD0B1E002072
:10FB080010B51346EFF3108472B60A46014603484F
:10FB1800F7F736F884F3108810BD00BF4C030020B7
:10FB280008B5014608224FF4D860FFF7E9FF002026
:10FB380008BD000007B5074B1B7840BAADF80400B4
:10FB48002BB9022201A940F2BC60FFF7D9FF03B02C
:10FB58005DF804FB0B1E002007B5074B1B7840BA65
:10FB6800ADF804002BB9022201A940F2BE60FFF7EC
:10FB7800C7FF03B05DF804FB0B1E002010B5134649
:10FB8800EFF3108472B60A4601460348F7F731F8D6
:10FB980084F3108810BD00BF4C03002010B5134635
:10FBA800EFF3108472B60A4601460348F7F713F9D3
:10FBB80084F3108810BD00BF4C0300200A4601469C
:10FBC8000020FFF7EBBF000010B51346EFF31084D9
:10FBD80072B60A4601460348F7F730F984F31088ED
:10FBE80010BD00BF4C03002010B51346EFF310847E
:10FBF80072B60A4601460348F7F736F884F31088C8
:10FC080010BD00BF4C03002013B504460020F4F7D4
:10FC18003BFC0220FFF744FF04F0070401220DF12A
:10FC2800070184208DF80740FFF7DEFF024B002212
:10FC38001A7002B010BD00BF0A1E002007B50122CD
:10FC48008DF807000DF107018020FFF7CDFF9DF823
:10FC58000730002B034B0CBF012202221A7003B09D
:10FC68005DF804FB0A1E002007B5094B8DF8060055
:10FC780004221A70030C8DF804300322030A01A928
:10FC880083208DF80530FFF7AFFF03B05DF804FB64
:10FC98000A1E002010B51446FFF790FF2046BDE865
:10FCA8001040FFF7E1BF000007B5094B8DF80600CB
:10FCB80005221A70030C8DF804300322030A01A9E7
:10FCC80082208DF80530FFF78FFF03B05DF804FB45
:10FCD8000A1E002073B5002640F6E2000196FFF7E1
:10FCE800CFFE00F0FE01054640F6E200FFF7B8FE41
:10FCF80040F6E500FFF7C4FE00F07F01044640F639
:10FD0800E500FFF7ADFE6FF07F40FFF7CDFF04225F
:10FD18000DEB020140F61900FFF730FF3046FFF700
:10FD28008DFF294640F6E200FFF79AFE214640F68D
:10FD3800E500FFF795FE019802B070BD13B50C4BB6
:10FD480004460522972140F6AC001A70FFF788FE9A
:10FD5800230C8DF804300322230A01A982208DF890
:10FD680005308DF80640FFF73FFF02B010BD00BF19
:10FD78000A1E002007B5030C8DF80030030A8DF821
:10FD880001300B0C49BA8DF80200ADF804100622B8
:10FD9800694694208DF80330FFF726FF024B0622B0
:10FDA8001A7003B05DF804FB0A1E0020002208B593
:10FDB8001146C520FFF718FF014B07221A7008BD2E
:10FDC8000A1E002000221146D120FFF70DBF002295
:10FDD8001146D220FFF708BF07B501228DF80700AA
:10FDE8000DF107019F20FFF7FFFE03B05DF804FB4C
:10FDF80007B501228DF807000DF10701A020FFF7D4
:10FE0800F3FE9DF807103F2907D901F0F8010131E9
:10FE1800C9B240F20670FFF723FE03B05DF804FB99
:10FE280007B5F4F757FB431E584258418DF80700B1
:10FE380001220DF107019620FFF7D6FE03B05DF809
:10FE480004FB07B500F07F008DF8070001220DF1D3
:10FE580007018920FFF7C8FE03B05DF804FB000026
:10FE6800154B984207B51BD8144B98421BD8144B16
:10FE780098421BD8134B98421BD8134B984295BFF6
:10FE880029226B222B236F238DF8042001A902223B
:10FE980098208DF80530FFF7A7FE03B05DF804FB46
:10FEA800E122E923F0E7D722DB23EDE7C122C523CE
:10FEB800EAE775228123E7E700E9A43580F8A9324B
:10FEC8008044E52D000B6B1B40FC541907B58DF8D9
:10FED800062004228DF804008DF8051095200DEBFE
:10FEE80002018DF80730FFF77FFE03B05DF804FBD1
:10FEF80007B552BAADF8042040BA082249BAADF89D
:10FF08000000ADF802105BBA69461046ADF806303D
:10FF1800FFF76AFE03B05DF804FB07B50B0C04227B
:10FF280000F0070049BA8DF80400ADF806109720D4
:10FF38000DEB02018DF80530FFF756FE03B05DF8B2
:10FF480004FB000010B508B1194B1860F2F7BCFCAF
:10FF58000220FFF7A5FD0024164B20461C70FFF772
:10FF68006DFEF4F7B5FA012817D14FF42071FFF7A9
:10FF7800D4FF40F611102146FFF772FD4FF07F00C5
:10FF8800FFF75FFF0E2140F61F10FFF769FDF4F73A
:10FF980047FA094B01221A7010BD102140F61110C2
:10FFA800FFF75EFD102140F61210FFF759FDE9E753
:10FFB8000C1E0020081E00200A1E002037B50C4D1C
:10FFC8002B7804461BB9FFF74BFF01232B70002346
:10FFD800084A6006E109F1F797FD042200BA01908A
:10FFE8000DEB02018620FFF7FFFD03B030BD00BF17
:08FFF800081E00200048E8018A
:020000040801F1
:1000000007B5094B8DF807000146187018B940F282
:10001000AC60FFF729FD01220DF107018A20FFF7EF
:10002000E7FD03B05DF804FB0B1E0020012873B54B
:100030000C46164637D10020F4F752FAA042B8BF5A
:1000400044B20E2805461AD101231A460021042085
:10005000FFF740FF6FF010039C42B8BF1C46182109
:1000600040F6E700FFF700FD022201A98E208DF87F
:1000700004408DF80560FFF7BBFD02B070BD0123A1
:100080000A28E4B21A464FF0000105D11846FFF7DE
:1000900021FF033464B2DDE70720C5F10E05FFF749
:1000A00019FF2C44F6E740F6D800FFF7EDFC40F0CE
:1000B0001E01C9B240F6D800FFF7D6FC0120F4F7C4
:1000C0000FFAA042B8BF44B2142805464FF001030E
:1000D0004FF000020CD105210320FFF7FBFE023494
:1000E00064B26FF008039C42B8BF1C463821B7E7E2
:1000F000112805D103210220FFF7ECFE0534EFE7BC
:100100000E2804D102210846FFF7E4FEE9E7C5F115
:100110001605072104202544FFF7DCFE6CB2E0E75A
:1001200013B5314A0446516810686B4603C32F4B20
:1001300020781B78834201D0FFF762FF2378032BDE
:1001400027D8DFE803F00239283C6268284BB3FB6C
:10015000F2F31A0CA1688DF800208DF802301A0A0B
:10016000237B8DF80330637B8DF801208DF80430FC
:10017000204A00234806C909F1F7CAFC030C40BA1B
:100180008DF80530ADF80600082269468B20FFF790
:100190002FFD02B010BD2269154BB3FBF2F31A0C10
:1001A0008DF800208DF802301A0A237D8DF8012089
:1001B0008DF803300422E8E7A3690093FAE7626848
:1001C0000B4BB3FBF2F31A0C8DF800208DF80230C4
:1001D0001A0A237B8DF80330637B8DF801208DF89C
:1001E00004300522D1E700BFB81301080B1E002020
:1001F0000000093D0048E8011FB52E4A0446D168B9
:100200009068127C01AB03C31A702B4B20781B78CB
:10021000834201D0FFF7F4FE2378032B26D8DFE8D2
:1002200003F002383302637AF12B21D14FF6FF70CD
:10023000FFF784FC48F20500FFF792FC0223628876
:10024000A188ADF8061052BAE188ADF804208DF807
:100250000B30227AA37A8DF80A20ADF808108DF8B9
:100260000C30092201A98C20FFF7C2FC04B010BD9C
:10027000F22BE4D141F60F50FFF760FC41F2210070
:10028000FFF76EFC0623DAE7237B8DF804300122AA
:10029000E8E7E389094A5BBAADF80430237C1370C0
:1002A0008DF80630637C8DF80730638AADF808302E
:1002B0000622D7E7B81301080B1E0020091E0020F4
:1002C00007B502228DF804008DF805108F2001A9D2
:1002D000FFF78EFC03B05DF804FB000010B5134679
:1002E000EFF3108472B60A4601460348F6F7F8FCAD
:1002F00084F3108810BD00BF4C03002007B5012215
:1003000001A91520FFF7EAFF9DF8040040424010C4
:1003100003B05DF804FB000037B505460C46022229
:1003200001A91320FFF7DAFF0A4B1B78012B0DD12F
:10033000094B1B78012B09D140F20270FFF7A4FB97
:100340009DF805302870237003B030BD9DF804007F
:10035000F6E700BF0B1E0020091E0020F7B50D4672
:10036000064600240DF10701284617468DF8074080
:10037000FFF7D2FF2A78BA4207D89DF80700314626
:10038000FFF726FC204603B0F0BD0120FBE700008C
:1003900013B50322044601A91420FFF79FFF184B51
:1003A0001A7822704AB1012A17D01422002120465F
:1003B00000F0D2FA0F2323700DE09DF80430237172
:1003C0009DF80530A2605B425B10A3719DF806307A
:1003D0005B425B10637102B010BD9DF804305B425C
:1003E0005B1023739DF9053002339B1063739DF8F6
:1003F00006305B425B10A373024B1B682361EAE784
:100400000B1E0020041E0020012908B503460846E3
:100410000ED1012B07D10420FFF746FB0220BDE8D7
:100420000840F4F735B8022B14BF08460320F6E75E
:100430000120F4E738B50446F4F74CF850B102282F
:1004400014BF01250225284602222146FFF7EEFDB2
:10045000284638BD0F2CCCBF02250125F3E70A2022
:1004600070470000014B01201B6818470C1E00203C
:10047000014B02201B6818470C1E0020014B402036
:100480001B6818470C1E002011B1012904D07047C9
:10049000044B1B6880201847024B4FF480701B6888
:1004A000F9E700BF0C1E0020024B4FF400701B68E0
:1004B000184700BF0C1E0020014B20201B68184766
:1004C0000C1E0020014B04201B6818470C1E002046
:1004D000014B08201B6818470C1E0020014B102000
:1004E0001B6818470C1E0020024B4FF480401B680D
:1004F000184700BF0C1E002068B1084A002352F8BC
:100500003310814203D902EBC302107970470133E3
:10051000162BF4D1FEE71F20704700BF58240108B6
:1005200073B51D4B0193044640F607000D46FFF7D7
:10053000ABFAC0F3C10308336B4413F8042C00F08A
:100540000703013302FA03F3144AB2FBF3F2B2FBDE
:10055000F4F007281ED8400003288CBF0223042390
:100560004FF4D66002FB03F4FFF78EFA060240F266
:10057000B160FFF789FA06F470663043030544BFA3
:100580006FEA00506FEA105063094343DB112B60A0
:1005900002B070BD0123E3E704080A0C0048E8013B
:1005A0004FF0FF3070474FF0FF3070474FF0FF3093
:1005B00070477047002070470020704770474FF029
:1005C000FF3070474FF0FF307047704770477047FB
:1005D00070B5EFF3108672B6144B5C8A1A8A944297
:1005E00013D1C4F5806292B2904206D3844218D9E6
:1005F00001229A7000221C805A825A8A0A80024480
:10060000C2F309025A8200200DE006D9C4F58065C4
:10061000ADB28542F1D88242E9E7121B92B2824222
:10062000EBD84FF0FF3086F3108870BD1022002009
:10063000EFF3108172B6034AD38A0133D38281F378
:100640001088704710220020EFF3108172B6034A21
:10065000D38A013BD38281F3108870471022002097
:1006600010B508481822002100F076F906484FF42A
:100670008062002100F070F9044B05481B68BDE85A
:100680001040184710220020101E00207814010886
:1006900001080108014B5860704700BF102200207C
:1006A000014B1872704700BF1022002073B5EFF3A2
:1006B000108572B61C4CE08A00282FD1FFF7B8FFD6
:1006C000218A628A914227D0A378012B12D12388F4
:1006D00020805B1A9BB20221A382A17063B9A37030
:1006E0002382238A9A428BBFD21AC3F58063A282E7
:1006F000A38201E0002BF4D0238A0C4E1E4485F324
:100700001088F2F7D1F90A4BA18ADB6801933046D1
:1007100002B0BDE870401847FFF796FF85F31088D8
:10072000002002B070BD00BF10220020101E00206B
:100730007814010808B4F0B586B00023ADF8003095
:100740002C4B0B9C1D7A85424DD3D86881434DD1EB
:100750005B681BB112B1694602A898470CAB2246F0
:100760004FF400712448019300F0F6FBFFF760FF9F
:10077000BDF8003018440DF1020180B2FFF728FFE8
:1007800001302BD00022BDF80030BDF802701B48AC
:100790000DF1080C164691B217FA82F58B42ADB2F4
:1007A00016D83B449BB20EB1ADF80230BDF80250F2
:1007B000019B22464FF40071284400F0CDFBFFF767
:1007C00043FFFFF773FF06B0BDE8F04001B070478C
:1007D0001CF8011B415501320126DCE7FFF734FF0D
:1007E0006FF00200EFE76FF00400ECE76FF0050038
:1007F000E9E700BF1022002028220020101E002060
:1008000013B5EFF3108472B6204B9A78588A022AF7
:100810001DBF1A8A998A5218002214BFC2F3090216
:100820009A7090421A8228D0D98A012925D19978C4
:10083000012913D119888A1A022192B299700021D4
:100840009A82198062B99A701A821A8A90428BBF72
:10085000801AC2F5806298829A8201E00029F4D061
:100860001A8A0B48104484F310880A4A998AD3687C
:10087000019302B0BDE81040184784F31088F2F7E6
:1008800017F902B0BDE81040FFF7DEBE10220020CD
:10089000101E002078140108024A00231360024A47
:1008A000136070472C2400202824002010B5EFF39B
:1008B000108472B641B1012903D1064A136803437B
:1008C000136084F3108810BD024A136823EA000302
:1008D000F6E700BF2C24002010B5EFF3108472B6A9
:1008E00041B1012903D1064A13680343136084F31D
:1008F000108810BD024A136823EA0003F6E700BF20
:100900002824002038B5EFF3108572B60A4B0B4C43
:100910001B6833B1236898476368984785F310884C
:1009200038BD074B1B681BB1A3689847E368F4E721
:10093000236998476369F0E72C240020E413010839
:100940002824002001380A44914200D1704711F850
:10095000013B00F8013FF7E700F02CBC10B5EFF3C6
:10096000108472B6064A136803431360054A52F8AE
:100970003130034342F8313084F3108810BD00BF9A
:100980007C2400207424002070477047030C1B0453
:10099000C3B90004102310F07F4F02BF08330002D8
:1009A000DBB210F0704F08BF00014FEA1070064A2A
:1009B00008BF0433125C08BFDBB2C3F11F03981AEF
:1009C000C0B270470023E6E7082501082DE9F84F7B
:1009D000384D394ED5F80080DFF8E0B0DFF8E0A000
:1009E000DFF8E090D6F800C0374FDBF80010374C46
:1009F000DAF80020D9F8003008EA000028602868FA
:100A000000EA020E1EEA0C0F01D019421ED04FF070
:100A1000FF333B60FFF7B8FFEFF3108472B6336823
:100A2000DBF80020DAF800100B4029680B4205D1F2
:100A3000D9F80030134201D1F1F7C4FF84F31088D4
:100A4000FFF7A3FFC5F80080BDE8F88F236823688F
:100A50000340134062681A4204BF4FF0FF326260E5
:100A600060681840FFF792FF62683860012303FA5C
:100A700000F022EA00026260EFF3108172B63A6879
:100A80009340326822EA03023260226822EA0303BA
:100A9000236081F310880E4A3B6852F82330984750
:100AA000D6F800C0DBF80010DAF80020D9F80030E2
:100AB000A5E700BF440100207C240020342400204E
:100AC0004801002038240020302400207424002015
:100AD0003C24002010B51146EFF3108472B6FFF7E6
:100AE00055FF034B43F8201084F3108810BD00BF5E
:100AF0003C24002082B082B00DF1080C0CE9060005
:100B0000BDF8042003930B44BDF810100A4491B2C1
:100B100012B2B2F57A7FA2BFA1F57A72013312B296
:100B20000360828002B002B0704782B082B00DF1E3
:100B3000080C0CE90600BDF804200393CB1ABDF89D
:100B40001010521A91B212B2002ABEBF01F57A7289
:100B500003F1FF3312B20360828002B002B070472B
:100B600030B585B0114D6B4683E803000023029336
:100B7000ADF80C3003A82B699847009BBDF80440E2
:100B80000290181ABDF80C30E41AA3B224B2002C5B
:100B9000BEBF03F57A731CB200F1FF302B68984793
:100BA000AB682046984705B030BD00BF3814010837
:100BB00073B5114E002305460093ADF8043001A82B
:100BC00033699847F36800909847736804469847DC
:100BD000009B1844BDF8043023449AB21BB2B3F50D
:100BE0007A7FA2BF0130A2F57A731BB22860284633
:100BF000AB8002B070BD00BF3814010837B50023C8
:100C00000093ADF80430074B04461B6901A89847D0
:100C10006D46009095E8030084E80300204603B089
:100C200030BD00BF3814010837B50F4D02AB03E9E2
:100C30000300EB6898476B6804469847BDF804309A
:100C4000009A1B1B99B21BB2002BA2EB0002BEBF85
:100C500001F57A7102F1FF320BB24FF47A7000FBAA
:100C6000023003B030BD00BF381401082DE9F04157
:100C70004FF47A75B1FBF5F5C5EB4513DFF83C8011
:100C800005EB8303A1EBC3039CB2D8F80C300646F6
:100C90009847D8F8043007469847E31999B21BB231
:100CA000B3F57A7F2844A2BFA1F57A7301301BB255
:100CB0003060B3803046BDE8F08100BF38140108D1
:100CC000024B00221A60024B1B6818478024002048
:100CD0004C140108F8B50446174608461E467CB178
:100CE00073B1084B00255B6A25609847069B6060DE
:100CF0002581A572E6602361E77265612846F8BD2B
:100D00000120FCE74C14010810B5034CE369984737
:100D1000A36ABDE8104018474C14010870B5064D91
:100D2000EB69064698476B6A044630469847AB6ABB
:100D3000201ABDE8704018474C140108054B1B6889
:100D40000BB918467047834201D05B69F8E7012070
:100D5000704700BF802400202DE9F3410B4E336A19
:100D6000044698470123B7692372D4F800800546EA
:100D7000B8472844804502D2B84728442060B36869
:100D80002068019302B0BDE8F04118474C140108F7
:100D900070B520B3EFF3108672B6124D2B680122A6
:100DA000827253B10022427298425C690ED1027283
:100DB0003CB120462C60FFF7CFFF86F3108800205F
:100DC00070BD094BDB6898472C60F6E71A465B69F3
:100DD000002BF2D09842F9D143695361EDE701202D
:100DE000EEE700BF802400204C140108084B10B52A
:100DF0001A685369516911B95061416110BD0468A5
:100E000019688C4202D91A465B69F3E71946F3E781
:100E100080240020044A13680BB100211972436139
:100E20001060FFF799BF00BF802400202DE9F0413A
:100E3000044600282DD0FFF781FF50BB657A45BBE3
:100E4000EFF3108872B6144E6768336A984787428A
:100E50002CBF27602060114FA5724FF4807323814F
:100E60003B684BB9336998472046FFF7D3FF88F3B7
:100E700010882846BDE8F081B36998472368184474
:100E80003B6820601B6898422046EED3FFF7AEFF18
:100E9000EDE70125EDE700BF4C1401088024002098
:100EA00010B5044608467CB1084B5B6A9847606001
:100EB0002046FFF743FF40B12046FFF769FF204679
:100EC000BDE81040FFF7B2BF012010BD4C1401086F
:100ED0002DE9F041EFF3108772B61D4E1D4D736979
:100EE00098473369044698472B684BB94FF0000880
:100EF0002B688BB9286828BB87F31088BDE8F08180
:100F0000011B241A1A688A428CBF121900221A6027
:100F10005B69002BF6D1E9E71C681CB1B3699847FF
:100F20008442E7D22C6863692B60A4F80880D4E976
:100F3000033098476389B3F5807FD9D12046FFF706
:100F400075FFD5E7037A002BD6D1FFF705FFD3E76E
:100F50004C140108802400202DE9F04F97B000299F
:100F60008046039140F30E819A4604460399137814
:100F7000A4EB0800013923B90023237017B0BDE8A2
:100F8000F08F8842F8DA252B04D004F8013B16468E
:100F9000721CEBE792F801C0ACF13003D3F1000E04
:100FA0004EEB030EACF13003092B02F1010629D8F8
:100FB000324600254FF00A09164612F8013BA3F10C
:100FC0003000092819D93378692B00F09C801CD88F
:100FD000632B28D0642B00F09680582B5BD0252BF8
:100FE00019D13378002B00F0928004F8013BA4EB78
:100FF00008038B4280F28980CAE709FB0533A3F11D
:101000003005D9E74FF0FF35DDE7752B7DD0782B24
:1010100043D0732B1ED0252304F8013BA4EB080317
:101020008B4272DADDE7002D05F1FF39D8BF4FF0B2
:1010300000094A462046202100F0BCF85346A1444E
:10104000002D53F8042B89F80020D8BF01252C442B
:101050009A469DE74C4B5AF8047B002F08BF1F4669
:101060003846F0F7ADF9A5EB000B8542B8BF4FF05D
:10107000000B5A4681462021204600F09BF8A344ED
:1010800000234B4502DB0BEB090481E7FA5C0BF80C
:1010900003200133F5E74EF0400E1020DFF8EC900E
:1010A0003B4F1EF0400F08BF4F465346BCF1300F78
:1010B0000197A4EB08020CBF302720271EF0020F77
:1010C000A1EB0202029753F8041B22D0002920DA78
:1010D0004942013D4FF02D0E05AF0097002789468C
:1010E000DDF804A0B1FBF0F100FB119B48451AF8B4
:1010F0000BB0DDF800A00AF801BB07F10107CDF83D
:1011000000A0ECD90EE04EF0020E0A20C6E7013E28
:101110006DE711B14FF0000EDEE730208DF81400BE
:101120008E460127BCF1300FA5EB070504D0202027
:10113000002D05F1FF3509DCBEF1000F04D02D2193
:10114000013A04F8011B83D025440AE0013A04F86F
:10115000010BEDD17CE7029904F8011B013A3FF441
:1011600077AF291B0029F6DC05A93944224427441E
:10117000A7423FF46DAF11F8010D04F8010B944242
:10118000F6D165E70020F9E6182501081F250108BA
:101190004425010810B501390244904201D10020D4
:1011A00005E0037811F8014FA34201D0181B10BDD0
:1011B0000130F2E702440346934200D1704703F83E
:1011C000011BF9E770B50D4D0D4C641BA4100026F2
:1011D000A64209D10B4D0C4C00F0B2F8641BA410D0
:1011E0000026A64205D170BD55F8043B984701364C
:1011F000EEE755F8043B98470136F2E74C26010824
:101200004C2601084C2601085026010800F003B8BE
:10121000002200F00EB80A44914200F1FF3300D1E1
:10122000704710B511F8014B03F8014F9142F9D105
:1012300010BD13460A461946FFF7BCBF0000000068
:10124000C1F30A522DE9F843A2F2FF36132E0B46E2
:1012500007460C46054632DC002E14DA34A3D3E9E7
:101260000023F0F7BBF800220023F0F7EBFA38B1C7
:10127000002C56DA24F00044254355D02E4C00258E
:1012800023462F4625E02D4A42FA06F801EA0802D5
:1012900002431ED026A3D3E90023F0F79FF80022D3
:1012A0000023F0F7CFFA0028EAD0002CBEBF4FF49D
:1012B00080133341E41824EA08040025E0E7332EC4
:1012C0000BDDB6F5806F04D10246F0F787F80746CC
:1012D0000B4638461946BDE8F883A2F213424FF098
:1012E000FF3828FA02F810EA080FF2D010A3D3E969
:1012F0000023F0F773F800220023F0F7A3FA002888
:10130000BED0002C0ADA142E01D1013406E0C6F159
:1013100034060123B3401D44AF42F6D825EA080540
:10132000AEE700252C46ABE74FF00044A8E700BF2E
:101330009C7500883CE4377E0000F0BFFFFF0F0083
:10134000F8B500BFF8BC08BC9E467047F8B500BFB2
:08135000F8BC08BC9E46704782
:101358000000000001000000020000000000000082
:101368008813000010270000204E00003075000090
:10137800409C000050C3000060EA0000C0D4010097
:1013880080A903000053070000EA063700000000A8
:101398005000000040F7093700000000500000002E
:1013A800C194C10000000000B22700000000000046
:1013B8000000000000000000000000000000000025
:1013C80000000000B5010008F1010008CC13010875
:1013D800FC7F003F00350113C41200087327000882
:1013E800552700083927000859270008352700081D
:1013F800852700080D0A484D4143205665726966E5
:10140800792053756363657373203D202575200D1E
:101418000A005975336E3148344F3152354E3953BD
:1014280032543653256473253033643A0000000083
:10143800752C0008152D0008852C0008212D0008A2
:10144800E52C00082D2D000800000000952C000850
:101458004D2C0008192C0008D12B0008292C000855
:101468003D2C0008DD2B0008E12B0008F52B0008B7
:10147800D52F0008FD2F0008812F00086D2F0008C8
:10148800496E697469616C20414320434F4445208B
:10149800626C616E6B2E2E2E200D0A005354535F22
:1014A800534552564943455F4D41534B3A256420B5
:1014B8000D0A000D0A202D2D2D2D2D2D2D2D2D2D14
:1014C8002D2D2D2D2D2D2D2D2D5246414320507281
:1014D8006F636573730D0A0052464143000D0A207D
:1014E8002D2D2D2D2D2D2D2D2D2D2D2D2D2D2D2D24
:1014F8002D2D2D5665726966792052464143205339
:10150800756363657373206F72204E6F740D0A00E4
:1015180053776974636820746F20436C6173732018
:10152800256320646F6E650D0A0041424300414205
:1015380050004F544141000D0A2323232323232025
:101548003D204A4F494E4544203D2000414250200D
:101558003D3D3D3D3D3D3D3D3D3D3D3D3D3D3D3DB3
:101568003D3D3D3D3D3D0D0A004F544141203D3D2F
:101578003D3D3D3D3D3D3D3D3D3D3D3D3D3D3D3D93
:101588003D3D3D0D0A000D0A205354535F4C6F52E8
:10159800615F57414E5F4A6F696E6564203D202543
:1015A80073200D0A000D0A232323232323203D2023
:1015B8004A4F494E204641494C45440D0A002323D1
:1015C8002323232320552F4C204652414D453A4A88
:1015D8004F494E207C2044523A2564207C205057A5
:1015E800523A25640D0A000D0A2054785065726934
:1015F8006F646963697479206368616E67656420E4
:10160800746F20257520286D73656329200D0A00E5
:101618002A2A2A2A2A2A2A2A2A2A2A2A2A2A2A2A22
:1016280020486561727442656174506572696F64BF
:101638006963697479204368616E67656420746FB3
:101648003A20257520286D73290D0A004C6D4861D4
:101658006E646C65722053746F70206F6E20676FB4
:10166800696E67202E2E2E0D0A004C6D48616E643F
:101678006C65722053746F707065640D0A004C6D50
:1016880048616E646C65722073776974636820744E
:101698006F20414250206D6F64650D0A0053454E1E
:1016A8004420524551554553540D0A004E657874EF
:1016B80020547820696E20203A207E2564207365A6
:1016C800636F6E642873290D0A000D0A23232323F0
:1016D800232320424541434F4E204C4F53540D0A7B
:1016E800000D0A23232323232320424541434F4E41
:1016F800205245434549564544207C2044523A25CA
:1017080064207C20525353493A2564207C20534E50
:10171800523A2564207C2046513A2564207C205486
:10172800494D453A2564207C20444553433A256475
:10173800207C20494E464F3A3032582530325825C1
:10174800303258202530325825303258253032581A
:101758000D0A000D0A232323232323204245414356
:101768004F4E204E4F542052454345495645440D4F
:101778000A004E564D20444154412053544F52457F
:10178800440D0A004E564D204441544120524553C1
:10179800544F5245440D0A004E41434B000D0A2355
:1017A8002323232323203D3D3D3D3D3D3D3D3D3D00
:1017B800204D4350532D436F6E6669726D203D3D39
:1017C8003D3D3D3D3D3D3D3D3D3D3D0D0A00232315
:1017D8002323232320552F4C204652414D453A259B
:1017E800303464207C20504F52543A2564207C20A9
:1017F80044523A2564207C205057523A25640020F0
:101808007C204D534720545950453A00434F4E468B
:1018180049524D4544205B25735D0D0A00554E43E2
:101828004F4E4649524D45440D0A004E564D2044F0
:1018380041544120555020544F20444154450D0AED
:10184800004E564D20444154412053544F52452098
:101858004641494C45440D0A00232320425554541F
:101868004F4E2D312044455445435445443A202099
:10187800253264200D0A005056585858000D0A4960
:101888006E697469616C20426F6F7420776974683F
:1018980020456D70747920436F6E6669672C204609
:1018A8006C61736820776974682064656661756C1B
:1018B8007420636F6E6669672E2E2E2E0D0A000D3A
:1018C8000A0A0A23232323232059554E484F524EF0
:1018D8005F5354535F46573A25642053575625643F
:1018E800204857563A2564204D544D3A25642E25F4
:1018F8006420523A25642E25642E25642023232350
:10190800230D0A0A0A004150504C49434154494F9B
:101918004E5F56455253494F4E3A205625582E256C
:10192800582E25580D0A004D575F4C4F52415741CC
:101938004E5F56455253494F4E3A20205625582E51
:1019480025582E25580D0A004D575F524144494FDE
:101958005F56455253494F4E3A202020205625586D
:101968002E25582E25580D0A004C325F53504543FA
:101978005F56455253494F4E3A2020202020562585
:10198800582E25582E25580D0A0052505F535045A1
:10199800435F56455253494F4E3A20202020205647
:1019A80025582D25582E25582E25580D0A00215921
:1019B800756E486F726E205354532052657669765F
:1019C8006521000D0A2059756E686F726E20535498
:1019D80053204E6F646520526576697665202E2EF9
:1019E8002E200D0A003E3E3E3E3E3E3E3E3E3E3EE0
:1019F8003E3E3E3E3E3E3E3E3E3E204D61736B20A7
:101A08003D205B2025303278205D200D0A002323FD
:101A1800232323232059554E484F524E2050657298
:101A2800696F646963697479204368616E67656486
:101A380020746F205B202564205D205365636F6EE2
:101A480064730D0A002323232323232059554E486A
:101A58004F524E2053616D706C696E67204F722033
:101A680048656172742D4265617420496E746572AF
:101A780076616C204368616E67656420746F205BD3
:101A8800202564205D205365636F6E64730D0A0022
:101A98000D0A20746C765F627566202564203D20EF
:101AA80025303278206366672D3E705B25645D3D86
:101AB80025303278200D0A002323232323232052A4
:101AC80053532053696D706C65204346473D257319
:101AD8000D0A004C4544204F46460D0A004C45442B
:101AE800204F4E0D0A0023232323232320442F4C69
:101AF800204652414D453A25303464207C20504FD1
:101B080052543A2564207C2044523A2564207C2093
:101B1800534C4F543A2573207C20525353493A254D
:101B280064207C20534E523A25640D0A003100325D
:101B380000435F4D4300505F4D430000351B0108D3
:101B4800371B0108E3140108391B0108381501087F
:101B58003E1B01084D454D532049443D2530327800
:101B68002025303278200D0A000000000100000016
:101B78000300000005000000010000000100000053
:101B8800060000000A00000020000000020000001B
:101B980004000000080000001000000040000000E1
:101BA80080000000000100000002000000000000AA
:101BB800000000000000000000000000010000001C
:101BC800020000000300000004000000A0860100DD
:101BD800400D0300801A060000350C0040420F003B
:101BE80080841E0000093D0000127A000024F400E1
